:020000040000FA
:1000000000040020810A000015070000610A0000BA
:100010001F07000029070000330700000000000050
:10002000000000000000000000000000A50A000021
:100030003D070000000000004707000051070000D6
:100040005B070000650700006F07000079070000EC
:10005000830700008D07000097070000A10700003C
:10006000AB070000B5070000BF070000C90700008C
:10007000D3070000DD070000E7070000F1070000DC
:10008000FB070000050800000F0800001908000029
:10009000230800002D080000370800004108000078
:1000A0004B080000550800005F08000069080000C8
:1000B000730800007D080000870800009108000018
:1000C0009B080000A5080000AF080000B908000068
:1000D000C3080000CD080000D7080000E1080000B8
:1000E000EB080000F5080000FF0800000909000007
:1000F000130900001D090000270900003109000054
:100100003B0900001FB500F003F88DE80F001FBD8C
:1001100000F0ACBC40F6FC7108684FF01022401CA7
:1001200008D00868401C09D00868401C04D0086842
:1001300000F037BA9069F5E79069F9E7704770B554
:100140000B46010B184400F6FF70040B4FF0805073
:100150000022090303692403406943431D1B104621
:1001600000F048FA29462046BDE8704000F042BA47
:10017000F0B54FF6FF734FF4B4751A466E1E11E0DA
:10018000A94201D3344600E00C46091B30F8027B3B
:10019000641E3B441A44F9D19CB204EB134394B25D
:1001A00004EB12420029EBD198B200EB134002EBB2
:1001B000124140EA0140F0BDF34992B00446D1E952
:1001C0000001CDE91001FF224021684600F0F4FB58
:1001D00094E80F008DE80F00684610A902E004C8FB
:1001E00041F8042D8842FAD110216846FFF7C0FF7C
:1001F0001090AA208DF8440000F099F9FFF78AFFCB
:1002000040F6FC7420684FF01025401C0FD0206889
:1002100010226946803000F078F92068401C08D030
:100220002068082210A900F070F900F061F9A869AF
:10023000EEE7A869F5E74FF080500369406940F6A2
:10024000FC71434308684FF01022401C06D0086838
:1002500000F58050834203D2092070479069F7E788
:100260000868401C04D00868401C03D00020704778
:100270009069F9E70420704770B504460068C34DE3
:10028000072876D2DFE800F033041929631E250021
:10029000D4E9026564682946304600F062F92A46CE
:1002A0002146304600F031F9AA002146304600F0E0
:1002B00057FB002800D0032070BD00F009FC4FF46C
:1002C000805007E0201D00F040F90028F4D100F034
:1002D000FFFB60682860002070BD241D94E80700C3
:1002E000920000F03DFB0028F6D00E2070BDFFF715
:1002F000A2FF0028FAD1D4E901034FF0805100EBAE
:10030000830208694D69684382420ED840F6F8704E
:1003100005684FF010226D1C09D0056805EB8305B8
:100320000B6949694B439D4203D9092070BD55694A
:10033000F4E70168491C03D00068401C02D003E0C8
:100340005069FAE70F2070BD2046FFF735FFFFF731
:1003500072FF0028F7D1201D00F0F7F80028F2D135
:1003600060680028F0D100F0E2F8FFF7D3FE00F05B
:10037000BFF8072070BD10B50C46182802D0012028
:10038000086010BD2068FFF777FF206010BD41684E
:10039000054609B1012700E0002740F6F8742068FF
:1003A0004FF01026401C2BD02068AA68920000F065
:1003B000D7FA38B3A86881002068401C27D020688D
:1003C000FFF7BDFED7B12068401C22D026684FF051
:1003D0008050AC686D68016942695143A9420DD9EA
:1003E000016940694143A14208D92146304600F0E5
:1003F000B8F822462946304600F087F800F078F831
:100400007069D2E700F093F8FFF784FEF6E77069B1
:10041000D6E77669DBE740F6FC7420684FF01026DB
:10042000401C23D02068401C0CD02068401C1FD0EA
:100430002568206805F18005401C1BD027683879A5
:10044000AA2819D040F6F8700168491C42D001680A
:10045000491C45D00168491C3ED001680968491C07
:100460003ED00168491C39D000683EE0B069DAE747
:10047000B569DEE7B769E2E710212846FFF778FEA5
:100480003968814222D12068401C05D0D4F8001080
:1004900001F18002C03107E0B169F9E730B108CA63
:1004A00051F8040D984201D1012000E000208A4259
:1004B000F4D158B1286810B1042803D0FEE72846CB
:1004C000FFF765FF3149686808600EE0FFF722FE1C
:1004D00000F00EF87169BBE77169BFE7706904E06D
:1004E0004FF480500168491C01D000F0CBFAFEE7C0
:1004F000BFF34F8F26480168264A01F4E06111439B
:100500000160BFF34F8F00BFFDE72DE9F0411746B3
:100510000D460646002406E03046296800F054F8EF
:10052000641C2D1D361DBC42F6D3BDE8F08140F69B
:10053000FC700168491C04D0D0F800004FF48051D1
:10054000FDE54FF010208069F8E74FF080510A690F
:10055000496900684A43824201D810207047002050
:10056000704770B50C4605464FF4806608E0284693
:1005700000F017F8B44205D3A4F5806405F5805562
:10058000002CF4D170BD0000F40A0000000000202F
:100590000CED00E00400FA05144801680029FCD0C5
:1005A0007047134A0221116010490B68002BFCD0E0
:1005B0000F4B1B1D186008680028FCD0002010603D
:1005C00008680028FCD07047094B10B501221A605A
:1005D000064A1468002CFCD0016010680028FCD08A
:1005E0000020186010680028FCD010BD00E4014015
:1005F00004E5014070B50C46054600F073F810B9EB
:1006000000F07EF828B121462846BDE8704000F091
:1006100007B821462846BDE8704000F037B8000012
:100620007FB5002200920192029203920A0B000B06
:100630006946012302440AE0440900F01F0651F80C
:10064000245003FA06F6354341F82450401C8242F8
:10065000F2D80D490868009A10430860081D016827
:10066000019A1143016000F03DF800280AD00649C4
:1006700010310868029A10430860091D0868039A3F
:10068000104308607FBD00000006004030B50F4CED
:10069000002200BF04EB0213D3F800582DB9D3F8A1
:1006A000045815B9D3F808581DB1521C082AF1D3C3
:1006B00030BD082AFCD204EB0212C2F80008C3F8CD
:1006C00004180220C3F8080830BD000000E0014013
:1006D0004FF08050D0F83001082801D0002070473A
:1006E000012070474FF08050D0F83011062905D016
:1006F000D0F83001401C01D0002070470120704725
:100700004FF08050D0F830010A2801D00020704707
:100710000120704708208F490968095808471020B0
:100720008C4909680958084714208A4909680958FA
:100730000847182087490968095808473020854923
:100740000968095808473820824909680958084744
:100750003C20804909680958084740207D490968BC
:100760000958084744207B49096809580847482028
:1007700078490968095808474C207649096809589A
:10078000084750207349096809580847542071499F
:1007900009680958084758206E49096809580847E8
:1007A0005C206C4909680958084760206949096854
:1007B00009580847642067490968095808476820AC
:1007C00064490968095808476C2062490968095852
:1007D000084770205F4909680958084774205D4937
:1007E00009680958084778205A490968095808478C
:1007F0007C205849096809580847802055490968EC
:10080000095808478420534909680958084788202F
:1008100050490968095808478C204E490968095809
:10082000084790204B4909680958084794204949CE
:10083000096809580847982046490968095808472F
:100840009C204449096809580847A0204149096883
:1008500009580847A4203F49096809580847A820B3
:100860003C49096809580847AC203A4909680958C1
:100870000847B0203749096809580847B420354966
:10088000096809580847B8203249096809580847D3
:10089000BC203049096809580847C0202D4909681B
:1008A00009580847C4202B49096809580847C82037
:1008B0002849096809580847CC2026490968095879
:1008C0000847D0202349096809580847D4202149FE
:1008D000096809580847D8201E4909680958084777
:1008E000DC201C49096809580847E02019490968B3
:1008F00009580847E4201749096809580847E820BB
:100900001449096809580847EC2012490968095830
:100910000847F0200F49096809580847F4200D4995
:10092000096809580847F8200A490968095808471A
:10093000FC2008490968095808475FF48070054998
:10094000096809580847000003480449024A034B54
:100950007047000000000020000B0000000B0000AA
:1009600040EA010310B59B070FD1042A0DD310C82C
:1009700008C9121F9C42F8D020BA19BA884201D97E
:10098000012010BD4FF0FF3010BD1AB1D30703D0C6
:10099000521C07E0002010BD10F8013B11F8014B7C
:1009A0001B1B07D110F8013B11F8014B1B1B01D198
:1009B000921EF1D1184610BD02F0FF0343EA032254
:1009C00042EA024200F005B87047704770474FF0A6
:1009D00000020429C0F0128010F0030C00F01B800C
:1009E000CCF1040CBCF1020F18BF00F8012BA8BF1A
:1009F00020F8022BA1EB0C0100F00DB85FEAC17CDE
:100A000024BF00F8012B00F8012B48BF00F8012B90
:100A100070474FF0000200B51346944696462039C1
:100A200022BFA0E80C50A0E80C50B1F12001BFF4A7
:100A3000F7AF090728BFA0E80C5048BF0CC05DF80D
:100A400004EB890028BF40F8042B08BF704748BF5B
:100A500020F8022B11F0804F18BF00F8012B7047CF
:100A6000014B1B68DB6818470000002009480A4951
:100A70007047FFF7FBFFFFF745FB00BD20BFFDE719
:100A8000064B1847064A1060016881F308884068E1
:100A900000470000000B0000000B000017040000DE
:100AA000000000201EF0040F0CBFEFF30881EFF3ED
:100AB0000981886902380078182803D100E0000015
:100AC000074A1047074A12682C3212681047000084
:100AD00000B5054B1B68054A9B58984700BD0000B0
:100AE0007703000000000020F00A0000040000006E
:100AF000001000000000000000FFFFFF0090D00386
:100FF80000F002000000000000FFFFFF0090D00397
:10100000D80C00206586010069900000CB850100A6
:1010100069900000699000006990000000000000E5
:10102000000000000000000000000000C186010078
:1010300069900000000000006990000069900000C5
:10104000298701002F870100699000006990000046
:1010500069900000699000006990000069900000AC
:101060003587010069900000699000003B8701000E
:101070006990000041870100478701004D8701000A
:10108000699000006990000069900000699000007C
:10109000699000006990000069900000699000006C
:1010A000699000005387010069900000699000007A
:1010B000699000006990000069900000699000004C
:1010C0005987010069900000699000006990000054
:1010D000699000006990000069900000699000002C
:1010E000699000006990000069900000699000001C
:1010F000699000006990000069900000699000000C
:10110000699000006990000000F002F817F099FA69
:101110000AA090E8000C82448344AAF10107DA4552
:1011200001D117F08EFAAFF2090EBAE80F0013F0F2
:10113000010F18BFFB1A43F001031847807A010022
:10114000A07A01000A4410F8014B14F00F0508BF03
:1011500010F8015B240908BF10F8014B6D1E05D083
:1011600010F8013B6D1E01F8013BF9D1641E03D05C
:10117000641E01F8015BFBD19142E4D3704700008B
:101180000023002400250026103A28BF78C1FBD890
:10119000520728BF30C148BF0B6070471FB500F031
:1011A00031F88DE80F001FBDF0B440464946524665
:1011B0005B460FB402A0013001B50648004700BFEE
:1011C00001BC86460FBC8046894692469B46F0BCD1
:1011D00070470000091100008269034981614FF0E6
:1011E0000100104470470000ED11000001B41EB46E
:1011F00000B510F03DFA01B40198864601BC01B07B
:101200001EBD000017F01ABA70B51B4C0546092028
:101210002070A01C00F0D3F85920A0802946204659
:10122000BDE8704006F0D0BD06F0D9BD70B50C46E3
:101230001249097829B1A0F160015E2908D3012083
:1012400013E0602804D0692802D043F201000CE0CA
:1012500020CC0B4E94E80E0006EB8000A0F58050E9
:10126000241FD0F8806E2846B047206070BD012052
:10127000704706207047000008000020180000207A
:10128000888701003249884201D20120704700203E
:10129000704770B50446A0F500002E4EB0F1786F8F
:1012A00002D23444A4F500042948844201D2012525
:1012B00000E0002500F043F848B125B9B44204D35A
:1012C0002548006808E0012070BD002070BD002D99
:1012D000F9D1B442F9D321488442F6D2F3E710B5EC
:1012E0000446A0F50000B0F1786F03D21948044419
:1012F000A4F5000400F023F84FF0804130B1164807
:10130000006804E08C4204D2012003E013488442C8
:10131000F8D2002080F0010010BD10B520B1FFF719
:10132000DEFF08B1012010BD002010BD10B520B1B6
:10133000FFF7AFFF08B1012010BD002010BD084825
:1013400008490068884201D1012070470020704799
:1013500000900100000000201C0000200800002078
:101360004C000020BEBAFECA10B504460021012080
:1013700000F032F800210B2000F02EF80421192093
:1013800000F02AF804210D2000F026F804210E2098
:1013900000F022F804210F2000F01EF80421C843B9
:1013A00000F01AF80621162000F016F80621152084
:1013B00000F012F82046FFF727FF002010BDB821EB
:1013C00001807047FFF730BF002070470A48704720
:1013D000FFF72CBF704770474907090E002804DB50
:1013E00000F1E02080F80014704700F00F0000F1D9
:1013F000E02080F8141D704703F9004230B5FF4D1E
:101400000446062CA9780ED2DFE804F0030E0E0E77
:101410000509FFDF08E0022906D0FFDF04E0032909
:1014200002D0FFDF00E0FFDFAC7030BDF34810B545
:10143000407E4108F14800F11A0005D00BF0D7FBBF
:10144000BDE8104006F04ABB0BF0B8FBF8E730B53A
:101450000446A1F120000D460A2847D2DFE800F03B
:1014600005070C19202532373C41FFDF3FE020788B
:1014700020283CD1FFDF3AE0E0488078052836D0CC
:101480002078242833D0252831D023282FD0FFDFFF
:101490002DE0207822282AD0232828D8FFDF26E034
:1014A0002078222823D0FFDF21E0207822281ED0B8
:1014B00024281CD026281AD0272818D0292816D04E
:1014C000FFDF14E02078252811D0FFDF0FE020781F
:1014D00025280CD0FFDF0AE02078252807D0FFDF81
:1014E00005E02078282802D0FFDF00E0FFDF25702C
:1014F00030BD1FB50022ADF800200C88ADF80240C9
:101500004B88ADF80430CA88ADF808208988ADF85A
:1015100006100021ADF80A10ADF80C1080B14FF69E
:10152000FF700621844201D1ADF80210834201D13F
:10153000ADF80410824203D14FF44860ADF80800C2
:1015400068460BF071FC06F0C9FA04B010BD70B526
:1015500014460D460646FFF79CFE60B90DB1A54244
:1015600001D90C2070BD002409E000BF56F824000A
:10157000FFF78FFE08B1102070BD641CE4B2AC42CE
:10158000F4D3002070BD2DE9F04105461F4690467A
:101590000E4600240068FFF7C9FE30B9A988286804
:1015A0000844401EFFF7C2FE10B11020BDE8F081D4
:1015B00028680028A88802D0B84202D850E0002845
:1015C000F4D00920F2E72968085DB8B1671CCA5D4C
:1015D000152A2ED03CDC152A3AD2DFE802F0391267
:1015E000222228282A2A31313939393939393939E9
:1015F00039392200085D30BB641CA4B2A242F9D87C
:1016000033E00228DDD1A01C085C88F80000072820
:1016100001D2400701D40A20C8E7307840F0010029
:1016200015E0C143C90707E0012807D010E00620F4
:10163000BCE70107A1F180510029F5D01846B5E7B4
:101640003078810701D50B20B0E740F00200307000
:101650002868005D384484B2A888A04202D2B0E76E
:101660004FF4485382B2A242ADD800209EE710B595
:101670000278540809D0012243F20223012C07D03A
:10168000022C0DD0032C13D10FE00020087005E0D0
:1016900080790324B4EB901F0AD10A70002010BD9A
:1016A0008079B2EB901F03D1F7E780798009F4D0FD
:1016B000184610BD08B500208DF800004F4890F87E
:1016C000221051B190F8230002280FD003280FD028
:1016D000FFDF00BF9DF8000008BD4848694619308B
:1016E00001F095F80028F5D0FFDFF3E7032000E0D4
:1016F00001208DF80000EDE738B50C460546694637
:1017000001F085F800280DD19DF80010207861F3D4
:101710004700207055F8010FC4F80100A888A4F80C
:101720000500002038BD38B51378C0B1022816D0A6
:1017300033A46D46246800944C7905EB9414247806
:1017400064F34703137003280ED003F0FE001070FB
:101750000868C2F801008888A2F8050038BD23F0A7
:10176000FE0313700228EED1D8B240F00100EEE77C
:1017700002210CF095BC38B50C460978222901D21B
:10178000082038BDADF800008DF8022068460BF047
:101790006DFA06F0A3F9050003D121212046FFF7D9
:1017A00056FE284638BD1CB500208DF80000CDF847
:1017B0000100ADF80500114890F82200022801D080
:1017C000012000E000208DF8070068460BF0BCFA0D
:1017D000002800D0FFDF1CBD2DE9FF478CB000259D
:1017E000BDF8346082461C4690468DF81C50700748
:1017F00003D56068FFF74DFD90B903E0A401002018
:101800000302FF01FD4F4FF0010997F8220058B184
:1018100097F82300022807D16068FFF787FD18B109
:10182000102010B0BDE8F087300702D5A0898028CD
:1018300015D8700704D4B8F1000F01D0387E70B10C
:10184000E07DC0F300108DF81B00617D072041B1E1
:10185000012906D00229E4D00429E2D117E00720AB
:10186000DFE78DF817908DF819908DF81580606876
:1018700078B107A9FFF7FBFE0028D2D1606850F8C5
:10188000011FCDF80F108088ADF8130005E0062089
:10189000C7E7CDF80F50ADF81350E07B0028F6D124
:1018A000207C0028F3D1607C0028F0D1A07C0028A7
:1018B000EDD1E07CC006EAD18DF800A0BDF834007F
:1018C000ADF80200A0680190A0680290CCA0D0E919
:1018D0000010CDE90A10E07C0AA901EB5010007855
:1018E0008DF80C00FFF7E6FE8DF80D009DF81C004A
:1018F0008DF80E008DF818508DF816508DF81A508E
:1019000009A968460BF0DFFA06F0E8F889E7F0B5B8
:101910008FB000248DF830408DF814408DF834409D
:1019200006468DF82840019402940394049419B15A
:101930000FC901AD85E80F00B04DA878052801D08A
:1019400004280CD101986968884200D120B9039815
:10195000E968884203D110B108200FB0F0BD1F27FD
:101960003B460DAA05A903A8FFF70DFE0028F4D1F8
:101970003B460AAA0CA901A8FFF705FE0028ECD1F6
:101980009DF81400C00701D00A20E6E7A88A4107A5
:1019900008D4A97D31B19DF82810890702D043F2FF
:1019A0000120DAE79DF82810C90709D0400707D4BD
:1019B000288818B144F25061884201D90720CCE749
:1019C0008DF818408DF81960BDF80800ADF81A00C0
:1019D0000198079006A80BF090FA06F07FF800280F
:1019E000BBD18DF820408DF82160BDF81000ADF816
:1019F00022000398099008A80BF09EFA06F06EF8F2
:101A00000028AAD101AC2D1D94E80F0085E80F0035
:101A10000020A2E72DE9FE43040000D1FFDF20787B
:101A2000764E20F00F00801C20F0F0007030207007
:101A300060680178C91F122929D2DFE801F04BE85C
:101A40002809E8E838E7282864E7E62828E7E7E5F2
:101A500086883046FFF78CFE0546304609F0A0FD2B
:101A6000B8B16068807985F83E0021212846FFF7EB
:101A7000EEFC304603F0FBF9304604F0A9FB31469A
:101A8000012010F02FF8A87F20F01000A877BDE803
:101A9000FE83207820F0F000203020700320207298
:101AA000668060688079607206F00FFADDE78588ED
:101AB0002846FFF75DFE00B9FFDF606880780128E7
:101AC00000D0FFDF6068817903B02846BDE8F043AD
:101AD00009F098BE86883046FFF74AFE050000D11F
:101AE000FFDF06F0F2F960683146C088288160683F
:101AF0000089688160684089A88101200FF0F2FFA9
:101B00000020A875C3E780780228C0D000B1FFDFAD
:101B100006F0DBF96568A879AD1C00B9FFDFF7783E
:101B2000B5F80290B046384605F078FF060000D1BF
:101B3000FFDF0022022148460CF0A9FA040000D180
:101B4000FFDF22212046FFF782FCA17F012060F306
:101B50000101A177298B2181698B6181A98BA181E9
:101B600084F822708DF8080002AA032148460CF080
:101B70008EFA00B9FFDFB088ADF80400B0788DF8B8
:101B8000060001AA052148460CF081FA00B9FFDFE2
:101B9000B088ADF80000F0788DF802006A460421A4
:101BA00048460CF074FA00B9FFDF062105F1120077
:101BB00000F04AFE08B36879800700D5FFDF697935
:101BC000E07D61F34700E075D5F80600A061688903
:101BD000A083062105F10C0000F036FE10B398F842
:101BE00019104A08617862F347016170D8F81A1039
:101BF000C4F80210B8F81E001DE009E0A40100209E
:101C000007060504030201001FE02AE025E017E0B3
:101C1000E07D20F0FE00801CE075D5F81200A06188
:101C2000E88AD5E7607820F0FE00801C6070E868E4
:101C3000C4F80200288AE0800320FFF7DFFB26E7D4
:101C40002046BDE8FE4301F0A0BC06F03EF916F8C0
:101C5000240F40F00400307019E7BDE8FE4306F0A1
:101C600034B9B178052908D00429E8D106F02DF956
:101C70000220BDE8FE43FFF7C1BB80780028DED01C
:101C8000F07800F0ABFD06F020F90320F1E72DE934
:101C9000F047054600780027000991460C463E466D
:101CA000012874D0022873D007280AD00A2825D02A
:101CB000FFDF00BFA9F800600CB12780668000201C
:101CC000B0E5D5F804C0DFF8B4874FF0010A9CF8FE
:101CD00000004FF6FF7113287AD008DC07280ED0D9
:101CE0000E281FD0112826D0122806D186E01628EB
:101CF0000BD0172859D018286CD02146FBE01227AA
:101D00001026BCF804002146B8E01C270A26ECB3D4
:101D1000BCF80200A0806868007920726868407989
:101D20006072C7E71B27092684B303202072686806
:101D30004088A080BEE79CF802003C28BAD010275B
:101D40002C260CF1020C0CB3BCF80200A080BCF8ED
:101D500018006082BCF818002082BCF81A00A0822B
:101D6000BCF81C00E0829CF8050004F108020CF1AC
:101D70000601FFF7D8FC9CF8040001289AD184F8EA
:101D80000FA00020207608F1040002E00AE06DE0D8
:101D900077E090E80E00D8F81000C4E90930C4E9F3
:101DA000071287E7A9F8006089E720271126002C91
:101DB000F8D0A180686804F10A028078207268680F
:101DC000807A60726968C878091DFFF7ACFC71E71A
:101DD00029E0FFE721270A26002CE3D0BCF8020007
:101DE000A08068680079207268684079607298F80D
:101DF000241021F0040188F824105BE722270B2629
:101E0000002CCFD0BCF80400A080686880782072D5
:101E10006868807900F027FD60726868C07900F01A
:101E200022FDA07246E726271C26002CBAD0A180EE
:101E30006868C078607268688079A07208F10400F0
:101E400090E80E00D8F81000C4E90530C4E9031288
:101E5000686880783C2803D0432804D0FFDF29E756
:101E600084F808A026E70220207223E7287A0228B7
:101E700001D0FFDF1EE712271026688800F0D1FC92
:101E800018E7287AB0B3012835D0022833D00328C8
:101E900001D0FFDF0EE711270926002C82D0B5F80C
:101EA00002804046FFF764FC90F822A0A4F804806A
:101EB000687A2072042140460CF004F9052140465E
:101EC0000CF000F9002140460CF0FCF801214046DE
:101ED0000CF0F8F8032140460CF0F4F802214046DB
:101EE0000CF0F0F8062140460CF0ECF8504600F0FB
:101EF00075FCDFE6FFE72846BDE8F04701F07CBC53
:101F000070B5012801D0FFDF70BD8DB22846FFF704
:101F10002FFC040000D1FFDF20782128F4D005F049
:101F2000D1FF80B1017821F00F01891C21F0F0016F
:101F3000103101700221017245800020A075BDE8BA
:101F4000704005F0C2BF21462846BDE8704013220C
:101F500011E42DE9F04116460C00804600D1FFDF68
:101F6000307820F00F00801C20F0F000103030702E
:101F70002078022802D0FFDFBDE8F0814046FFF75D
:101F8000F7FB050000D1FFDF61884FF6FF700027E7
:101F9000814202D1A288824203D0814201D1A0882D
:101FA00048B105F092FF2068B0606068F060208959
:101FB0003082AF75E0E7A87D0128DDD178230022CB
:101FC00041460FF0E5FC0220A875D5E738B5054677
:101FD0000C460846FFF75DF968B9203D062D30D262
:101FE000DFE805F00305222F271B062038BD6068B7
:101FF000FFF793F908B1102038BD618820886A4640
:102000000BF0F0F805F06AFD0028F5D161680029B1
:10201000F2D0BDF800200A8038BDA07800F00101A0
:1020200020880BF010F908E02068BDE8384001F086
:1020300018BE618820880BF06EF8BDE8384005F0C6
:102040004DBD072038BD70B505460C460846FFF764
:1020500046F908B1102070BD202D07D0212D0DD0DC
:10206000222D0BD0252D09D0072070BD2088A11C62
:102070000AF050FEBDE8704005F030BD062070BD8E
:10208000FE481930704708B52821FC4816F075FA4B
:102090000120FFF7B3F9F94968461A3105F0A8FEA7
:1020A000F6489DF80020417E62F3470121F00101CE
:1020B0004176002180F822104FF4617101840221E1
:1020C00080F82310FFF7B2F900B1FFDF00F0FCFB4E
:1020D00001F02EFA08BD10B50C464021204616F03E
:1020E0002AFAA07F20F00300A07720202070002093
:1020F000A07584F8230010BD70472DE9FC41074608
:10210000FFF7C7F810B11020BDE8FC81DB4E06F1E7
:102110001901D6F819000090B6F81D50ADF804501A
:10212000F47F8DF806403846FFF7E6FA0028EBD139
:10213000FFF77CF90028E7D0009946F8191FB58011
:10214000B471E1E710B50446FFF7C9F808B11020F3
:1021500010BDCA48C9492246407E1A314008FFF7DF
:10216000E2FA002010BD3EB504460D460846FFF7D2
:10217000B6F808B110203EBD14B143F204003EBDD4
:10218000BE488078052803D0042801D008203EBD31
:10219000694602A809F0B3FD2A4669469DF8080081
:1021A000FFF7C1FA00203EBDFEB50D4604004FF01A
:1021B000000712D00822FFF7CAF9002812D1002622
:1021C00009E000BF54F826006946FFF750FA0028DE
:1021D00008D1761CF6B2AE42F4D30AF047FC10B137
:1021E00043F20320FEBDA54E3776FCB100271AE06E
:1021F00054F8270002A9FFF73AFA00B1FFDF9DF873
:1022000008008DF8000054F8270050F8011FCDF8A1
:1022100001108088ADF8050068460AF04CFC00B15A
:10222000FFDF7F1CFFB2AF42E2D335760020FEBD58
:102230002DE9F0478AB01546894604001DD00F46A7
:1022400008222946FFF783F9002810D1002612E062
:1022500054F826006946103000F0D9FA002806D15B
:102260003FB157F82600FFF714F810B110200AB05C
:1022700026E5761CF6B2AE42EAD30026A5F10108A7
:102280001CE000BF06F1010A0AF0FF0712E000BFE0
:1022900054F82600017C4A0854F827100B7CB2EB56
:1022A000530F05D106221130113116F099F858B1AB
:1022B0007F1CFFB2AF42EBD30AF0FF064645E1DBDD
:1022C0004E4624B1012003E043F20520CFE7002071
:1022D0000AF010FC10B90AF019FC10B143F2042006
:1022E000C5E75CB300270DF1170825E054F8270077
:1022F0006946103000F08BFA00B1FFDF54F8270078
:10230000102250F8111FCDF801108088ADF805009B
:1023100054F827100DF1070016F08EF896B156F814
:1023200027101022404616F087F868460AF0A8FBEE
:1023300000B1FFDF7F1CFFB2AF42D7D3FFF733FA04
:10234000002094E7404601F080FCEEE730B585B010
:102350000446FEF79EFF18B96068FEF7E7FF10B16C
:10236000102005B030BD60884AF2B811884206D806
:102370002078424D28B1012806D0022804D0072039
:10238000EFE7FFF753F818E06078022804D003283D
:1023900002D043F20220E4E785F82300C1B2002016
:1023A0000090ADF8040002292CD0032927D0FFDFCC
:1023B00068460AF01CFC05F091FB0028D1D160684A
:1023C00001F036FC207858B101208DF800000DF1A5
:1023D000010001F03AFC68460AF08EFF00B1FFDF11
:1023E000207885F82200FFF7DEF9608860B1288444
:1023F00080B20AF077FB00B1FFDF0020B1E78DF873
:102400000500D5E74020FAE74FF46170EFE710B51B
:102410000446FEF764FF20B9606838B1FEF77DFF1F
:1024200008B1102010BD606801F00FFC134830F8AF
:10243000201F6180C178617080782070002010BDFD
:102440002DE9F843144689460646FEF748FFB8B919
:102450004846FEF76BFF98B92046FEF767FF78B94C
:10246000064DA878012800D154B13178FF2909D050
:1024700061B143F20400BDE8F8830000A40100202C
:102480001020F8E7012801D00420F4E7CCB3052898
:1024900011D004280FD06946204600F0EFF900283B
:1024A000E9D1217D49B1012909D0022909D00329A7
:1024B00009D00720DFE70820DDE7024604E001221B
:1024C00002E0022200E00322804623461746002055
:1024D0000099FFF781F90028CDD1A0892880A07B41
:1024E000E875BDF80000A882AF75BDF800100907B7
:1024F00001D5A18931B1A1892980C00704D0032069
:1025000003E006E08021F7E70220FEF777FF86F878
:1025100000804946BDE8F8430020FFF7F8B92DE9EF
:10252000FC41E84C06460D46A078022803D003285B
:1025300001D00820E8E516B143F20400E4E50620E6
:102540000BF062FD10B9A078032849D00DF0BEFC55
:1025500007460EF097FE381A00F0FF0806200BF031
:102560004BFD074606200BF04FFD391AA0780428D2
:1025700009D000221144A8EB010111F0FF0F04D093
:10258000032804D00DE00122F4E71320BCE528461F
:1025900005F044FA10B3407810B3284605F039FD31
:1025A000E570FFF787F809F0F5FA01208DF80000D3
:1025B0008DF801008DF802602088ADF80400E07D00
:1025C0008DF8060068460AF069FD05F087FA0028D4
:1025D000B0D1A078032805D0042010E0052093E5B1
:1025E000122091E5E07805F019FA040000D1FFDF30
:1025F000607800B9FFDF6078401E60700520FEF74C
:10260000FDFE002080E51CB510B143F204001CBDA6
:10261000AC4CA078042803D0052801D008201CBDAC
:1026200000208DF8000001218DF801108DF80200C6
:1026300068460AF033FD05F051FA0028EFD1A07882
:10264000052805D05FF00200FEF7D8FE00201CBD73
:10265000E07800F0C3F80320F6E72DE9FC4180465E
:102660000D4603260846FEF761FE08B110204BE533
:102670004046FFF77DF8040004D02078222804D2D9
:10268000082041E543F202003EE5A07F00F0030789
:102690003DB1012F0AD000202946FEF72AFF06008F
:1026A000E5D1012F04D0FFDF30462DE50120F3E70F
:1026B000A07D2946022801D011B107E0112023E5B1
:1026C000684600F00EFA0028D1D16946404609F06C
:1026D00079F80600E8D10120A075E5E770B50C4651
:1026E0000546FFF745F8010005D022462846BDE81B
:1026F0007040FFF740B843F2020070BD10B50128EA
:1027000007D1704B9B78012B00D011B143F204002C
:1027100010BD0AF019FABDE8104005F0DFB9012339
:1027200000F066B800231A46194600F061B870B58B
:10273000064615460C460846FEF7D1FD18B9284650
:10274000FEF7CDFD08B1102070BD2A462146304667
:102750000AF030FD05F0C2F90028F5D121787F2973
:10276000F2D1052070BD7CB505460C460846FEF743
:1027700090FD08B110207CBD2846FEF7F9FF20B17E
:102780000078222804D208207CBD43F202007CBDE0
:102790004C4890F82400400701D511207CBD2178D9
:1027A000C80802D16078C20801D007207CBD890822
:1027B00001D1800801D006207CBDADF80050207802
:1027C0008DF8020060788DF803000220ADF8040057
:1027D00068460AF016FB05F081F97CBD10B505F0DE
:1027E0001DF9040000D1FFDF6078401C607010BD4F
:1027F0001CB5ADF800008DF802308DF803108DF88F
:10280000042068460AF0A5FC05F068F91CBD0278B2
:10281000520804D0012A02D043F202207047FEF78A
:1028200026BF70B50C0006460DD0FEF7A1FF0500CF
:1028300000D1FFDFA68028892081288960816889EE
:10284000A081A889E08170BD10B500231A4603E07D
:10285000845C2343521CD2B28A42F9D30BB10020CC
:1028600010BD012010BD00B530B1012803D00228F1
:1028700001D0FFDF002000BDFF2000BD00220A8044
:1028800092B222F060020A800078062817D2DFE8B0
:1028900000F0160306090C1142F0110007E042F0A7
:1028A0001D0009E042F0150006E042F0100040F083
:1028B000020001E042F0100008800020704707206D
:1028C00070470000A4010020FE4800210160416023
:1028D000018170472DE9F743044692B09146406864
:1028E000FEF71BFD40B16068FEF720FD20B960785F
:1028F00000F00300022801D0012000E00020F14E8A
:1029000030724846FEF7C5FC18B1102015B0BDE87E
:10291000F08349460120FEF7ECFD0028F6D10125A1
:102920008DF842504FF4C050ADF84000002210A97D
:10293000284603F015FF0028E8D18DF842504FF4E7
:1029400028504FF00008ADF8400047461C2168466B
:10295000CDF81C8015F011FE9DF81C0008AA20F08F
:102960000F00401C20F0F00010308DF81C00207883
:102970008DF81D0061789DF81E0061F3420040F063
:1029800001008DF81E009DF800000AA940F0020029
:102990008DF800002089ADF83000ADF83270608904
:1029A00007AFADF834000B97606810AC0E900A9436
:1029B000684603F0C8FC0028A8D1BDF8200030808C
:1029C0008DF8425042F60120ADF840009DF81E00FF
:1029D00008AA20F00600801C20F001008DF81E00DF
:1029E0000220ADF83000ADF8340013A80E900AA90B
:1029F000684603F0A8FC002888D1BDF8200070804C
:102A0000311D484600F033F9002887D18DF8425037
:102A100042F6A620ADF840001C216846CDF81C8087
:102A200015F0ABFD9DF81C00ADF8345020F00F0000
:102A3000401C20F0F00010308DF81C009DF81D00A7
:102A400008AA20F0FF008DF81D009DF81E000AA9BD
:102A500020F0060040F00100801C8DF81E009DF85B
:102A600000008DF8445040F002008DF80000CDE9E0
:102A70000A4711A80E90ADF83050684603F063FC89
:102A8000002899D1BDF82000F08000203EE73EB537
:102A900004460820ADF800002046FEF7FAFB08B116
:102AA00010203EBD21460120FEF723FD0028F8D16D
:102AB0002088ADF804006088ADF80600A088ADF865
:102AC0000800E088ADF80A007E4801AB6A468088BD
:102AD000002104F041F8BDF800100829E1D00320DE
:102AE0003EBD1FB50446002002900820ADF8080046
:102AF000CDF80CD02046FEF7CCFB10B1102004B06E
:102B000010BD704802AA81884FF6FF7004F066FA83
:102B10000028F4D1BDF80810082901D00320EEE701
:102B2000BDF800102180BDF802106180BDF80410CE
:102B3000A180BDF80610E180E1E701B582B0022076
:102B4000ADF800005F4802AB6A464088002104F0FF
:102B500003F8BDF80010022900D003200EBD1CB5FB
:102B6000002100910221ADF800100190FEF7B7FBA3
:102B700008B110201CBD53486A4641884FF6FF70CB
:102B800004F02CFABDF800100229F3D003201CBD7C
:102B9000FEB54C4C06461546207A0F46C00705D0B8
:102BA0000846FEF776FB18B11020FEBD0F20FEBDD3
:102BB000F82D01D90C20FEBD3046FEF76AFB18BB8C
:102BC000208801A903F0C4F80028F4D130788DF8EA
:102BD0000500208801A903F09DFF0028EBD100909B
:102BE0009DF800009DF8051040F002008DF80000EF
:102BF000090703D040F008008DF8000020886946DE
:102C000003F025FF0028D6D1ADF8085020883B46B8
:102C100002AA002103F0A0FFBDF80810A942CAD003
:102C20000320FEBD7CB50546002000900190088879
:102C3000ADF800000C4628460195FEF76EFB18B96A
:102C40002046FEF74CFB08B110207CBD15B1BDF845
:102C5000000050B11B486A4601884FF6FF7004F02F
:102C6000BDF9BDF8001021807CBD0C207CBD30B5C5
:102C700093B0044600200D460090142101A815F0E1
:102C80007CFC1C2108A815F078FC9DF80000CDF80C
:102C900008D020F00F00401C20F0F00010308DF81C
:102CA00000009DF8010020F0FF008DF801009DF864
:102CB000200040F002008DF8200001208DF8460031
:102CC00002E00000CC01002042F60420ADF84400F0
:102CD00011A801902088ADF83C006088ADF83E0056
:102CE000A088ADF84000E088ADF842009DF80200F1
:102CF00006AA20F00600801C20F001008DF80200DA
:102D00000820ADF80C00ADF810000FA8059001A93F
:102D100008A803F018FB002803D1BDF8180028808C
:102D2000002013B030BD00004FF0E0214FF4004010
:102D3000C1F88001BFF34F8FBFF36F8F00F021B850
:102D400010B5044600F01DF8002C09D0124A1248B4
:102D500012491432124B012C03D0022C07D0FFDF92
:102D600010BD0224046011604FF0407004E00324A1
:102D7000046011604FF40000186010BD00B5FFDF63
:102D800000BD054800210160016005494FF06070F9
:102D9000091D08607047000000F500404C0200204B
:102DA00004F501400DF092BF0449002008604FF087
:102DB000E0210220C1F8800270470000FC1F0040A3
:102DC00010B50D2000F06FF8C4B26FF0040000F0F1
:102DD0006AF8C0B2844200D0FFDF3A49012008609F
:102DE00010BD70B50D2000F040F8374C0020C4F83D
:102DF00000010125C4F804530D2000F047F82560B8
:102E00004FF0E0216014C1F8000170BD10B50D2035
:102E100000F02BF82C48012141600021C0F800117E
:102E2000BDE810400D2000F031B8274910B5D1F8A9
:102E30000001012801D0FFDF10BD2248001D0068FD
:102E40000022C0B2C1F80021BDE810400EF08ABBDC
:102E500010B51D48D0F800110029FBD0FFF7E5FFA1
:102E6000BDE810400D2000F011B800280DDB00F087
:102E70001F02012191404009800000F1E020C0F8CC
:102E80008011BFF34F8FBFF36F8F7047002809DBAE
:102E900000F01F02012191404009800000F1E02074
:102EA000C0F880127047002804DB00F1E02090F8A1
:102EB000000405E000F00F0000F1E02090F8140D90
:102EC0004009704704D5004000D00040704770476B
:102ED0007047704770477047704700004FF0E0211F
:102EE0004FF00070C1F8800101F5C071BFF34F8F42
:102EF000BFF36F8FC1F80001334B802283F80024A9
:102F000041F8800C704700B5024604202F4903E0C9
:102F100001EBC0031B792BB1401EC0B2F8D2FFDF1A
:102F2000FF2000BD41F8302001EBC00100224A71B2
:102F30008A7101220A7100BD244A002102EBC000FF
:102F40000171704710B50446042800D3FFDF1F4805
:102F500000EBC4042079012800D0FFDF6079A1795B
:102F6000401CC0B2814200D060714FF0E0214FF0B0
:102F70000070C1F8000210BD70B51348042590F828
:102F80000004124E4009124C042818D0FFDF16E04E
:102F9000217806EBC1000279012A08D142798379B0
:102FA0009A4204D04279827156F8310080472078E5
:102FB000401CC0B22070042801D3002020706D1E78
:102FC000EDB2E5D270BD000019E000E098040020E9
:102FD000480000200348044A0168914201D10021C1
:102FE000016070474C000020BEBAFECA70477047AF
:102FF00070477047704770477047704770470000D0
:103000002CFFFFFFDBE5B15100900100B800FFFF8E
:103010007000000069915B00935FFEEDA0843C733B
:10302000F87462145E06C0CB72F2136010B50446E9
:10303000FEF72FF908B1102010BD2078C0F3021060
:10304000042807D86078072804D3A178102901D86C
:10305000814201D2072010BDE078410706D42179D2
:103060004A0703D4000701D4080701D5062010BD84
:10307000002010BD70B514460D46064604F022FF30
:1030800080B10178182221F00F01891C21F0F00194
:10309000A03100F8081B214615F013FABDE8704076
:1030A00004F013BF29463046BDE870401322FEF7F6
:1030B00062BB2DE9F047064608A8894690E830042F
:1030C0001F4690461421284615F057FA0021CAF8E9
:1030D0000010B8F1000F03D0B9F1000F03D114E0D4
:1030E0003878C00711D02068FEF7F9F8C0BBB8F1F6
:1030F000000F07D120681230286020681430686003
:103100002068A8602168CAF800103878800724D5A4
:103110006068FEF702F918BBB9F1000F21D0FEF785
:10312000AFFF0168C6F868118188A6F86C11807934
:1031300086F86E0101F033FAF84FEF60626862B111
:1031400096F8680106F2691140081032FEF7EBFAB2
:1031500010223946606815F06FF90020BDE8F0874D
:1031600006E0606820B1E8606068C6F86401F4E7D2
:103170001020F3E730B5054608780C4620F00F0024
:10318000401C20F0F001103121700020607095F893
:10319000230030B104280FD0052811D0062814D000
:1031A000FFDF20780121B1EB101F04D295F8200039
:1031B00000F01F00607030BD21F0F000203002E010
:1031C00021F0F00030302070EBE721F0F0004030CB
:1031D000F9E7F0B591B0022715460C4606463A4687
:1031E000ADF80870082103AB08F0DEF80490002861
:1031F00010D004208DF804008DF80170E034099699
:1032000005948DF818500AA968460CF039FC00B1F5
:10321000FFDF012011B0F0BD2DE9F84F0646808A8E
:103220000C4680B28246FEF7A3FA0546BB4F3078C3
:10323000203F4FF002094FF000080F287CD2DFE852
:1032400000F07BA39D082C5B6A7CBADAFD97489757
:103250009700012150460AF023FF040000D1FFDF50
:1032600097F85C00C00701D0386E0BE0032104F131
:103270001D000EF058F9D4F81D00A949B0FBF1F279
:1032800001FB1200C4F81D0070686067B068A06799
:103290002878252872D0FFDF70E0012150460AF01F
:1032A000FFFE060000D1FFDF3078810702D52978C4
:1032B000252904D040F001003070BDE8F88F84F873
:1032C0000090307F207106F11D002D36C4E9020602
:1032D000F3E7012150460AF0E3FE050000D1FFDFCD
:1032E0002878C10604D5072020703D356560E4E7E5
:1032F00040F008002870E0E7E87F000700D5FFDF16
:10330000307CB28800F0010301B05046BDE8F04FB8
:10331000082108F07FB905B9FFDF716821B11022DB
:1033200005F1240015F088F828212846FEF78FF8CB
:10333000307A85F82000C0E7F8E0012150460AF015
:10334000AFFE050000D1FFDF022105F185000EF080
:10335000EAF80420207005F5B4706060B5F88500C7
:1033600020826E4810387C356561C4E90270A4E79C
:10337000012150460AF094FE00B9FFDF324629468B
:103380005046BDE8F84F75E605B9FFDF28782128DB
:1033900093D93079012803D1E87F40F00800E8771D
:1033A000324629465046FFF765FE2846BDE8F84FED
:1033B0002321FEF74CB83279A28004F108030821DA
:1033C000504607F0F1FFE06010B10520207074E76F
:1033D0004546012150460AF063FE040000D1FFDF9C
:1033E00004F1620102231022081F0AF0FEFC05709E
:1033F0003179417061E7012150460AF051FE040025
:1034000000D1FFDF94F8840000F00300012859D1B7
:10341000E87F10F0010103D194F8A000C0072AD082
:10342000D4F8602132B394F88330107C63F38700C2
:103430001074AA7FD30963F3410000E072E0D4F86E
:1034400060211074D4F8602161F30000107491B110
:10345000D4F86001102205F12401883414F0ECFF47
:10346000207E40F001002076207820F0010004F852
:10347000880919E0C1B994F88800C00714D0D4F8BD
:103480005C0188B194F88330027C63F38702027494
:10349000A87FC309D4F85C0163F341020274D4F835
:1034A0005C0161F30002027494F88800800709D57A
:1034B00094F87C00D4F86421400804F17D011032B6
:1034C000FEF731F98DF8009094F884006A4600F018
:1034D00003008DF8010094F888108DF8021094F81C
:1034E000A0008DF803002946504601F041F82878E5
:1034F000252805D0212807D0FFDF2878222803D9E6
:1035000022212846FDF7A3FF012150460AF0DAFDEB
:1035100000283FF4DDAEFFDFCFE60000F801002019
:1035200040420F00716881F80180C6E6FFDFC4E603
:1035300070B5FE4C002584F85C5025660CF06DFAE1
:1035400004F11001204604F079FC84F8305070BD7D
:1035500070B50D46FEF70CF9040000D1FFDF4FF403
:10356000B871284615F009F82434012105F1E0006E
:103570002C610CF053FA002800D0FFDF70BD0A4622
:10358000014602F1E0000CF069BA70B505464068EA
:1035900086B00178082906D00B2933D00C292FD00A
:1035A000FFDF06B070BD46883046FEF7E1F8040044
:1035B00000D1FFDF20782128F3D028281BD16868AC
:1035C00002210C3000F09FFFA8B168680821001D9F
:1035D00000F099FF78B104F12401304609F060FD54
:1035E00004F07CFA00B1FFDF06B02046BDE8704071
:1035F0002921FDF72CBF06B0BDE8704004F065BC82
:1036000001218171686886883046FEF7B1F80400B0
:1036100000D1FFDF20782128C3D06868817909B103
:10362000807808B1FFDFBCE704F04FFCA07F000604
:1036300023D5E07FC00705D094F8200000F01F00DC
:10364000102818D05FF0050084F82300207829287E
:1036500015D02428A5D1314604200EF043FA2221AA
:103660002046FDF7F4FE012130460AF02BFD00282C
:1036700097D0FFDF95E70620E6E70420E4E7012185
:1036800030460AF00DFD050000D1FFDF2521204660
:10369000FDF7DDFE03208DF80000694605F1E0002E
:1036A0000CF0D3F90228BED00028BCD0FFDF78E7A9
:1036B0002DE9F04788B09A46164688468146FEF7BF
:1036C00057F805003AD02878222837D3232835D058
:1036D000E87F000732D40027012148460AF0E0FCC9
:1036E000040005D10121002248460AF0D0FC04461E
:1036F000694600F064FF009800B9FFDF00983CB114
:10370000E03404612878222804D0242802D005E07F
:10371000076103E025212846FDF799FE0098012165
:103720004170C0F824908680C0E9028A01A90CF09B
:10373000A7F9022802D0002800D0FFDF08B00DE56D
:1037400070B586B00546FEF713F80078222814D924
:10375000012128460AF0A4FC04002CD1FFDF2AE056
:10376000B4F85E0004F1620630440178427829B171
:1037700021462846FFF72DFDB0B912E7ADF8042029
:103780000821284602AB07F00FFE03900028F4D072
:1037900005208DF80000694604F1E0000CF055F9B1
:1037A000022801D000B1FFDF02231022314604F1CC
:1037B0005E000AF050FBB4F860000028D0D1F0E6BB
:1037C00010B586B00446FDF7D3FF0078222811D942
:1037D000012120460AF064FC040000D1FFDF06202E
:1037E0008DF80000694604F1E0000CF02EF9002885
:1037F00000D0FFDF06B010BD2DE9F84F0546007878
:103800000C460027010904F1080090463E46BA46DE
:10381000009002297ED0072902D00A2909D142E06E
:1038200068680178082905D00B292CD00C292AD0EA
:10383000FFDF72E114271C26002C6CD04088A0808A
:10384000FDF796FF5FEA000900D1FFDF99F8170046
:1038500009F118014008009AFDF765FF6868808942
:10386000208268684168C4F812108068C4F81600A5
:10387000A07E20F0060040F00100A07699F81E001E
:1038800040F020014FE01A270A26002CD5D080886E
:10389000A080FDF76DFF050000D1FFDF28460099ED
:1038A000FFF768FC39E10CB1A88BA080287A4FF0B3
:1038B000010B0B287ED006DC01287CD0022808D022
:1038C000032804D137E00D2876D00E2875D0FFDF0D
:1038D00023E11E270926002CAFD0A088FDF748FF62
:1038E0005FEA000900D1FFDF287B00F00300012818
:1038F000207A1DD020F001002072297B890861F315
:1039000041002072297BC90861F382002072297B63
:10391000090901E0F7E0AEE061F3C300207299F815
:103920001E0040F0400189F81E10F6E0D80100208A
:1039300040F00100E0E713270D26002CA6D0A08858
:10394000FDF716FF81460121A0880AF0A9FB0500BA
:1039500000D1FFDF686F817801F003010129217A2E
:1039600050D021F00101217283789B0863F341015B
:1039700021728378DB0863F38201217283781B094B
:1039800063F3C3012172037863F306112172437854
:1039900063F3C711217284F809A0C178A17202797A
:1039A000E17A62F30001E1720279520862F34101A7
:1039B000E17203E029E067E04EE05FE002799208FF
:1039C00062F38201E1720279D20862F3C301E1720B
:1039D0004279217B62F3000121734279520862F33C
:1039E000410121734279920862F382012173407987
:1039F000C00860F3C301217399F8000023282AD975
:103A0000262139E041F00101ADE71827102694B3D3
:103A1000A088FDF7ADFE00900121A0880AF040FBD0
:103A20005FEA000900D1FFDFE868A06099F80000B4
:103A300040F0040189F8001099F80100800708D5CA
:103A400084F80CB000980078232866D927210098C4
:103A500052E084F80CA060E015270F265CB1A08826
:103A6000FDF786FE81460622E868009907F020FCF3
:103A700084F80EB085E042E048463DE0162709266E
:103A8000ECB3287B207248E0287B19270E26B4B3BC
:103A9000C4F808A0A4F80CA0012807D0022808D078
:103AA00003280CD004280AD0FFDF15E084F808B002
:103AB00001E002202072607A20F003000BE0697BB5
:103AC000042801F00F0141F080012172F3D1607AE6
:103AD00020F00300401C6072A088FDF749FE0546F7
:103AE0000078212819D0232800D0FFDF0121A088E9
:103AF0000AF0E8FA22212846FDF7A9FC0DE0FFE7CD
:103B0000A8F800600EE00CB16888A080287A10B395
:103B1000012809D002283AD0FFDFA8F800600CB1D4
:103B200027806680002006E415270F26002CE7D0AA
:103B3000A088FDF71DFE0121A0880AF0B1FA05005A
:103B400000D1FFDFD5F81D000622009907F0B0FB79
:103B500084F80EA0E1E717270926002CD0D0A08812
:103B6000FDF706FE81460121A0880AF099FA0500BA
:103B700000D1FFDF6878800701D5022000E0012036
:103B8000207299F800002328C7D9272174E7192744
:103B90000E26002CB4D0A088FDF7EAFD5FEA0009EC
:103BA00000D1FFDFC4F808A0A4F80CA084F808A096
:103BB000A07A40F00300A07299F81E10C90961F3C1
:103BC0008200A07299F81F2099F81E1012EAD11FE6
:103BD00005D099F8201001F01F01102925D020F000
:103BE0000800A07299F81F10607A61F3C300607238
:103BF000697A01F0030101298FD140F0040060725D
:103C0000E87A217B60F300012173AA7A607B62F37A
:103C100000006073EA7A520862F341012173A97AC5
:103C2000490861F34100607377E740F00800D8E786
:103C300010B5F84C30B10146102204F1200014F008
:103C4000FBFB012084F8300010BD10B5044600F0E5
:103C5000A6FCF04920461022BDE81040203114F0A7
:103C6000EBBB70B5EB4D06004FF0000412D0FDF732
:103C700010FB08B110240BE00621304607F0FFFAD4
:103C8000411C04D02866012085F85C0000E0072470
:103C9000204670BD0020F7E7007810F00F0204D036
:103CA000012A05D0022A0CD110E0000909D10AE04E
:103CB0000009012807D0022805D0032803D00428D2
:103CC00001D0072070470870002070470620704719
:103CD00005282AD2DFE800F003070F171F00087835
:103CE00020F0FF001EE0087820F00F00401C20F0BC
:103CF000F000103016E0087820F00F00401C20F093
:103D0000F00020300EE0087820F00F00401C20F07A
:103D1000F000303006E0087820F00F00401C20F062
:103D2000F0004030087000207047072070472DE9F0
:103D3000F043804687B00D464FF000090846FDF776
:103D4000F5FAA8B94046FDF713FD060003D0307818
:103D500022280BD104E043F2020007B0BDE8F08353
:103D600035B1B07FC10601D4000703D50820F4E7C0
:103D70001020F2E7F07F000701D50D20EDE70027C6
:103D8000012140460AF08CF9040006D101210022ED
:103D900040460AF07CF9040005D0694600F00FFCAB
:103DA000009818B901E00420D7E7FFDF009802214E
:103DB000E0344170C0F82480446107810121017121
:103DC000297801F00102017E62F3010101762A786F
:103DD000520862F3820101762A78920862F3C301E5
:103DE00001762A78D20862F3041101762421304644
:103DF000FDF72DFB01A900980BF042FE022801D02F
:103E000000B1FFDF4846A8E72DE9FF4F0E46824983
:103E1000904697B09A4607C914AB4FF0000983E863
:103E200007001798FDF7A4FC050006D0287826287F
:103E300006D008201BB0BDE8F08F43F20200F9E77E
:103E400026B94046FFF7F2F80028F3D10121179870
:103E50000AF026F9040000D1FFDF852E27D007DC09
:103E6000EEB1812E1DD0822E1DD0832E08D11CE0F4
:103E7000862E1ED0882E1ED0892E1ED08A2E1ED0B1
:103E80000F2020710F281CD004F01CF8D8B101209D
:103E90008DF83400201D0E902079B0B126E100206D
:103EA000EFE70120EDE70220EBE70320E9E705203B
:103EB000E7E70620E5E70820E3E70920E1E70A2035
:103EC000DFE70720B6E71120B4E798F80000D4E94F
:103ED0001D764208A87F002162F3C710A87798F8E2
:103EE00000008208E87F62F30000E87798F800009D
:103EF000C209607862F34100607098F8000002091E
:103F0000207862F34710207098F80000C2086078AB
:103F100062F30000607098F80100607198F800008A
:103F200000F00102B07862F30100B070AA7FD209FC
:103F300062F38200B070EA7F62F3C300B07062780F
:103F400062F30410B0702278C0F3C00052093270DE
:103F50006278C2F34002727098F80220F2707171B8
:103F60003171B978C1F3C00108405FEA000B2ED06F
:103F70005046FDF78EF978BBDAF80C00FDF789F9A9
:103F800050BBDAF81C00FDF784F928BBDAF80C0006
:103F9000A060DAF81C00E06060787A7842EA5001AC
:103FA00061F341006070B978C0B200EA111161F3A9
:103FB000000060700020207705F117006061681C28
:103FC000A061B07800F00300012806D046E06078D8
:103FD0007A7802EA5001E3E719E0B87800F00300CC
:103FE00001283BD1321D711D404600F097FA31790E
:103FF000387901408DF8281070797A7910408DF861
:10400000300001432AD05046FDF743F930B110206B
:1040100010E70000D8010020FC8801000AF1100020
:1040200004F5AE7304F18C028DE80D0000210AAB9B
:104030005A462046FFF73DF80028E9D104F5B07252
:1040400004F1A403CDF800A0CDE9013201210CABAD
:104050005A462046FFF72DF80028D9D1607880070E
:1040600022D4B078B978C0F38000C1F3800108434E
:104070001AD0307814AA397832F810204B00DA4080
:1040800002F00309B9F1030F01D14FF00209BBF1AE
:10409000000F09D0012801D0042805D1012901D041
:1040A000042901D14FF00409A87F40F08000A877CF
:1040B000E97F6BF30001E9776078800706D503207C
:1040C000A071BBF1000F11D100202BE00220B9F14B
:1040D000020F1AD0B9F1010F19D0B9F1040F29D08C
:1040E0000020A071A87F20F08000A8772521284615
:1040F000FDF7ADF90DA904F1E0000BF0A6FC10B13D
:10410000022800D0FFDF002094E6A071DCE7A07158
:104110000D2104F1200014F030FA207840F0020064
:10412000207001208DF84C0013AA2946179800F042
:104130001FFADBE70120A071D8E72DE9F04387B033
:104140009046894604460025FDF712FB070004D07F
:104150003878272804D00820FFE543F20200FCE568
:104160000121204609F09CFF040000D1FFDFA67961
:104170005FEA090005D0012821D0B9F1020F26D14C
:1041800010E0B8F1000F22D1012E05D0022E05D08B
:10419000032E05D0FFDF2DE00C252BE0012529E0C3
:1041A000022527E04046FDF774F8B0B9032E0ED182
:1041B0001022414604F11D0014F03EF91AE0012ED0
:1041C00002D0022E03D104E0B8F1000F12D0072074
:1041D000C3E54046FDF75DF808B11020BDE51021AC
:1041E00004F11D0014F0A7F90621404607F047F836
:1041F000C4F81D002078252140F0020020703846C8
:10420000FDF725F92078C10713D020F001002070B8
:1042100002208DF8000004F11D0002908DF804507A
:104220006946C3300BF011FC022803D010B1FFDF48
:1042300000E02577002090E530B587B00D460446B4
:10424000FDF796FA60B10121204609F029FF04002C
:104250000CD02846FDF71DF828B1102007B030BD5E
:1042600043F20200FAE72078400701D40820F5E77E
:10427000294604F13D002022054614F0DDF820789F
:1042800040F01000207001070FD520F008002070CA
:1042900007208DF80000694604F1E00001950BF05D
:1042A000D4FB022801D000B1FFDF0020D6E770B5B3
:1042B0000D460646FDF75CFA18B10078272817D19D
:1042C00002E043F2020070BD0121304609F0E8FE31
:1042D000040000D1FFDFA079022809D16078C0076F
:1042E00006D02A4621463046FEF773FF10B10FE094
:1042F000082070BDB4F860000E280BD204F16201F2
:1043000002231022081F09F070FD01210170457081
:10431000002070BD112070BD70B5064614460D46D4
:104320000846FCF7B6FF18B92046FCF7D8FF08B1DD
:10433000102070BDA6F57F40FF380ED03046FDF747
:1043400017FA38B1417822464B08811C1846FDF710
:10435000EAF907E043F2020070BD2046FDF7F2FEE5
:104360000028F9D11021E01D0DF0DDF8E21D2946ED
:1043700004F1170000F033F9002070BD2DE9F04181
:1043800004468AB015460E4600270846FCF7CEFFC5
:1043900018B92846FCF7CAFF18B110200AB0BDE8CA
:1043A000F0812046FDF7E4F95FEA000804D098F8B0
:1043B0000000272810D102E043F20200EEE70121BD
:1043C000204609F06DFE040000D1FFDF2078400791
:1043D00002D56078800701D40820DFE7D4E91D0109
:1043E000497801B18DB1407800B176B1ADB1EA1D27
:1043F00006A8E16800F0F3F8102206A905F11700FD
:1044000013F0EEFF18B1042707E00720C6E71022DB
:10441000E91D04F12D0014F00FF82EB11022F11D4A
:1044200004F11D0014F008F82078252140F0020066
:1044300020704046FDF70BF82078C10715D020F01A
:104440000100207002208DF8000004F11D00029090
:10445000103003908DF804706946B3300BF0F5FA14
:10446000022803D010B1FFDF00E02777002095E796
:1044700070B50D4606460BB1072070BDFDF778F903
:10448000040007D02078222802D3A07F800604D41D
:10449000082070BD43F2020070BDADB12946304620
:1044A00008F0FEFD03F01AFB297C4A08A17F62F3A5
:1044B000C711A177297CE27F61F30002E277297CB2
:1044C000890884F8201004E0304608F00CFE03F060
:1044D00005FBA17F21F02001A17770BD70B50D46CD
:1044E000FDF746F9040005D02846FCF7F8FE20B198
:1044F000102070BD43F2020070BD29462046FEF731
:1045000039FE002070BD04E010F8012B0AB1002034
:104510007047491E89B2F7D20120704710B5C478A0
:104520000B7864F300030B70C478640864F34103F0
:104530000B70C478A40864F382030B70C478E40899
:1045400064F3C3030B700379117863F300011170F6
:1045500003795B0863F34101117003799B0863F3EE
:10456000820111700079C00860F3C301117010BDA1
:1045700070B51546064603F0A5FC040000D1FFDF28
:10458000207820F00F00801C20F0F00020302070F8
:1045900066802868A060BDE8704003F096BC10B546
:1045A000134C94F83000002808D104F12001A1F147
:1045B00010000BF08CFA012084F8300010BD10B10F
:1045C00090F8B9202AB10A4890F8350018B10020B7
:1045D00003E0B83001E0064834300860704708B5A1
:1045E0000023009313460A4609F055FF08BD00005A
:1045F000D8010020F0B5007B059F1E4614460D46ED
:10460000012800D0FFDF0C2030803A203880002CB9
:1046100008D0287A032806D0287B012800D0FFDFA5
:1046200017206081F0BDA889FBE72DE9F04786B02F
:10463000144691F80C900E9A0D46B9F1010F0BD06B
:104640001021007B2E8A8846052807D0062833D003
:10465000FFDF06B0BDE8F0870221F2E7E8890C2110
:1046600000EB400001EB4000188033201080002C4C
:10467000EFD0E889608100271AE00096688808F189
:10468000020301AA696900F084FF06EB0800801CA0
:1046900007EB470186B204EB4102BDF804009081AC
:1046A0000DF1060140460E320BF087FA7F1CBFB2B7
:1046B0006089B842E1D8CCE734201080E889B9F1AC
:1046C000010F11D0122148430E301880002CC0D0A9
:1046D000E88960814846B9F1010F00D002202073BB
:1046E00000270DF1040A1FE00621ECE70096688818
:1046F00008F1020301AA696900F04BFF06EB08000C
:10470000801C86B2B9F1010F12D007EBC70004EB91
:104710004000BDF80410C18110220AF102011030DE
:1047200013F08AFE7F1CBFB26089B842DED890E7E2
:1047300007EB470104EB4102BDF80400D0810AF108
:104740000201404610320BF038FAEBE72DE9F04752
:104750000E4688B090F80CC096F80C80378AF58920
:104760000C20109902F10C044FF0000ABCF1030F69
:1047700008D0BCF1040F3ED0BCF1070F7DD0FFDFA5
:1047800008B067E705EB850C00EB4C001880312082
:104790000880002AF4D0A8F1060000F0FF09558136
:1047A00025E0182101A813F0E8FE00977088434621
:1047B00001AA716900F0EDFEBDF804002080BDF88B
:1047C0000600E080BDF808002081A21C0DF10A015E
:1047D00048460BF0F2F9B9F1000F00D018B184F897
:1047E00004A0A4F802A007EB080087B20A346D1EEB
:1047F000ADB2D6D2C4E705EB850C00EB4C001880B7
:1048000032200880002ABBD0A8F1050000F0FF0983
:10481000558137E000977088434601AA716900F01E
:10482000B8FE9DF80600BDF80410E1802179420829
:1048300060F3000162F34101820862F38201C20861
:1048400062F3C301020962F30411420962F34511E4
:10485000820962F386112171C0096071BDF80700F9
:10486000208122460DF1090148460BF0A6F918B146
:1048700084F802A0A4F800A000E007E007EB08001D
:1048800087B20A346D1EADB2C4D279E7A8F1020036
:1048900084B205FB08F000F10E0CA3F800C035232C
:1048A0000B80002AA6D055819481009783B270882E
:1048B0000E32716900F06DFE62E72DE9F84F1E4679
:1048C0000A9D0C4681462AB1607A00F58070D0803E
:1048D000E089108199F80C000C274FF000084FF088
:1048E0000E0A0D2873D2DFE800F09E070E1C283058
:1048F0003846556A73737300214648460095FFF7A2
:1049000079FEBDE8F88F207B9146082802D0032865
:1049100000D0FFDF378030200AE000BFA9F80A800E
:10492000EFE7207B9146042800D0FFDF378031205D
:104930002880B9F1000FF1D1E3E7207B91460428EC
:1049400000D0FFDF37803220F2E7207B914602283B
:1049500000D0FFDF37803320EAE7207B17460228AC
:1049600000D0FFDF3420A6F800A02880002FC8D098
:10497000A7F80A80C5E7207B1746042800D0FFDF90
:104980003520A6F800A02880002FBAD04046A7F80E
:104990000A8012E0207B1746052802D0062800D0A6
:1049A000FFDF1020308036202880002FA9D0E0893A
:1049B0007881A7F80E80B9F80E00B881A1E7207BB6
:1049C0009146072800D0FFDF37803720B0E72AE084
:1049D0004FF0120018804FF038001700288090D058
:1049E000E0897881A7F80E80A7F8108099F80C006C
:1049F0000A2805D00B2809D00C280DD0FFDF80E74E
:104A0000207B0A2800D0FFDF01200AE0207B0B2852
:104A100000D0FFDF042004E0207B0C2800D0FFDF63
:104A2000052038736DE7FFDF6BE770B50C46054670
:104A3000FCF79EFE20B10078222804D2082070BD29
:104A400043F2020070BD0521284609F029FB2060D1
:104A500008B1002070BD032070BD30B448800878D4
:104A600020F00F00C01C20F0F000903001F8080B7F
:104A70001DCA81E81D0030BC03F027BA2DE9FF47AD
:104A800084B00027824602970798904689461230E4
:104A900004F046FB401D20F00306079828B907A93B
:104AA0005046FFF7C2FF002854D1B9F1000F05D0DE
:104AB0000798017B19BB052504681BE098F80000E6
:104AC000092803D00D2812D0FFDF46E007990325FF
:104AD0004868B0B3497B42887143914239D98AB260
:104AE000B3B2011D09F06DF90446078002E0079C8E
:104AF000042508340CB1208810B1032D29D02CE0F6
:104B000007980121123004F03DFBADF80C0002467D
:104B100002AB2946504606F047FC070001D1A01C15
:104B2000029007983A461230C8F80400A8F802A08C
:104B300003A94046029B04F032FBD8B10A2817D2E1
:104B400000E006E0DFE800F007091414100B0D1474
:104B50001412132014E6002012E6112010E608209B
:104B60000EE643F203000BE6072009E60D2007E6F8
:104B7000032005E6BDF80C002346CDE900702A4667
:104B80005046079900F015FD57B9032D08D1079835
:104B9000B3B2417B406871438AB2011D09F025F927
:104BA000B9F1000FD7D0079981F80C90D3E72DE920
:104BB000FE4F91461A881C468A468046FAB102ABDF
:104BC000494606F0F1FB050019D04046A61C27888F
:104BD00009F0AAFB3246072629463B46009608F014
:104BE000D6FF20882346CDE900504A46514640462C
:104BF00000F0DFFC002020800120BDE8FE8F0020B7
:104C0000FBE710B586B01C46AAB104238DF800302E
:104C10001388ADF808305288ADF80A208A788DF8EC
:104C20000E200988ADF80C1000236A462146FFF7D4
:104C300025FF06B010BD1020FBE770B50D4605211D
:104C400009F02EFA040000D1FFDF294604F112001A
:104C5000BDE8704004F07FBA2DE9F8430D46804668
:104C6000002603F02FF904462878102878D2DFE8D0
:104C700000F0773B34533131123131310831313169
:104C800031312879001FC0B2022801D0102810D17C
:104C900014BBFFDF35E004B9FFDF0521404609F012
:104CA000FFF9007B032806D004280BD0072828D062
:104CB000FFDF072655E02879801FC0B2022820D0E8
:104CC00050B1F6E72879401FC0B2022819D0102849
:104CD00017D0EEE704B9FFDF13E004B9FFDF28794E
:104CE00001280ED1172137E00521404609F0D8F9F7
:104CF000070000D1FFDF07F11201404604F008FA77
:104D00002CB12A4621464046FFF7A7FE29E0132191
:104D10004046FDF7E3FC24E004B9FFDF05214046EF
:104D200009F0BEF9060000D1FFDF694606F1120066
:104D300004F0F8F9060000D0FFDFA988172901D296
:104D4000172200E00A46BDF80000824202D901465F
:104D500002E005E01729C5D3404600F03AFCD0E751
:104D6000FFDF3046BDE8F883401D20F0030219B193
:104D700002FB01F0001D00E000201044704713B555
:104D8000009848B10024684608F0C5FF002C02D105
:104D9000F74A009911601CBD01240020F4E72DE9B9
:104DA000F0470C4615462421204613F0E6FB05B9D2
:104DB000FFDFA87860732888DFF8B4A3401D20F0D7
:104DC0000301AF788946DAF8000008F0C2FF060058
:104DD00000D1FFDF4FF000082660A6F8008077B111
:104DE00009FB07F1091D0AD0DAF8000008F0B1FF4D
:104DF000060000D1FFDF6660C6F8008001E0C4F85D
:104E00000480298804F11200BDE8F04704F072B96B
:104E10002DE9F047804601F112000D46814604F06D
:104E20007FF9401DD24F20F003026E7B14462968A3
:104E3000386808F0B9FF3EB104FB06F2121D03D03A
:104E40006968386808F0B0FF052009F0D5F8044615
:104E5000052009F0D9F8201A012802D1386808F095
:104E60006DFF49464046BDE8F04704F058B970B5BB
:104E70000546052109F014F9040000D1FFDF04F113
:104E800012012846BDE8704004F042B92DE9F04F08
:104E900091B04FF0000BADF834B0ADF804B04788D6
:104EA0000C46054692460521384609F0F9F80600F9
:104EB00000D1FFDF24B1A780A4F806B0A4F808B0A1
:104EC000297809220B20B2EB111F7DD12A7A04F137
:104ED000100138274FF00C084FF001090391102AF8
:104EE00073D2DFE802F072F2F1F07F08D2888D9F72
:104EF0003DDBF3EEB6B6307B022800D0FFDFA88999
:104F000008EBC001ADF804103021ADF83410002CCE
:104F100025D06081B5F80E9000271DE004EBC7088E
:104F2000317C88F80E10F189A8F80C10CDF80090AB
:104F30006888042304AA296900F02BFBBDF810102F
:104F4000A8F8101009F10400BDF812107F1C1FFA18
:104F500080F9A8F81210BFB26089B842DED80DE11E
:104F6000307B022800D0FFDFE98908EBC100ADF8F3
:104F700004003020ADF83400287B0A90001FC0B236
:104F80000F90002CEBD06181B5F81090002725E040
:104F9000CDF800906888696903AA0A9B00F0F9FAC5
:104FA0000A9804EBC70848441FFA80F908F10C027C
:104FB00004A90F980AF001FE18B188F80EB0A8F8FD
:104FC0000CB0BDF80C1001E0D4E0CFE0A8F8101050
:104FD000BDF80E107F1CA8F81210BFB26089B8424D
:104FE000D6D8CBE00DA8009001AB2246294630462A
:104FF000FFF71BFBC2E0307B082805D0FFDF03E092
:10500000307B082800D0FFDFE8891030ADF80400BD
:105010003620ADF83400002C3FD0A9896181F18998
:10502000A18127E0307B092800D0FFDFA88900F1AB
:105030000C01ADF804103721ADF83410002C2CD041
:105040006081E8890090AB89688804F10C022969C5
:1050500056E0E8893921103080B2ADF80400ADF88F
:105060003410002C74D0A9896181287A0E280AD0C6
:1050700002212173E989E181288A0090EB896888FF
:105080006969039A3CE00121F3E70DA8009001ABA8
:10509000224629463046FFF759FB6FE0307B0A284D
:1050A00000D0FFDF1220ADF80400ADF834704CB32F
:1050B000A9896181A4F810B0A4F80EB084F80C900E
:1050C0005CE020E002E031E039E042E0307B0B2898
:1050D00000D0FFDF288AADF834701230ADF804003C
:1050E00084B104212173A9896181E989E181298A37
:1050F0002182688A00902B8A688804F1120269690B
:1051000000F047FA3AE0307B0C2800D0FFDF122095
:10511000ADF80400ADF834703CB305212173A4F858
:105120000AB0A4F80EB0A4F810B027E00DA80090C3
:1051300001AB224629463046FFF75CFA1EE00DA877
:10514000009001AB224629463046FFF7B6FB15E03A
:1051500034E03B21ADF80400ADF8341074B3A4F88A
:105160000690A4F808B084F80AB007E0FFDF05E075
:1051700010000020297A012917D0FFDFBDF80400B4
:10518000AAF800006CB1BDF834002080BDF804001E
:105190006080BDF83400392803D03C2801D086F85F
:1051A0000CB011B00020BDE8F08F3C21ADF8040038
:1051B000ADF8341014B1697AA172DFE7AAF80000E3
:1051C000EFE72DE9F84356880F468046154605213E
:1051D000304608F065FF040000D1FFDF1234009470
:1051E0003B46414630466A6804F00DF9BAE570B5B1
:1051F0000D46052108F054FF040000D1FFDF2946C9
:1052000004F11200BDE8704003F097BF70B50D4681
:10521000052108F045FF040000D1FFDF294604F115
:105220001200BDE8704003F0B5BF70B5054605211A
:1052300008F036FF040000D1FFDF04F10803214627
:105240002846BDE870400422B1E470B5054605214A
:1052500008F026FF040000D1FFDF2146284623681E
:10526000BDE870400522A2E470B50646052108F0AD
:1052700017FF040000D1FFDF04F1120003F050FF1C
:10528000401D20F0030511E0011D00880322431892
:1052900021463046FFF78BFC00280BD0607BABB279
:1052A000684382B26068011D08F0D5FD60684188DE
:1052B0000029E9D170BD70B50E46054602F002FE28
:1052C000040000D1FFDF0120207266726580207823
:1052D00020F00F00C01C20F0F00030302070BDE83E
:1052E000704002F0F2BD2DE9F0438BB00D4614463C
:1052F000814606A9FFF799FB002814D14FF6FF76E7
:1053000001274FF420588CB103208DF800001020A5
:10531000ADF8100007A8059007AA204604A90AF0D6
:105320006BFC78B107200BB0BDE8F0830820ADF826
:1053300008508DF80E708DF80000ADF80A60ADF8D9
:105340000C800CE00698A17801742188C1818DF849
:105350000E70ADF80850ADF80C80ADF80A606A46E2
:1053600002214846069BFFF789FBDCE708B50122CE
:105370008DF8022042F60202ADF800200A4603230F
:105380006946FFF73EFC08BD08B501228DF80220F2
:1053900042F60302ADF800200A4604236946FFF7EF
:1053A00030FC08BD00B587B079B102228DF800202D
:1053B0000A88ADF808204988ADF80A1000236A462B
:1053C0000521FFF75BFB07B000BD1020FBE709B12B
:1053D000072316E40720704770B588B00D461446C1
:1053E000064606A9FFF721FB00280ED17CB1062056
:1053F000ADF808508DF80000ADF80A40069B6A46EB
:105400000821DC813046FFF739FB08B070BD05206C
:105410008DF80000ADF80850F0E700B587B059B13D
:1054200007238DF80030ADF80820039100236A4669
:105430000921FFF723FBC6E71020C4E770B588B049
:105440000C460646002506A9FFF7EFFA0028DCD136
:1054500006980121123003F095FE9CB121780629AF
:1054600021D2DFE801F0200505160318801E80B266
:10547000C01EE28880B20AB1A3681BB1824203D980
:105480000C20C2E71020C0E7042904D0A08850B93E
:1054900001E00620B9E7012913D0022905D004292B
:1054A0001CD005292AD00720AFE709208DF800007D
:1054B0006088ADF80800E088ADF80A00A0680390A5
:1054C00023E00A208DF800006088ADF80800E0882D
:1054D000ADF80A00A0680A25039016E00B208DF8AD
:1054E00000006088ADF80800A088ADF80A00E088E8
:1054F000ADF80C00A0680B25049006E00C208DF898
:10550000000060788DF808000C256A462946304670
:10551000069BFFF7B3FA78E700B587B00D228DF848
:105520000020ADF8081000236A461946FFF7A6FAD6
:1055300049E700B587B071B102228DF800200A88D2
:10554000ADF808204988ADF80A1000236A46062104
:10555000FFF794FA37E7102035E770B586B00646B6
:1055600001200D46ADF808108DF80000014600231B
:105570006A463046FFF782FA040008D129463046D1
:1055800001F004FB0021304601F01EFB204606B06E
:1055900070BDF8B51C4615460E46069F08F0B2FED3
:1055A0002346FF1DBCB231462A46009408F0BBFAE0
:1055B000F8BD30B41146DDE902423CB1032903D005
:1055C000002330BC06F026B80123FAE71A8030BC6D
:1055D000704770B50C460546FFF72FFB214628465D
:1055E00001F0E3FA2846BDE87040012101F0ECBA71
:1055F00018B18178012938D101E010207047018865
:1056000042F60112881A914231D018DC42F60102AA
:10561000A1EB020091422AD00CDC41B3B1F5C05F8E
:1056200025D06FF4C050081821D0A0F57060FF3865
:105630001BD11CE001281AD002280AD117E0B0F5CE
:10564000807F14D008DC012811D002280FD0032855
:105650000DD0FF2809D10AE0B0F5817F07D0A0F571
:105660008070033803D0012801D0002070470F203C
:1056700070470A281FD008DC0A2818D2DFE800F09B
:10568000191B1F1F171F231D1F21102815D008DCF1
:105690000B2812D00C2810D00D2816D00F2806D1B8
:1056A0000DE011280BD084280BD087280FD00320C1
:1056B00070470020704705207047072070470F2073
:1056C000704704207047062070470C20704743F253
:1056D0000200704738B50C46050041D06946FEF718
:1056E000DBFA002819D19DF80010607861F3020000
:1056F00060706946681CFEF7CFFA00280DD19DF84E
:105700000010607861F3C5006070A978C1F34101B1
:10571000012903D0022905D0072038BD217821F0C6
:10572000200102E0217841F020012170410704D0DE
:10573000A978C90861F386106070607810F0380F9E
:1057400007D0A978090961F3C710607010F0380F0D
:1057500002D16078400603D5207840F040002070E8
:10576000002038BD70B504460020088015466068EA
:10577000FFF7B0FF002816D12089A189884211D8EF
:1057800060688078C0070AD0B1F5007F0AD840F27F
:105790000120B1FBF0F200FB1210288007E0B1F508
:1057A000FF7F01D90C2070BD01F20121298000206A
:1057B00070BD10B50478137864F300031370047897
:1057C000640864F3410313700478A40864F382034B
:1057D00013700478E40864F3C30313700478240995
:1057E00064F3041313700478640964F345131370AD
:1057F0000078800960F38613137031B10878C1070F
:1058000001D1800701D5012000E0002060F3C7131B
:10581000137010BD4278530702D002F0070306E070
:1058200012F0380F02D0C2F3C20300E001234A781D
:1058300063F302024A70407810F0380F02D0C0F3D0
:10584000C20005E0430702D000F0070000E001209D
:1058500060F3C5024A7070472DE9F04F95B00D0016
:10586000824612D01221284612F065FE4FF6FF7BC9
:1058700005AA0121584605F02AFB00242646374692
:105880004FF420586FF4205973E0102015B0BDE894
:10589000F08F00BF9DF81E0001280AD1BDF81C1032
:1058A00041450BD011EB09000AD001280CD0022889
:1058B0000CD0042C0ED0052C0FD10DE0012400E0FB
:1058C0000224BDF81A6008E0032406E00424BDF8B1
:1058D0001A7002E0052400E00624BDF81A105145B4
:1058E00047D12C74BEB34FF0000810AA4FF0070A3E
:1058F000CDE90282CDE900A80DF13C091023CDF8D5
:10590000109042463146584605F094FB08BBBDF85E
:105910003C002A46C0B210A90AF04FF9C8B9AE81BE
:10592000CFB1CDE900A80DF1080C0AAE40468CE8D5
:105930004102132300223946584605F07BFB40B94B
:10594000BDF83C00F11CC01EC0B22A1D0AF035F99A
:1059500010B103209AE70AE0BDF82900E881062C7F
:1059600005D19DF81E00A872BDF81C0028810020FA
:105970008CE705A805F0B7FA00288BD0FFF779FE71
:1059800084E72DE9F0471C46DDE90978DDF8209031
:1059900015460E00824600D1FFDF0CB1208818B1F9
:1059A000D5B11120BDE8F087022D01D0012100E022
:1059B000002106F1140004F079F9A8F8000002466D
:1059C0003B462946504605F0EFFCC9F8000008B9EF
:1059D000A41C3C600020E5E71320E3E7F0B4144684
:1059E000DDE904528DB1002314B1022C09D101E08C
:1059F000012306E00D7CEE0703D025F0010501230D
:105A00000D742146F0BC05F005BE1A80F0BC70474D
:105A10002DE9FE4F91461A881C468A468046FAB107
:105A200002AB494605F0C0FC050019D04046A61C53
:105A3000278808F079FC3246072629463B4600961F
:105A400008F0A5F820882346CDE900504A46514683
:105A50004046FFF7C3FF002020800120BDE8FE8FF5
:105A60000020FBE72DE9F04786B082460EA890465D
:105A700090E8B000894604AA05A903A88DE80700AC
:105A80001E462A4621465046FFF77BFF039901B187
:105A900001213970002818D1F94904F1140204AB2E
:105AA0000860039805998DE807004246494650462C
:105AB00004F0B3FCA8B1092811D2DFE800F0050812
:105AC0000510100A0C0C0E00002006B06AE7112029
:105AD000FBE70720F9E70820F7E70D20F5E70320AB
:105AE000F3E7BDF810100398CDE9000133462A46CC
:105AF00021465046FFF772FFE6E72DE9F04389B0F3
:105B00000D46DDE9108781461C461646142103A880
:105B100012F033FD012002218DF810108DF80C00D9
:105B20008DF81170ADF8146064B1A278D20709D075
:105B30008DF81600E088ADF81A00A088ADF81800BE
:105B4000A068079008A80095CDE90110424603A976
:105B500048466B68FFF786FF09B0BDE8F083F0B5F3
:105B60008BB000240646069407940727089405A8DE
:105B70000994019400970294CDE903400D46102347
:105B80002246304605F056FA78B90AA806A90194CB
:105B900000970294CDE90310BDF814300022294685
:105BA000304605F01DF8002801D0FFF762FD0BB06C
:105BB000F0BD04F0BDBE2DE9FC410C468046002638
:105BC00002F080F9054620780D287DD2DFE800F04C
:105BD000BC0713B325BD49496383AF959B00A84813
:105BE000006820B1417841F010014170ADE04046BD
:105BF00002F098F9A9E00421404608F051FA0700A4
:105C000000D1FFDF07F11401404603F0E3FFA5BB1D
:105C100013214046FCF762FD97E00421404608F05E
:105C20003FFA070000D1FFDFE088ADF80000002058
:105C3000B8819DF80000010704D5C00602D5A088F0
:105C4000B88105E09DF8010040067ED5A088F88166
:105C500005B9FFDF22462946404601F0BDFC022679
:105C600073E0E188ADF800109DF8011009060FD52A
:105C7000072803D006280AD00AE024E00421404681
:105C800008F00EFA060000D1FFDFA088F08102269E
:105C9000CDB9FFDF17E00421404608F001FA070004
:105CA00000D1FFDF07F1140004F079FE90F0010F3E
:105CB00002D1E079000648D5387C022640F0020087
:105CC000387405B9FFDF00E03EE022462946404631
:105CD00001F082FC39E00421404608F0E1F9017C42
:105CE000002D01F00206C1F340016171017C21F039
:105CF00002010174E7D1FFDFE5E7022601214046FA
:105D000002F042F921E00421404608F0C9F90546B5
:105D1000606800902089ADF8040001226946404681
:105D200002F053F9287C20F0020028740DE0002DC9
:105D3000C9D1FFDFC7E7022600214046FFF766FA18
:105D4000002DC0D1FFDFBEE7FFDF3046BDE8FC819C
:105D50003EB50C0009D001466B4601AA002005F0B3
:105D6000EBF920B1FFF785FC3EBD10203EBD0020C1
:105D70002080A0709DF8050002A900F00700FDF743
:105D8000A7FF50B99DF8080020709DF8050002A9F2
:105D9000C0F3C200FDF79CFF08B103203EBD9DF893
:105DA000080060709DF80500C109A07861F3041037
:105DB000A0709DF80510890961F3C300A0709DF8DB
:105DC0000410890601D5022100E0012161F342009F
:105DD0009DF8001061F30000A07000203EBD70B57A
:105DE000144606460D4651EA040005D075B1084632
:105DF000FBF793FA78B901E0072070BD29463046D9
:105E000005F0FBF910B1BDE8704032E454B1204612
:105E1000FBF783FA08B1102070BD21463046BDE87B
:105E2000704095E7002070BD2DE9FC5F0C46904660
:105E30000546002701780822007A3E46B2EB111F82
:105E40007ED104F10A0100910A31821E4FF0020A4C
:105E500004F1080B0191092A73D2DFE802F0ECDFAC
:105E600005F427277AA9CD006888042108F018F9DD
:105E7000060000D1FFDFB08920B152270726C2E01B
:105E80003C02002051271026002C7DD06888A0807D
:105E90000120A071A88900220099FFF7A0FF002827
:105EA00073D1A8892081288AE081D1E0B5F81290C9
:105EB000072824D1E87B000621D5512709F11400D9
:105EC00086B2002CE1D0A88900220099FFF787FF55
:105ED00000285AD16888A08084F806A0A88920816B
:105EE0000120A073288A2082A4F81290A88A00902A
:105EF00068884B46A969019A01F04BFBA8E050273E
:105F000009F1120086B2002C3ED0A8890022594621
:105F1000FFF765FF002838D16888A080A889E08055
:105F2000287A072813D002202073288AE081E87B92
:105F3000C0096073A4F81090A88A0090688801E0F6
:105F400083E080E04B4604F11202A969D4E7012006
:105F5000EAE7B5F81290512709F1140086B2002C37
:105F600066D06888042108F09BF883466888A08082
:105F7000A88900220099FFF732FF00286ED184F82B
:105F800006A0A889208101E052E067E00420A07308
:105F9000288A2082A4F81290A88A009068884B462C
:105FA000A969019A01F0F5FAA989ABF80E104FE042
:105FB0006888FBF7DDFB07466888042108F070F865
:105FC000064607B9FFDF06B9FFDF687BC00702D0CE
:105FD0005127142601E0502712264CB36888A08070
:105FE000502F06D084F806A0287B594601F0E1FA2C
:105FF0002EE0287BA11DF9E7FE49A8894989814245
:1060000005D1542706269CB16888A08020E053273C
:106010000BE06888A080A889E08019E068880421E6
:1060200008F03EF800B9FFDF55270826002CF0D114
:10603000A8F8006011E056270726002CF8D06888E1
:10604000A080002013E0FFDF02E0012808D0FFDF7E
:10605000A8F800600CB1278066800020BDE8FC9F96
:1060600057270726002CE3D06888A080687AA071A3
:10607000EEE7401D20F0030009B14143091D01EB8B
:106080004000704713B5DB4A00201071009848B1FA
:106090000024684607F03FFE002C02D1D64A009942
:1060A00011601CBD01240020F4E770B50D460646C2
:1060B00086B014465C21284612F05FFA04B9FFDF6F
:1060C000A0786874A2782188284601F09CFA002004
:1060D000A881E881228805F11401304603F05FFDB4
:1060E0006A460121304604F0F2FE19E09DF80300F3
:1060F000000715D5BDF806103046FFF730FD9DF8B6
:106100000300BDF8061040F010008DF80300BDF844
:106110000300ADF81400FF233046059A05F038F867
:10612000684604F0E0FE0028E0D006B070BD10B56F
:106130000C4601F1140003F069FD0146627C204623
:10614000BDE8104001F094BA30B50446A94891B0BA
:106150004FF6FF75C18905AA284604F0B8FE30E065
:106160009DF81E00A0422AD001282AD1BDF81C00AB
:10617000B0F5205F03D042F60101884221D1002012
:1061800002AB0AAA0CA9019083E80700072000903F
:10619000BDF81A1010230022284604F04BFF38B92E
:1061A000BDF828000BAAC0B20CA909F006FD10B179
:1061B000032011B030BD9DF82E00A04201D1002077
:1061C000F7E705A804F08FFE0028C9D00520F0E706
:1061D00070B50546042107F063FF040000D1FFDF1E
:1061E00004F114010C46284603F0F4FC214628462D
:1061F000BDE8704003F0F5BC70B58AB00C460646A9
:10620000FBF7B6FA050014D02878222827D30CB162
:10621000A08890B101208DF80C0003208DF81000AB
:1062200000208DF8110054B1A088ADF81800206846
:1062300007E043F202000AB070BD0920FBE7ADF8A9
:10624000180005900421304607F02AFF040000D111
:10625000FFDF04F1140003F0F0FC000701D4082074
:10626000E9E701F02FFE60B108A802210094CDE912
:10627000011095F8232003A930466368FFF7F2FB6D
:10628000D9E71120D7E72DE9F04FB2F802A08346F5
:1062900089B0154689465046FBF76AFA074604213D
:1062A000504607F0FDFE0026044605964FF0020812
:1062B0000696ADF81C6007B9FFDF04B9FFDF414661
:1062C000504605F029FB50B907AA06A905A88DE894
:1062D00007004246214650466368FFF752FB454897
:1062E00007AB0660DDE9051204F11400CDF800905B
:1062F000CDE90320CDE9013197F8232059465046D6
:106300006B6803F0E3FC06000AD0022E04D0032ED3
:1063100014D0042E00D0FFDF09B03046BDE8F08F66
:10632000BDF81C000028F7D00599CDE900104246C1
:10633000214650466368FFF751FBEDE7687840F06F
:1063400008006870E8E72DE9F04F99B004464FF077
:1063500000082848ADF81C80ADF82080ADF82480F6
:10636000A0F80880ADF81480ADF81880ADF82C8046
:10637000ADF82880007916460D464746012808D01A
:10638000022806D0032804D0042802D0082019B01F
:10639000C4E72046FAF77DFF80BB2846FAF779FF6D
:1063A00060BB6068FAF7C2FF40BB606848B16089B3
:1063B0002189884202D8B1F5007F01D90C20E6E797
:1063C00080460EAA06A92846FFF7CCF90028DED1A0
:1063D00068688078C0F34100022808D19DF8190050
:1063E00010F0380F03D02869FAF797FF30B905A9E4
:1063F000206904E03C0200201400002020E0FFF7A8
:1064000069F90028C3D1206948B1607880079DF8F8
:10641000150000F0380001D5F0B300E0E0BB9DF8B6
:10642000140080060ED59DF8150010F0380F03D02B
:106430006068FAF772FF18B96068FAF777FF08B179
:106440001020A4E70AA96069FFF744F900289ED14B
:10645000606940B19DF8290000F0070101293CD195
:1064600010F0380F39D00BA9A069FFF733F90028D5
:106470008DD19DF8280080062FD49DF82C00800631
:106480002BD4A06950B19DF82D0000F0070101291F
:1064900023D110F0380F00E01FE01ED0E06818B1E3
:1064A0000078D0B11C2818D20FAA611C2046FFF733
:1064B00080F90121384661F30F2082468DF8521091
:1064C000B94642F603000F46ADF850000DF13F0209
:1064D00018A9286809F090FB08B1072057E79DF834
:1064E000600015A9CDF80090C01CCDE9019100F025
:1064F000FF0B00230BF20122514614A804F02AFCE2
:10650000F0BBBDF854000C90FD492A89286900921F
:10651000CDE901016B89BDF838202868069904F09F
:1065200019FC01007ED120784FF0020AC10601D487
:1065300080062BD5ADF80C90606950B90AA906A861
:10654000FFF768F99DF8290020F00700401C8DF83E
:1065500029009DF8280008A940F0C8008DF82800FF
:106560008DF8527042F60210ADF8500003AACDF833
:1065700000A0CDE90121002340F2032214A800E08D
:106580001EE00A9904F0E6FB01004BD1DC484D46C1
:1065900008385B460089ADF83D000FA8CDE90290B0
:1065A000CDF80490CDF810904FF007090022CDF8F7
:1065B0000090BDF854104FF6FF7004F011FB10B1BD
:1065C000FFF757F8E3E69DF83C00000625D529467D
:1065D000012060F30F218DF852704FF42450ADF874
:1065E0005000ADF80C5062789DF80C00002362F367
:1065F00000008DF80C006278CDF800A0520862F31C
:1066000041008DF80C0003AACDE9012540F20322D8
:1066100014A804F09FFB010004D1606888B32069CE
:10662000A8B900E086E005A906A8FFF7F3F86078AE
:10663000800706D49DF8150020F038008DF815006D
:1066400005E09DF8140040F040008DF814008DF82E
:10665000527042F60110ADF85000208940F201213D
:10666000B0FBF1F201FB1202606809ABCDF80080CB
:10667000CDE90103002314A8059904F06BFB010088
:1066800058D12078C00729D0ADF80C50A06950B976
:106690000BA906A8FFF7BEF89DF82D0020F0070013
:1066A000401C8DF82D009DF82C008DF8527040F0A4
:1066B00040008DF82C0042F60310ADF8500007A9F9
:1066C00003AACDF800A0CDE90121002340F2032266
:1066D00014A80B9904F03EFB01002BD1E06868B3CD
:1066E0002946012060F30F218DF8527042F6041004
:1066F000ADF85000E068002302788DF8582040780B
:106700008DF85900E06816AA4088ADF85A00E06894
:1067100000798DF85C00E068C088ADF85D00CDF8C8
:106720000090CDE901254FF4027214A804F012FB89
:10673000010003D00C9800F0C7FF28E67048032141
:106740000838017156B100893080BDF8240070808E
:10675000BDF82000B080BDF81C00F080002016E6D7
:1067600070B501258AB016460B46012802D00228D2
:1067700016D104E08DF80E504FF4205003E08DF850
:106780000E5042F60100ADF80C005BB10024601C15
:1067900060F30F2404AA08A9184609F02DFA18B1CD
:1067A000072048E5102046E504A99DF8202054481C
:1067B000CDE90021801E02900023214603A802F2A9
:1067C000012204F0C7FA10B1FEF753FF33E54C483D
:1067D00008380EB1C1883180057100202BE5F0B575
:1067E00093B0074601268DF83E6041F60100ADF8F2
:1067F0003C0012AA0FA93046FFF7B2FF002848D18B
:106800003F4C0025083CE7B31C2102A811F0B5FE5F
:106810009DF808008DF83E6040F020008DF80800DB
:1068200042F60520ADF83C000E959DF83A00119512
:1068300020F00600801C8DF83A009DF838006A466A
:1068400020F0FF008DF838009DF8390009A920F0EC
:10685000FF008DF839000420ADF82C00ADF83000B1
:106860000EA80A9011A80D900FA80990ADF82E500F
:1068700002A8FFF768FD00280BD1BDF80000608179
:1068800000E008E0BDF80400A081401CE081257113
:10689000002013B0F0BD6581A581BDF84800F4E784
:1068A0002DE9F74F1649A0B00024083917940A794A
:1068B000A146012A04D0022A02D0082023B02DE5E7
:1068C000CA88824201D00620F8E721988A4682428F
:1068D00001D10720F2E701202146ADF848004FF62C
:1068E000FF788DF86E0042F6020B60F30F21ADF8D1
:1068F0004A80ADF86CB006918DF8724002E000005D
:10690000440200201CA9ADF870401391ADF85080EE
:1069100012A804F00CFB00252E462F460DAB0722D3
:1069200012A9404604F006FB78B10A285DD195B360
:106930008EB3ADF86450ADF866609DF85E008DF8DA
:10694000144019AC012864D06BE09DF83A001FB3E5
:10695000012859D1BDF8381059451FD118A809A9E7
:1069600001940294CDE9031007200090BDF8361081
:1069700010230022404604F05DFBB0BBBDF8600070
:10698000042801D006284AD1BDF82410219881425C
:106990003AD10F2092E73AE0012835D1BDF838000E
:1069A000B0F5205F03D042F6010188422CD1BAF83D
:1069B0000600BDF83610884201D1012700E000270B
:1069C00005B19EB1219881421ED118A809AA01944F
:1069D0000294CDE90320072000900D4610230022E9
:1069E000404604F027FB00B902E02DE04E460BE0E4
:1069F000BDF86000022801D0102810D1C0B217AA3B
:106A000009A909F0DAF850B9BDF8369086E70520F3
:106A100054E705A917A8221D09F0EEF808B10320D4
:106A20004CE79DF814000023001DC2B28DF814201D
:106A300022980092CDE901401BA8069904F08AF93A
:106A400010B902228AF80420FEF713FE36E710B5CB
:106A50000B46401E88B084B205AA00211846FEF7F6
:106A6000A8FE00200DF1080C06AA05A901908CE8EB
:106A70000700072000900123002221464FF6FF70F7
:106A800004F0AEF80446BDF81800012800D0FFDF7E
:106A90002046FEF7EEFD08B010BDF0B5F74F0446F6
:106AA00087B038790E46032804D0042802D0082085
:106AB00007B0F0BD04AA03A92046FEF753FE050067
:106AC000F6D160688078C0F3410002280AD19DF8B1
:106AD0000D0010F0380F05D02069FAF71EFC08B140
:106AE0001020E5E7208905AA21698DE80700638960
:106AF000BDF810202068039904F02CF910B1FEF7BE
:106B0000B8FDD5E716B1BDF8140030800420387107
:106B10002846CDE7F8B50C0006460CD001464FF6E6
:106B2000FF7500236A46284604F006FB28B100BF23
:106B3000FEF79FFDF8BD1020F8BD69462046FEF720
:106B4000C9FD0028F8D1A078314600F0010328469D
:106B5000009A04F01DFBEBE730B587B01446002225
:106B60000DF1080C05AD01928CE82C000722009273
:106B70000A46014623884FF6FF7004F031F8BDF84D
:106B800014102180FEF775FD07B030BD70B50D46BD
:106B9000042107F085FA040000D1FFDF294604F143
:106BA0001400BDE8704003F041B870B50D460421F3
:106BB00007F076FA040000D1FFDF294604F1140043
:106BC000BDE8704003F055B870B50D46042107F0DC
:106BD00067FA040000D1FFDF294604F11400BDE884
:106BE000704003F06DB870B50546042107F058FAFF
:106BF000040000D1FFDF214628462368BDE870402D
:106C00000122FEF705BF70B50646042107F048FAD9
:106C1000040000D1FFDF04F1140002F0F7FF401D73
:106C200020F0030511E0011D0088002243182146D1
:106C30003046FEF7EDFE00280BD0607CABB2684317
:106C400082B2A068011D07F006F9A06841880029FA
:106C5000E9D170BD70B50546042107F021FA0400A2
:106C600000D1FFDF214628466368BDE8704002225C
:106C7000FEF7CEBE70B50E46054601F023F90400BE
:106C800000D1FFDF0120207266726580207820F03D
:106C90000F00001D20F0F00040302070BDE8704073
:106CA00001F013B910B50446012900D0FFDF2046DA
:106CB000BDE810400121FEF7A9BA2DE9F04F97B0C9
:106CC0004FF0000A0C008346ADF814A0D04619D04E
:106CD000E06830B1A068A8B10188ADF81410A0F840
:106CE00000A05846FAF744FD070043F2020961D0BC
:106CF000387822285CD30421584607F0D1F90500E2
:106D000005D103E0102017B0BDE8F08FFFDF05F1DB
:106D1000140002F07BFF401D20F00306A07801283C
:106D200003D0022801D00720EDE7218807AA5846A2
:106D300004F0CDF830BB07A804F0D5F810BB07A8C5
:106D400004F0D1F848B99DF82600012805D1BDF816
:106D50002400A0F52451023902D04FF45050D2E75C
:106D6000E068B0B1CDE902A00720009005AACDF8F7
:106D700004A00492A2882188BDF81430584603F07C
:106D80002FFF10B1FEF775FCBDE7A168BDF8140038
:106D900008809DF81F00C00602D543F20140B2E70B
:106DA0000B9838B1A1780078012905D080071AD452
:106DB0000820A8E74846A6E7C007F9D002208DF8CA
:106DC0003C00A8684FF00009A0B1697C428871437B
:106DD00091420FD98AB2B3B2011D06F0F2FF80468C
:106DE000A0F800A006E003208DF83C00D5F8008054
:106DF0004FF001099DF8200010F0380F00D1FFDF9F
:106E00009DF820001E49C0F3C200084497F82310E3
:106E100010F8010C884201D90F2074E72088ADF8E2
:106E2000400014A90095CDE90191434607220FA91E
:106E30005846FEF717FE002891D19DF8500050B932
:106E4000A078012807D1687CB3B2704382B2A868E9
:106E5000011D06F0CAFF002055E770B5064615462D
:106E60000C460846FEF7C4FB002805D12A462146F9
:106E70003046BDE8704073E470BD11E53C0200206F
:106E80000689010070B51E4614460D0009D044B1B4
:106E9000616831B138B1FC49C988814203D007200B
:106EA00070BD102070BD2068FEF7A2FB0028F9D14C
:106EB000324621462846BDE87040FFF744BA70B517
:106EC00015460C0006D038B1EF490989814203D03C
:106ED000072070BD102070BD2068FEF789FB0028D8
:106EE000F9D129462046BDE87040D6E570B5064682
:106EF00086B00D4614461046FAF7F1F9D0BB60682B
:106F0000FAF714FAB0BBA6F57F40FF3803D030463D
:106F1000FAF72EFC80B128466946FEF79DFC002852
:106F20000CD19DF810100F2008293DD2DFE801F0A8
:106F300008060606060A0A0843F2020006B070BDFB
:106F40000320FBE79DF80210012908D1BDF80010CD
:106F5000B1F5C05FF2D06FF4C052D142EED09DF8CF
:106F6000061001290DD1BDF80410A1F528510629FC
:106F700007D200E029E0DFE801F003030403030384
:106F8000DCE79DF80A1001290FD1BDF80810B1F512
:106F9000245FD3D0A1F60211B1F50051CED0012962
:106FA000CCD0022901D1C9E7FFDF606878B900239E
:106FB00005AA2946304604F0BFF810B1FEF759FB88
:106FC000BCE79DF81400800601D41020B6E7618864
:106FD000224628466368FFF7BFFDAFE72DE9F0437F
:106FE000814687B0884614461046FAF778F918B1FA
:106FF000102007B0BDE8F083002306AA41464846AA
:1070000004F09AF818B100BFFEF733FBF1E79DF8E2
:107010001800C00602D543F20140EAE70025072721
:1070200005A8019500970295CDE9035062884FF6B7
:10703000FF734146484603F0FDFF060013D1606828
:10704000FAF74DF960B960680195CDE902500097F3
:107050000495238862884146484603F0EBFF0646C4
:10706000BDF8140020803046CEE739B1864B0A883F
:107070009B899A4202D843F2030070471DE610B57F
:1070800086B0814C0423ADF81430638943B1A489E0
:107090008C4201D2914205D943F2030006B010BDE3
:1070A0000620FBE7ADF81010002100910191ADF82A
:1070B000003002218DF8021005A9029104A9039164
:1070C000ADF812206946FFF7F8FDE7E72DE9FC4728
:1070D00081460D460846FAF7DCF888BB4846FAF7C1
:1070E00047FB5FEA00080AD098F80000222829D35D
:1070F0000421484606F0D4FF070005D103E043F21F
:107100000200BDE8FC87FFDF07F1140002F095FDE7
:1071100006462878012803D0022804D00720F0E78B
:10712000B0070FD502E016F01C0F0BD0A8792C1D6C
:10713000C00709D0E08838B1A068FAF7AAF818B1FA
:107140001020DEE70820DCE721882A780720B1F547
:10715000847F35D01EDC40F20315A1F20313A9424F
:1071600026D00EDCB1F5807FCBD003DCF9B101294C
:1071700026D1C6E7A1F58073013BC2D0012B1FD1F8
:1071800013E0012BBDD0022B1AD0032BB9D0042B56
:1071900016D112E0A1F20912082A11D2DFE802F09A
:1071A0000B04041010101004ABE7022AA9D007E06A
:1071B000012AA6D004E0320700E0F206002AA0DA95
:1071C000CDB200F07FFE50B198F82300CDE9000564
:1071D000FA89234639464846FEF78FFC91E711208D
:1071E0008FE72DE9F04F8BB01F4615460C468346BE
:1071F0000026FAF7BDFA28B10078222805D2082027
:107200000BB081E543F20200FAE7B80801D007208D
:10721000F6E7032F00D100274FF6FF79CCB1022DFE
:1072200073D32046FAF782F830B904EB0508A8F1C9
:107230000100FAF77BF808B11020E1E7AD1EAAB211
:107240002146484604F046F838F8021C88425CD1D2
:10725000ADB20D49B80702D58889401C00E0012075
:107260001FFA80F8F80701D08F8900E04F4605AA81
:107270004146584603F02BFE4FF0070A4FF0000935
:10728000DCB320460BE000003C02002040881028C0
:107290003BD8361D304486B2AE4236D2A0190288A1
:1072A0004245F3D351E000BF9DF8170002074CD5CB
:1072B00094B304EB0608361DB8F80230B6B2102BB2
:1072C00023D89A19AA4220D8B8F8002091421CD19C
:1072D000C0061CD5CDE900A90DF1080C0AAAA11918
:1072E00048468CE80700B8F800100022584603F022
:1072F00077FC20B1FEF7BDF982E726E005E0B8F89B
:107300000200BDF82810884201D00B2078E7B8F8B9
:107310000200304486B207E0FFE7C00604D55846B5
:10732000FEF71DFC002888D19DF81700BDF81A1043
:1073300020F010008DF81700BDF81700ADF8000020
:10734000FF235846009A03F023FF05A803F0CBFD66
:1073500018B9BDF81A10B942A6D90421584606F04A
:107360009FFE040000D1FFDFA2895AB1CDE900A938
:107370004D46002321465846FEF7BFFB0028BBD1EF
:10738000A5813DE700203BE72DE9FF4F8BB01E466E
:1073900017000D464FF0000412D0B00802D00720AD
:1073A0000FB0B1E4032E00D100265DB10846F9F715
:1073B000B4FF28B93888691E0844F9F7AEFF08B150
:1073C0001020EDE7C64AB00701D5D18900E00121C0
:1073D000F0074FF6FF7802D0D089401E00E040460B
:1073E00086B206AA0B9803F072FD4FF000094FF029
:1073F000070B0DF1140A38E09DF81B00000734D587
:10740000CDF80490CDF800B0CDF80890CDE9039AFE
:10741000434600220B9803F00DFE60BB05B3BDF898
:1074200014103A8821442819091D8A4230D3BDF826
:107430001E2020F8022BBDF8142020F8022BCDE9E5
:1074400000B9CDE90290CDF810A0BDF81E10BDF82E
:10745000143000220B9803F0EDFD08B103209FE7E4
:10746000BDF814002044001D84B206A803F03BFDC3
:1074700020B10A2806D0FEF7FCF891E7BDF81E10EF
:10748000B142B9D934B17DB13888A11C884203D248
:107490000C2085E7052083E722462946404603F075
:1074A00019FF014628190180A41C3C80002077E7C1
:1074B00010B50446F9F713FF08B1102010BD884835
:1074C000C0892080002010BDF0B58BB00D46064667
:1074D000142103A811F051F801208DF80C008DF84B
:1074E000100000208DF81100ADF814503046FAF766
:1074F0003FF948B10078222812D30421304606F023
:10750000CFFD040005D103E043F202000BB0F0BD53
:10751000FFDF04F11400074602F08FFB800601D460
:107520000820F3E7207C022140F00100207409A824
:107530000094CDE90110072203A930466368FEF7E5
:1075400091FA20B1217C21F001012174DEE7294666
:107550003046FDF74CFE08A9384602F05DFB00B14D
:10756000FFDFBDF82040172C01D2172000E0204695
:10757000A84201D92C4602E0172C00D2172421463C
:107580003046FFF712FB21463046FDF756FB002040
:10759000BCE7F8B51C4615460E46069F06F0B2FE3F
:1075A0002346FF1DBCB231462A46009406F0BBFAC2
:1075B000F8BD70B50C4605460E21204610F0BBFF05
:1075C000002020802DB1012D01D0FFDF70BD0620ED
:1075D00000E00520A07170BD10B548800878134602
:1075E00020F00F00001D20F0F00080300C460870E5
:1075F0001422194604F1080010F063FF00F065FC46
:107600003748046010BD2DE9F047DFF8D890491DD8
:10761000064621F0030117460C46D9F8000006F093
:1076200098FB050000D1FFDF4FF000083560A5F89A
:1076300000802146D9F8000006F08BFB050000D140
:10764000FFDF7560A5F800807FB104FB07F1091D1D
:107650000BD0D9F8000006F07CFB040000D1FFDF5E
:10766000B460C4F80080BDE8F087C6F80880FAE787
:107670002DE9F0411746491D21F00302194D064638
:1076800001681446286806F08FFB22467168286856
:1076900006F08AFB3FB104FB07F2121D03D0B1686C
:1076A000286806F081FB042006F0A6FC04460420AE
:1076B00006F0AAFC201A012804D12868BDE8F04190
:1076C00006F03CBBBDE8F08110B50C4603F0CBFBE7
:1076D00000B1FFDF2046BDE81040FDF7CABF000043
:1076E0003C0200201400002038B582880A800C4635
:1076F000C188121D90B26A4605F0D9FDBDF80000A0
:10770000032800D30320C1B2208800F0B4FF38BDA5
:1077100038B582880A800C46C188121D90B26A462C
:1077200005F0C5FDBDF80000022800D30220C1B25B
:10773000208800F0A0FF401CC0B238BD2DE9FE4FEC
:1077400082468B46F74814460BF10302D0E900103D
:10775000CDE9011022F0030268462C21009206F0C8
:10776000DAFAF14E002C02D1F04A009991600099AA
:1077700001440091357E05F1010504D1E8B208F01D
:10778000B5F900B1FFDF009800EB0510C01C20F038
:107790000301009144B9727A00200870B08B80B266
:1077A00003F0E9F900B1FFDF0098F16908440090A7
:1077B0002146684600F023FF80460098C01C20F058
:1077C00003000090717A04B1002006F08EFB00994E
:1077D000084400902146684600F058FFD248002730
:1077E0003D4690F801900CE0284600F0EBFE06467E
:1077F00081788088FDF7B8FA71786D1C00FB0177FD
:10780000EDB24D45F0D10098C01C20F0030000906F
:1078100004B100203946FDF7B2FA00990027084468
:107820000090C1483D4690F801900CE0284600F0D9
:10783000C9FE0646C1788088FEF71BFC71786D1C76
:1078400000FB0177EDB24D45F0D10098C01C20F04F
:107850000300009004B100203946FEF713FC0099A4
:10786000084400210090084603F07EFE2146684649
:1078700000F08BFE0098C01D20F007000090DAF8A1
:107880000010814204D3A0EB0B01B1F5803F04DB73
:107890004FF00408CAF8000004E0CAF80000B8F18C
:1078A000000F02D04046BDE8FE8F34BBA049002047
:1078B000009AFBF70FFBFAF7E6FB9B4801AA0021B1
:1078C0000C30FBF707F800B1FFDF9748407EFEF76A
:1078D00086FF00B1FFDF94484FF4F671343010F0AA
:1078E0004CFE91480421343080F8E91180F8EA1107
:1078F000062180F8EB11032101710020D3E770B558
:10790000894C06463434207804EB4015E07808357D
:1079100090B9A01990F8E80100280ED0A0780F289F
:1079200000D3FFDF2021284610F027FE687866F399
:10793000020068700120E070284670BD2DE9F0411A
:1079400005460C4600270078052190463E46B1EBDF
:10795000101F00D0FFDF287A50B101280ED0FFDFC2
:10796000A8F800600CB1278066800020BDE8F08197
:107970000127092674B16888A08008E00227142630
:1079800044B16888A0802869E060A88A2082287BAA
:107990002072E5E7A8F80060E7E730B5624C012007
:1079A0000021207061702072607221730521A18214
:1079B0001F21E18260735FA121610A212176607637
:1079C0005A4D4FF4B060E0616868C11C21F00301BA
:1079D000814200D0FFDF6868606030BD30B5534C35
:1079E0001568636808339D4202D20420136030BDDD
:1079F0004D4B5D785A6802EBC50210705170032040
:107A0000D080172090800120D07090705878401C52
:107A10005870606808306060002030BD70B5064660
:107A200041480024457807E0204600F0CBFD01786E
:107A3000B14204D0641CE4B2AC42F5D1002070BD68
:107A4000F7B5064608780C46F8B1FFF7E7FF05469C
:107A5000202E06D0212E1AD0222E18D0232E14D15B
:107A600010E000F0BAFD0DB1697800E00021401A85
:107A700081B2A0780144FF2907D830B1A08802283C
:107A800005D202E06088172801D20720FEBD65B943
:107A9000207802AA0121FFF7A1FF0028F6D1207863
:107AA000FFF7BCFF050000D1FFDF202E08D0212EFC
:107AB0000ED0222E0FD0232E07D0FFDF0020FEBDD8
:107AC000A0786870A088E880F8E76088A880F5E76B
:107AD000A078A870F2E7A078E870EFE71A2841D004
:107AE0000DDC13283ED2DFE800F01B3D2C3D3D337A
:107AF000332F31393D3D353D3D3D3D3B0F00302875
:107B000002D003DC1E282DD1072070473A380928FF
:107B100028D2DFE800F021271B272727272713007B
:107B2000002070470C890100780200201800002016
:107B3000000000206E5246357800000043F2040039
:107B4000EFE743F20200ECE70420EAE70D20E8E764
:107B50000F20E6E70820E4E71120E2E71320E0E742
:107B60000620DEE70320DCE710B5007800F0010016
:107B700005F093FBBDE81040B0E710B5007818B1F0
:107B8000012801D0072010BD05F0C7FBBDE810405B
:107B9000A4E710B5007800F0010005F083FBBDE814
:107BA00010409BE70EB5017801F001018DF800103F
:107BB000417801F001018DF801100178C1F3400115
:107BC0008DF802104178C1F340018DF8031001785F
:107BD00089088DF80410417889088DF8051081789E
:107BE0008DF80610C1788DF8071000798DF808001F
:107BF000684605F009F8FFF771FF0EBD2DE9F84F53
:107C0000DFF8F883FE4C00261FE0012000F081FD24
:107C10000120FFF774FE05462C214746D8F80800DE
:107C200006F097F8686000B9FFDF686804F0DFFECF
:107C3000A8B12846F9F7EEFE284600F070FD20B9FD
:107C40002C226968B86806F0AFF894F9E9010428B5
:107C5000DBDA022006F0D0F907460025A5E02C2249
:107C60006968D8F8080006F09FF8F2E7B8F8021043
:107C70004046491C89B2A8F80210B94201D300213C
:107C800041800221B8F8020006F00AFA002864D008
:107C9000B8F80200694605F07EFAFFF71FFF00B151
:107CA000FFDF9DF8000078B1B8F8020006F03CFB59
:107CB0005FEA000900D1FFDF484605F0C8FD18B1B2
:107CC000B8F8020003F017FEB8F8020006F01AFB3D
:107CD0005FEA000900D1FFDF484605F0B0FDE0BBD8
:107CE0000321B8F8020006F0DBF95FEA000B47D188
:107CF000FFDF45E0DBF80C0010B10078FF2849D029
:107D0000022000F006FD0220FFF7F9FD82464846FA
:107D100005F0A1FECAF8040000B9FFDFDAF804009C
:107D200005F069FF002100900170B8F8021050467C
:107D3000AAF8021003F0B5FC484605F05EFF00B952
:107D4000FFDF504600F0EBFC18B99AF8010000077D
:107D500004D50099CBF80C1012E024E0DBF80C00FD
:107D600038B10178491C11F0FF01017008D1FFDF23
:107D700006E000221146484600F005FC00B9FFDF8E
:107D800094F9EA01022805DBB8F8020003F064FC6C
:107D90000028AFD194F9E901042804DB484605F036
:107DA00090FF00B101266D1CEDB2BD4204D294F9E2
:107DB000EA010228BFF65AAF002E7FF424AFBDE8D7
:107DC000F84F032000F0A5BC10B58C4CE0600868AB
:107DD0002061AFF2D710FBF796F8607010BD8848AD
:107DE000002134380170854801708649416098E669
:107DF00070B505464FF080500C46D0F8A410491CD1
:107E000005D1D0F8A810C9430904090C0BD050F8CB
:107E1000A01F01F001012970416821608068A080E5
:107E2000287830B970BD0621204609F07CFB01207E
:107E30002870607940F0C000607170BD70B54FF07F
:107E400080540D46D4F88010491C0BD1D4F884100E
:107E5000491C07D1D4F88810491C03D1D4F88C10E0
:107E6000491C0CD0D4F880100160D4F88410416013
:107E7000D4F888108160D4F88C10C16002E0102121
:107E800009F051FBD4F89000401C0BD1D4F89400B9
:107E9000401C07D1D4F89800401C03D1D4F89C00B2
:107EA000401C09D054F8900F286060686860A06892
:107EB000A860E068E86070BD2846BDE87040102109
:107EC00009F031BB4E48007919E570B54C4CE078AB
:107ED00030B3207804EB4010407A00F007002044D3
:107EE00090F9E801002800DCFFDF2078002504EB92
:107EF0004010407A00F00700011991F8E801401E97
:107F000081F8E8012078401CC0B220700F2800D111
:107F10002570A078401CA07009F0FCF9E57070BDD8
:107F2000FFDF70BD3EB50546032106F0B9F80446F3
:107F3000284606F0E7F9054604B9FFDFE06818B106
:107F40000078FF2800D1FFDF01AA6946284600F02B
:107F50001AFB60B9FFDF0AE0002202A9284600F000
:107F600012FB00B9FFDF9DF8080000B1FFDF9DF8AC
:107F70000000411E8DF80010EED2E06801998842A1
:107F800001D10020E0603EBD70B50546A0F57F4000
:107F90000C46FF3800D1FFDF012C01D0FFDF70BDA0
:107FA000FFF790FF040000D1FFDF207820F00F00E2
:107FB000401D20F0F00050302070658000202072BD
:107FC00001202073BDE870407FE72DE9F04116469F
:107FD0000D460746FFF776FF040000D1FFDF20784B
:107FE00020F00F00401D20F0F0005030207067801E
:107FF0000120207228682061A88805E01800002070
:10800000AC020020340E0020A0822673BDE8F041AF
:108010005BE77FB5FFF702FD040000D1FFDF02A997
:108020002046FFF761FB054603A92046FFF770FBDA
:108030008DF800508DF80100BDF80800001DADF866
:108040000200BDF80C00001DADF80400E088ADF89A
:108050000600684605F009F9002800D0FFDF7FBD63
:108060002DE9F05FFA4F8046387810B10820BDE85E
:10807000F09F4046F9F733F908B11020F7E7F54DC6
:10808000287808B9FFF789FC6C7A464600F0A5FA13
:10809000A04207D2201AC1B232460020FFF79EFC50
:1080A0000028E4D17968BB46C91C21F0030179603E
:1080B0000027E8483E46B946BA463C46457807E0C0
:1080C000204600F07FFA4078641C0644E4B27F1C2E
:1080D000AC42F5D1C6EBC601DE4E0AEB870000EBE1
:1080E0008100717A00EB890000EBC100DBF804101D
:1080F0005C464518012229464046FFF71FFB070052
:1081000012D00020FFF78AFC05000BD005F10B0010
:10811000616820F00300884200D0FFDF7078401EC5
:10812000707065603846A2E7002229464046FFF796
:1081300005FB00B1FFDFD8F8000060604FF6FF706C
:10814000608001202070002091E72DE9F041044675
:10815000BF4817460D46007808B1082006E40846D7
:10816000F9F797F808B11020F8E7BA4E307808B957
:10817000FFF713FC601E1E2807D8012C3DD128787C
:10818000FE283AD830760020E8E7A4F120001F2826
:1081900005D8E0B23A462946BDE8F04150E4A4F1E2
:1081A00040004FF000081F281FD8402C02D0412C5F
:1081B00023D115E028786C78012801D91320CDE768
:1081C000FF2C08D807F082FE074609F05BF8381A42
:1081D000401EA04201DA1220C0E72888308124E046
:1081E0002846BDE8F04100F0C2BAA4F1A0001F2863
:1081F00003D8A02C03D0A12C06D00720AEE7287806
:1082000000F00100707610E029680920F829A5D354
:108210008A07A3D1727B02F00302012A04D1F28AF9
:10822000D73293B28B4299D8F161404696E72DE957
:10823000F04781460E460846F9F751F848B94846D6
:10824000F9F76BF828B909F1030020F0030149455B
:1082500002D01020BDE8F0877E484FF0000A34308D
:10826000817869B14178804600EB41140834378841
:1082700032460021204600F060FA050004D027E0D5
:10828000A6F800A00520E5E7B9F1000F24D030885A
:10829000B84201D90C251FE0607800F00705284698
:1082A00000F037FA08EB0507324697F8E80149462F
:1082B000401C87F8E801204607F5F47700F03DFA06
:1082C00005463878401E3870032000F022FA2DB1A0
:1082D0000C2D01D0A6F800A02846BBE760785C4EC4
:1082E00000F00701012923D002290CD0032933D043
:1082F000FFDF98F801104046491CC9B288F8011008
:108300000F2934D035E0616821B1000702D46088BC
:10831000FFF708FE98F8EA014746012802D1707875
:10832000FAF710FE97F9EA010428E2DBFFDFE0E745
:10833000616819B12C22B06805F036FD98F8E901A2
:108340004746032802D17078FAF7FCFD97F9E90156
:108350000428CEDBFFDFCCE7C00602D56088FFF73C
:10836000E1FD98F9EB010628C3DBFFDFC1E780F8E8
:1083700001A08178491E8170617801F0070101EB4D
:10838000080090F8E811491C80F8E811A4E770B5DE
:108390000D460446F8F77DFF18B92846F8F79FFF09
:1083A00008B1102070BD29462046BDE8704007F096
:1083B000D4BB70B5054607F0F3FBC4B22846F8F706
:1083C000ACFF08B1102070BD35B128782C7018B101
:1083D000A04201D0072070BD2046FDF7B5FE05285C
:1083E00005D107F0E1FB012801D0002070BD0F206E
:1083F00070BD70B5044615460E460846F8F749FFAD
:1084000018B92846F8F76BFF08B1102070BD022C90
:1084100003D0102C01D0092070BD2A4631462046D9
:1084200007F0CBFB0028F7D0052070BD70B51446CF
:108430000D460646F8F72DFF38B92846F8F74FFFE6
:1084400018B92046F8F769FF30B1102070BD000060
:10845000180000207802002022462946304607F006
:10846000CBFB0028F2D00720F0E73EB50446F8F732
:1084700036FF08B110203EBD684604F054FBFFF7FC
:108480002DFB0028F7D19DF806002070BDF80800EC
:108490006080BDF80A00A08000203EBD70B5054692
:1084A0000C460846F8F739FF20B93CB12068F8F7C8
:1084B00016FF08B11020C9E7A08828B12146284638
:1084C000BDE87040FDF798BE0920BFE770B50446CF
:1084D0000D460846F8F7DDFE30B9601E1E2814D898
:1084E0002846F8F7D6FE08B11020AFE7042C01D9D2
:1084F0000720ABE704B9FFDFC24800EB840050F867
:10850000041C2846BDE870400847A4F120001F283D
:1085100005D829462046BDE87040F9F757BDF02C34
:10852000E6D1A868F8F7B5FE0028DDD1284604F0AA
:10853000F9FEBDE87040FFF7D1BA70B504460D46AC
:108540000846F8F7CCFE30B9601E1E2811D8284620
:10855000F8F79FFE08B1102078E7012C05D0022C17
:1085600003D0032C01D0042C01D106206EE7072094
:108570006CE7A4F120001F28F9D829462046BDE861
:108580007040F9F760BD05F029B908B5002918D188
:1085900002F052FE9C4800224178C06804F0FBF9CA
:1085A00099481030C0788DF8000010B1012802D031
:1085B00004E0012000E000208DF80000684604F08F
:1085C0000AFB08BD30B5914D04466878A04200D83A
:1085D000FFDF686800EBC40030BD70B58B48002534
:1085E0002C46467807E02046FFF7ECFF4078641CF5
:1085F0002844C5B2E4B2B442F5D1284626E72DE9B5
:10860000F041054681484FF00008427A9600FF2E5F
:1086100001D94FF013082868C01C20F003022A601B
:1086200051EA080121D17948F3B20521203009F03F
:108630007FF9002408E0052C0FD2DFE804F00503E1
:1086400007070900724804E0724802E0724800E03F
:10865000724809F08DF9074600E0FFDFA74200D01D
:10866000FFDF641CE4B2052CE5D3286800EB06109C
:108670002860404672E5021D5143452900D245213C
:108680000844C01CB0FBF2F0C0B270472DE9FC5F9B
:1086900006465E484FF000088B464746444690F831
:1086A000019022E02046FFF78DFF050000D1FFDF9B
:1086B000687869463844C7B22846FFF715F88246FD
:1086C00001A92846FFF724F80346BDF804005246E6
:1086D000001D81B2BDF80000001D80B205F05EFDF6
:1086E0006A78641C00FB0288E4B24C45DAD1306839
:1086F000C01C20F003003060BBF1000F00D0002050
:108700004246394605F058FD316808443060BDE8FE
:10871000FC9F3E49343108710020C87070473B49C6
:108720003431CA782AB10A7801EB4211083181420A
:1087300001D001207047002070472DE9F041064626
:108740000078154600F00F0400201080601E0F46D0
:10875000052800D3FFDF2B482A46183800EB840099
:10876000394650F8043C3046BDE8F041184738B56A
:108770000446407800F00300012803D002280BD003
:10878000072038BD606858B1F8F7D0FDD0B96068EF
:10879000F8F7C3FD20B915E06068F8F77AFD88B9ED
:1087A00069462046FBF778FA0028EAD1607800F0A5
:1087B0000300022808D19DF8000028B16068F8F78E
:1087C000ACFD08B1102038BD6189F8290DD8208989
:1087D00088420AD8607800F003020C48012A06D1CA
:1087E000D731C26989B28A4201D2092038BD94E8E2
:1087F0000E0000F10C0585E80E000AB90021818207
:10880000002038BD2C8901001800002078020020CB
:10881000011F0000B3B50000AD900000DFF80000BC
:1088200070B50B2000F0B9F9082000F0B6F900216E
:108830000B2000F0D0F90021082000F0CCF9EE4C1C
:1088400001256560A5600020C4F84001C4F844011A
:10885000C4F848010B2000F0B1F9082000F0AEF98F
:108860000B2000F08DF9256070BD10B50B2000F0D5
:1088700094F9082000F091F9DF48012141608160FE
:10888000DE490A68002AFCD10021C0F84011C0F876
:108890004411C0F848110B2000F090F9BDE81040D9
:1088A000082000F08BB910B50B2000F087F9BDE867
:1088B0001040082000F082B900B530B1012806D080
:1088C000022806D0FFDF002000BDCD4800BDCD4806
:1088D00000BDCC48001D00BD70B5CB494FF0004035
:1088E0000860CA4DC00BC5F80803C94800240460DD
:1088F000C5F840410820C43500F04FF9C5F83C41A7
:10890000C448047070BD08B5BB4A002128B10128D5
:1089100011D002281CD0FFDF08BD4FF48030C2F810
:108920000803C2F84803B5483C300160C2F8401162
:10893000BDE80840D0E74FF40030C2F80803C2F8A1
:108940004803AE4840300160C2F84411AD480CE025
:108950004FF48020C2F80803C2F84803A748443007
:108960000160C2F84811A748001D0068009008BDCA
:1089700070B516460D460446022800D9FFDF0022D6
:108980009D48012304F110018B4000EB8401C1F8E4
:10899000405526B1C1F84021C0F8043303E0C0F8C7
:1089A0000833C1F84021C0F8443370BD2DE9F041CF
:1089B0001D46144630B1012833D0022838D0FFDFDD
:1089C000BDE8F081891E002221F07F411046FFF7AB
:1089D000CFFF012D23D000208E4D8C4F01266870D3
:1089E0003E618B4900203C3908600220091D086067
:1089F000874904203039086085483D3404600820E8
:108A00006C6000F0DBF83004C7F80403082000F0C5
:108A1000B7F87D49F007091F08602E70D0E70120E4
:108A2000DAE7012B02D00022012005E00122FBE75A
:108A3000012B04D000220220BDE8F04198E701227A
:108A4000F9E76E480068704770B56B4CD4F8400188
:108A50000025012809D1D4F80803C00305D54FF437
:108A60008030C4F80803C4F84051D4F84401012808
:108A70000CD1D4F80803800308D54FF40030C4F8B3
:108A80000803C4F84451012008F08CF8D4F84801D8
:108A900001280ED1D4F8080340030AD54FF48020F2
:108AA000C4F80803C4F84851BDE87040022008F03B
:108AB00079B870BD10B5574C207850B1FFF70CFF56
:108AC0006078002807D000206070BDE8104008F0F2
:108AD00069B80320F9E710BD4FF0E0214FF4001012
:108AE000C1F800027047152000F068B8474901201E
:108AF0000861082000F062B844494FF47C10C1F8C6
:108B0000080300204FEA000201EB8003C3F8402570
:108B1000C3F84021401CC0B20628F5D37047410A73
:108B200043F609525143C0F3080010FB02F000F570
:108B3000807001EB5020704710B5430B48F237644A
:108B400063431B0C5C020C60334C03FB0400334B8F
:108B50004CF2F72443435B0D13FB04F404EB402079
:108B600000F580704012107008681844086010BD4D
:108B700028484068704725490120C1F80002704725
:108B8000002809DB00F01F0201219140400980000C
:108B900000F1E020C0F80011704700280DDB00F064
:108BA0001F02012191404009800000F1E020C0F83F
:108BB0008011BFF34F8FBFF36F8F7047002809DB21
:108BC00000F01F02012191404009800000F1E020E7
:108BD000C0F8801270474907090E002804DB00F135
:108BE000E02080F80014704700F00F0000F1E02052
:108BF00080F8141D7047000000B0004004B500402C
:108C00004081004044B1004008F501400080004030
:108C1000408500402C000020F7C2FFFF6F0C0100D0
:108C200010B5EFF3108000F0010472B6FE484178F1
:108C3000491C41704078012801D108F093FB002CB9
:108C400000D162B610BD70B5F74CA07848B90125C7
:108C5000A570FFF7E5FF08F096FB20B1002008F0B3
:108C600060FB002070BD4FF08040E570C0F80453F9
:108C7000F7E770B5EFF3108000F0010572B6EA4C2B
:108C8000607800B9FFDF6078401E6070607808B9D6
:108C900008F06CFB002D00D162B670BDE24810B543
:108CA000817821B10021C1708170FFF7E2FF0020BF
:108CB00010BD10B5044608F066FBDB498978084012
:108CC00000D001202060002010BD10B5FFF7A8FFE4
:108CD00008F059FB02220123D349540728B1D34895
:108CE000026023610320087202E00A72C4F80433B0
:108CF0000020887110BD2DE9F84FDFF82C934278E1
:108D0000817889F80420002689F80510074689F83B
:108D100006600078DFF818B3354620B1012811D07D
:108D2000022811D0FFDF08F040FB4FF0804498B1DB
:108D300008F042FBB0420FD1304608F041FB00285A
:108D4000FAD041E00126EEE7FFF76AFF58460168D6
:108D5000C907FCD00226E6E70120E060C4F8045110
:108D6000B4490E600107D1F84412B24AC1F342314E
:108D700024321160AF49343108604FF0020AC4F860
:108D800004A3A060AC480168C94341F3001101F19C
:108D90000108016841F01001016000E020BFD4F833
:108DA00004010028FAD0304608F00AFB0028FAD067
:108DB000B8F1000F04D1A048016821F01001016052
:108DC000C4F808A3C4F8045199F805004E4680B1D0
:108DD000387870B908F0D7FA804608F06BFC6FF06D
:108DE0000042B8F1000F02D0C6E9032001E0C6E955
:108DF0000302DBF80000C00701D008F0C0FA3878A1
:108E000010B13572BDE8F88F4FF01808C4F8088328
:108E10000127A7614FF4A070ADF80000BDF8000075
:108E2000411EADF80010F9D2C4F80C51C4F810512D
:108E30007D48C01D08F0D6FA3570FFF746FF676120
:108E40007C49307920310860C4F80483DAE770B5D2
:108E5000050000D1FFDF4FF080424FF0FF30C2F835
:108E600008030021C2F80011C2F80411C2F80C1165
:108E7000C2F810116C4C617008F091FA10B1012029
:108E8000A07060706A480068C00701D008F077FAE7
:108E90002846BDE870402EE76348007A002800D0DD
:108EA000012070472DE9F84F4FF08044D4F80801B5
:108EB00000B10120D4F8001111B14FF0010801E018
:108EC0004FF00008D4F8041101B101218B46D4F809
:108ED0000C1101B101218A46D4F8101101B1012110
:108EE000514D894629780026009120B1C4F80861C7
:108EF000012008F016FA4C48C01D08F07BFA00B1BA
:108F0000FFDF0127B8F1000F10D0C4F80873E8782C
:108F100018B1EE70002008F004FA287A022805D172
:108F2000032028724148022101602761BBF1000F34
:108F300001D0C4F80461BAF1000F0AD0C4F80C6182
:108F4000287A032800D0FFDF384806602F72FFF729
:108F500090FEB9F1000F07D0C4F81061287A0128FB
:108F600001D100F049F86761009838B12E70287A75
:108F7000012801D1FFF7A9FEFFF77BFEBDE8F84FFE
:108F80002948C01D08F04CBA274810B5C01D08F08C
:108F900031FA254940B1012008704FF0E021C1F8B5
:108FA0000002BDE810403BE6087A012801D1FFF736
:108FB0008CFE1D48BDE81040C01D08F031BA70B5E8
:108FC000194CA07808B908F0D1F901208507A861EB
:108FD000207A0026032809D1D5F80C0120B90020F9
:108FE00008F0EEF90028F7D1C5F80C6126724FF0B1
:108FF000FF30C5F8080370BD70B50B4C607930B315
:10900000012803D0A179401E814222DA08F0BBF981
:10901000054608F04FFB6179012902D9A179491C65
:10902000A1715DB121690AE034000020340C0040D8
:109030000C0400401805004010ED00E0E168411A02
:10904000022902DA11F1020F06DC0DB1206100E005
:10905000E060BDE8704038E670BD00000F4A12685D
:109060000D498A420CD118470C4A12680A4B9A42A1
:1090700006D101B508F0F0FAF9F72AFFBDE8014082
:10908000074909680958084706480749054A064B31
:109090007047000000000000BEBAFECA4C0000206D
:1090A00004000020D80C0020D80C002070B50C461D
:1090B000054600F045FB21462846BDE8704001F01A
:1090C0002ABC0000F8B51D46DDE906470E000AD0AF
:1090D00005F02AF92346FF1DBCB231462A4600940A
:1090E00004F055FDF8BDD019224619460FF0A4F939
:1090F0002046F8BD70B50D46044610210FF01BFA4E
:10910000258117206081A07B40F00A00A07370BD0C
:109110004FF6FF720A800146022008F0E3BC704758
:1091200000897047827BD30701D1920703D48089DD
:1091300008800020704705207047827B920700D589
:109140008181704701460020098841F6FE52114294
:1091500000D00120704700B50346807BC00701D0D6
:10916000052000BD59811846FFF7ECFFC00703D06A
:10917000987B40F004009873987B40F0010098734E
:10918000002000BD827B520700D509B1408970479D
:1091900017207047827B61F3C302827370472DE909
:1091A000FC5F0E46044601789646012000FA01F164
:1091B0004DF6FF5201EA020962684FF6FF7B118803
:1091C000594502D10920BDE8FC9FB9F1000F05D037
:1091D00041F6FE55294201D00120F4E741EA090198
:1091E00011801D0014D000232B7094F800C00521BD
:1091F00003221F464FF0020ABCF10E0F76D2DFE8C1
:109200000CF0F909252F47646B77479193B4D1D8B7
:109210000420D8E7616820898B7B9B0767D51728D6
:109220004AD30B89834247D38989172901D38142C5
:1092300042D185F800A0A5F80100328061688881DC
:109240006068817B21F002018173C6E004202870F0
:109250002089A5F801006089A5F803003180BCE0F1
:10926000208A3188C01D1FFA80F8414524D306208A
:1092700028702089A5F801006089A5F80300A0895D
:10928000A5F805000721208ACDE90001636941E0C6
:109290000CF0FF00082810D0082028702089A5F8BD
:1092A00001006089A5F8030031806A1D694604F158
:1092B0000C0006F0A1FC10B15EE01020EDE7308854
:1092C0009DF800100844308087E00A20287020892B
:1092D000A5F80100328044E00C2028702089A5F810
:1092E00001006089A5F8030031803AE082E064E083
:1092F0002189338800EB41021FFA82F843453BD3B2
:10930000B8F1050F38D30E222A700BEA4101CDE9DE
:109310000010E36860882A467146FFF7D3FEA6F87E
:1093200000805AE04020287060893188C01C1FFAF4
:1093300080F8414520D32878714620F03F00123054
:1093400028702089A5F801006089CDE900026088B5
:109350002A46E368FFF7B6FEA6F8008028784006A4
:109360003BD461682089888037E0A0893288401D1D
:109370001FFA80F8424501D204273DE016202870EC
:109380002089A5F801006089A5F80300A089CDE92E
:10939000000160882A4671462369FFF793FEA6F80C
:1093A0000080DEE718202870207A6870A6F800A0F8
:1093B00013E061680A88920401D405271CE0C9887B
:1093C0002289914201D0062716E01E2129703080A3
:1093D0006068018821F400510180B9F1000F0BD0C1
:1093E000618878230022022008F0D2FA6168207890
:1093F000887006E0338003276068018821EA09014C
:1094000001803846DFE62DE9FF4F85B01746129CF4
:109410000D001E461CD03078C10703D000F03F007D
:10942000192801D9012100E000212046FFF7AAFEFA
:10943000A8420DD32088A0F57F41FF3908D03078AD
:10944000410601D4000605D5082009B0BDE8F08F1B
:109450000720FAE700208DF800008DF80100307831
:109460006B1E00F03F0C0121A81E4FF0050A4FF0C3
:1094700002094FF0030B9AB2BCF1200F75D2DFE85E
:109480000CF08B10745E7468748C749C74B674BB2E
:1094900074C974D574E2747474F274F074EF74EE79
:1094A000748B052D78D18DF80090A0788DF804008C
:1094B0007088ADF8060030798DF80100707800F002
:1094C0003F000C2829D00ADCA0F10200092863D251
:1094D000DFE800F0126215621A621D622000122895
:1094E00024D004DC0E281BD01028DBD11BE016286A
:1094F0001FD01828D6D11FE02078800701E02078FF
:109500004007002848DAEFE020780007F9E72078E4
:10951000C006F6E720788006F3E720784006F0E7FB
:1095200020780006EDE72088C005EAE7208840059E
:10953000E7E720880005E4E72088C004E1E7207819
:10954000800729D5032D27D18DF800B0B6F801008A
:1095500082E0217849071FD5062D1DD381B270788E
:10956000012803D0022817D102E0CAE0022000E05F
:10957000102004228DF8002072788DF80420801CC1
:10958000B1FBF0F2ADF8062092B242438A4203D119
:109590000397ADF80890A7E07AE02078000777D528
:1095A00098B282088DF800A0ADF80420B0EB820FCD
:1095B0006ED10297ADF8061096E02178C90667D5FE
:1095C000022D65D381B206208DF800007078022844
:1095D0005ED300BFB1FBF0F28DF80400ADF80620B9
:1095E00092B242438A4253D1ADF808907BE0207892
:1095F00080064DD5072003E0207840067FD508205F
:109600008DF80000A088ADF80400ADF80620ADF894
:10961000081068E02078000671D50920ADF8042014
:109620008DF80000ADF8061002975DE02188C905AD
:1096300065D5022D63D381B20A208DF800007078C1
:1096400004285CD3C6E72088400558D5012D56D1A3
:109650000B208DF80000A088ADF8040044E021E064
:1096600026E016E0FFE72088000548D5052D46D303
:109670000C208DF80000A088ADF80400B6F80300B7
:109680006D1FADF80850ADF80600ADF80AA02AE04D
:1096900035E02088C00432D5012D30D10D208DF861
:1096A000000021E02088800429D4B6F80100E08081
:1096B000A07B000723D5032D21D3307800F03F0095
:1096C0001B2818D00F208DF80000208840F400508F
:1096D000A4F80000B6F80100ADF80400ED1EADF8E6
:1096E0000650ADF808B0039769460598FBF7B4FA41
:1096F000050008D016E00E208DF80000EAE70725E7
:1097000010E008250EE0307800F03F001B2809D05B
:109710001D2807D00220059908F0E4F9208800F4FC
:1097200000502080A07B400708D52046FFF70AFDA7
:10973000C00703D1A07B20F00400A073284684E674
:109740001FB5022806D101208DF8000088B26946B5
:10975000FBF782FA1FBD0000F8B51D46DDE906479C
:109760000E000AD004F0E0FD2346FF1DBCB23146D6
:109770002A46009404F00BFAF8BDD0192246194687
:109780000EF05AFE2046F8BD2DE9FF4F8DB09B46E6
:10979000DDE91B57DDF87CA00C46082B05D0E069FD
:1097A00001F002F950B11020D2E02888092140F0E0
:1097B000100028808AF80010022617E0E1690120D5
:1097C0008871E2694FF420519180E1698872E06903
:1097D00042F601010181E06900218173288811218D
:1097E00040F0200028808AF80010042638780A907B
:1097F0000A2038704FF0020904F118004D460C9011
:1098000001F095FBB04681E0BBF1100F0ED1022DA7
:109810000CD0A9EB0800801C80B20221CDE9001019
:1098200005AB52461E990D98FFF796FFBDF816102E
:109830001A98814203D9F74800790F9004E003D1C8
:109840000A9808B138702FE04FF00201CDE90019F5
:109850000DF1160352461E990D98FFF77DFF1D98D6
:109860000088401B801B83B2C6F1FF00984200D2E3
:1098700003461E990BA8D9B15FF00002DDF878C04D
:10988000CDE9032009EB060189B2CDE901C10F98AA
:109890000090BDF8161000220D9801F0CBFB387037
:1098A00070B1C0B2832807D0BDF8160020833AE01B
:1098B0000AEB09018A19E1E7022011B0BDE8F08F37
:1098C000BDF82C00811901F0FF08022D0DD09AF887
:1098D0000120424506D1BDF82010814207D0B8F1E1
:1098E000FF0F04D09AF801801FE08AF80180C94870
:1098F00000680178052902D1BDF81610818009EBB6
:1099000008001FFA80F905EB080085B2DDE90C10AC
:1099100005AB0F9A01F00EFB28B91D980088411B7A
:109920004145BFF671AF022D13D0BBF1100F0CD122
:10993000A9EB0800801C81B20220CDE9000105AB33
:1099400052461E990D98FFF707FF1D9805800020CD
:1099500038700020B1E72DE9F8439C46089E134675
:109960000027B26B9AB3491F8CB2F18FA1F57F45E6
:10997000FF3D05D05518AD882944891D8DB200E002
:1099800000252919B6F83C800831414520D82A44E1
:10999000BCF8011022F8021BBCF8031022F8021BCD
:1099A000984622F8024B914604F0ACFC4FF00C0CA8
:1099B00041464A462346CDF800C004F0B4F8F58786
:1099C000B16B00202944A41D2144088003E001E07C
:1099D000092700E083273846BDE8F88310B50B88D7
:1099E000848F9C420CD9846BE018048844B184882D
:1099F00024F40044A41D23440B801060002010BDFB
:109A00000A2010BD2DE9F0478AB00025904689460E
:109A10008246ADF8185007274BE0059806888088E5
:109A2000000446D4A8F8006007A8019500970295A5
:109A3000CDE903504FF4007300223146504601F047
:109A4000F9FA04003CD1BDF81800ADF820000598E3
:109A500004888188B44216D10A0414D40195029571
:109A6000039521F400410097049541F48043428816
:109A70002146504601F0B4F804000BD105988188C6
:109A800041F40041818005AA08A94846FFF7A6FFD6
:109A90000400DCD000970598029501950395049584
:109AA0000188BDF81C300022504601F099F80A2CBC
:109AB00006D105AA06A94846FFF790FF0400ACD0DE
:109AC000ADF8185004E00598818821F400418180A8
:109AD00005AA06A94846FFF781FF0028F3D00A2C03
:109AE00003D020460AB0BDE8F0870020FAE710B5A1
:109AF0000C46896B86B051B10C218DF80010A18FF6
:109B0000ADF80810A16B01916946FCF754F80020EC
:109B10004FF6FF71A063E187A08706B010BD2DE965
:109B2000F0410D460746896B0020069E1446002929
:109B300011D0012B0FD1324629463846FFF762FF7C
:109B4000002808D1002C06D0324629463846BDE808
:109B5000F04100F038BFBDE8F0812DE9FC4114462A
:109B6000DDE9087C0E46DDE90A15521DBCF800E06F
:109B700092B2964502D20720BDE8FC81ACF80020E5
:109B800017222A70A5F80160A5F803300522CDE957
:109B900000423B462A46FFF7DFFD0020ECE770B5A8
:109BA0000C461546482120460EF0E7FC04F108005B
:109BB00044F81C0F00204FF6FF71E061618420849F
:109BC000A5841720E08494F82A0040F00A0084F865
:109BD0002A0070BD4FF6FF720A800146032007F08D
:109BE00081BF30B585B00C460546FFF780FFA18EDA
:109BF000284629B101218DF800106946FBF7DBFFEB
:109C00000020E0622063606305B030BDB0F8400022
:109C1000704700005000002090F84620920703D4BF
:109C2000408808800020F3E70620F1E790F84620FE
:109C30009207EDD5A0F84410EAE701460020098814
:109C40000A0700D5012011F0F00F01D040F002000A
:109C5000CA0501D540F004008A0501D540F008008E
:109C60004A0501D540F010000905D1D540F020008B
:109C7000CEE700B5034690F84600C00701D00620A5
:109C800000BDA3F842101846FFF7D7FF10F03E0FB3
:109C900005D093F8460040F0040083F8460013F81E
:109CA000460F40F001001870002000BD90F84620DB
:109CB000520700D511B1B0F84200A9E71720A7E775
:109CC00010F8462F61F3C3020270A1E72DE9FF4FA0
:109CD0009BB00E00DDE92B34DDE92978289D24D0E6
:109CE0002878C10703D000F03F00192801D90121CD
:109CF00000E000212046FFF7D9FFB04215D32878B5
:109D0000410600F03F010CD41E290CD0218811F42B
:109D10007F6F0AD13A8842B1A1F57F42FF3A04D061
:109D200001E0122901D1000602D504201FB0C5E5CB
:109D3000F9491D984FF0000A08718DF818A08DF8A8
:109D40003CA00FAA0A60ADF81CA0ADF850A029787D
:109D5000994601F03F02701F5B1C04F1180C4FF094
:109D6000060E4FF0040BCDF858C01F2A7ED2DFE854
:109D700002F07D7D107D267DAC7DF47DF37DF27D4E
:109D8000F17DF47DF07D7D7DEF7DEE7D7D7D7D7DC2
:109D9000ED0094F84610B5F80100890701D5032EAF
:109DA00002D08DF818B022E34FF40061ADF85010E6
:109DB000608003218DF83C10ADF84000D8E2052EFC
:109DC000EFD1B5F801002083ADF81C00B5F8031001
:109DD000618308B1884201D901207FE10020A0728F
:109DE00020814FF6FF702084169801F0A0F805201E
:109DF00089F800000220029083460AAB1D9A16994A
:109E00001B9801F097F890BB9DF82E00012804D014
:109E1000022089F80100102003E0012089F80100E8
:109E200002200590002203A90BA805F0E5FEE8BB7F
:109E30009DF80C00059981423DD13A88801CA2EB27
:109E40000B01814237DB02990220CDE900010DF1BF
:109E50002A034A4641461B98FFF77EFC02980BF105
:109E6000020B801C80B217AA03A901E0A0E228E03F
:109E700002900BA805F0C0FE02999DF80C00CDE9F8
:109E8000000117AB4A4641461B98FFF765FC9DF859
:109E90000C100AAB0BEB01001FFA80FB02981D9A15
:109EA000084480B2029016991B9800E003E001F08C
:109EB00041F80028B6D0BBF1020F02D0A7F800B0DD
:109EC00053E20A208DF818004FE200210391072E7B
:109ED000FFF467AFB5F801002083ADF81C00B5F8BA
:109EE0000320628300283FF477AF90423FF674AFBF
:109EF0000120A072B5F8050020810020A073E06960
:109F000000F052FD78B9E16901208871E2694FF4EF
:109F100020519180E1698872E06942F60101018176
:109F2000E06900218173F01F20841E986062072081
:109F30006084169800F0FBFF072089F800000120DC
:109F4000049002900020ADF82A0028E01DE2A3E171
:109F50003AE1EAE016E2AEE086E049E00298012844
:109F600014D0E0698079012803D1BDF82800ADF84C
:109F70000E00049803ABCDE900B04A4641461B9859
:109F8000FFF7EAFB0498001D80B20490BDF82A0098
:109F9000ADF80C00ADF80E00059880B202900AAB47
:109FA0001D9A16991B9800F0C5FF28B902983988A8
:109FB000001D05908142D1D20298012881D0E0692C
:109FC0008079012805D0BDF82810A1F57F40FF3821
:109FD00003D1BDF82800ADF80E00049803ABCDE91D
:109FE00000B04A4641461B98FFF7B6FB0298BBE11A
:109FF000072E02D0152E7FF4D4AEB5F801102183C0
:10A00000ADF81C10B5F80320628300293FF4E4AEDC
:10A0100091423FF6E1AE0121A1724FF0000BA4F88E
:10A0200008B084F80EB0052E07D0C0B2691DE269F1
:10A0300005F0C3FD00287FF444AF4FF6FF70208485
:10A0400001A906AA14A8CDF800B081E885032878F4
:10A05000214600F03F031D9A1B98FFF795FB8246AF
:10A06000208BADF81C0080E10120032EC3D14021DC
:10A07000ADF85010B5F801102183ADF81C100AAAF4
:10A08000B8F1000F00D00023CDE9020304921D981F
:10A09000CDF80480009038880022401E83B21B98BF
:10A0A00000F0C8FF8DF8180090BB0B2089F8000065
:10A0B000BDF8280037E04FF0010C052E9BD1802021
:10A0C000ADF85000B5F801102183B5F803002084E5
:10A0D000ADF81C10B0F5007F03D907208DF81800EB
:10A0E00085E140F47C4222840CA8B8F1000F00D036
:10A0F0000023CDE90330CDE9018C1D98009038880C
:10A10000401E83B21B9800F095FF8DF8180028B10F
:10A110008328A8D10220BDE0500000200D2189F83D
:10A120000010BDF83000401C1EE1032E04D248068A
:10A130007FF537AE002017E1B5F80110ADF81C101F
:10A140002878400602D58DF83CE002E007208DF823
:10A150003C004FF000080320CDE902081E9BCDF81B
:10A1600010801D980193A6F1030B00901FFA8BF34A
:10A1700042461B9800F034FD8DF818008DF83C80A5
:10A18000297849060DD52088C00506D5208BBDF855
:10A190001C10884201D1C4F8248040468DF81880F4
:10A1A000E2E0832801D14FF0020A4FF48070ADF84D
:10A1B0005000BDF81C002083A4F820B01E986062F7
:10A1C000032060841321CCE0052EFFF4EAADB5F83E
:10A1D0000110ADF81C10A28F62B3A2F57F43FE3BC5
:10A1E00028D008228DF83C204FF0000B0523CDE944
:10A1F000023BDDF878C0CDF810B01D9A80B2CDF8E2
:10A2000004C040F400430092B5F803201B9800F00E
:10A21000E7FC8DF83CB04FF400718DF81800ADF8F4
:10A220005010832810D0F8B1A18FA1F57F40FE38DF
:10A2300007D0DCE00B228DF83C204FF6FE72A2879F
:10A24000D2E7A4F83CB0D2E000942B4631461E9AE7
:10A250001B98FFF780FB8DF8180008B183284BD1BD
:10A26000BDF81C00208355E700942B4631461E9A0A
:10A270001B98FFF770FB8DF81800E8BBE18FA06B0F
:10A280000844811D8DE882034388828801881B98D9
:10A29000FFF763FC824668E095F80180022E70D1DA
:10A2A0005FEA080002D0B8F1010F6AD109208DF8E9
:10A2B0003C0007A800908DF84080434600222146CC
:10A2C0001B98FFF72CFC8DF842004FF0000B8DF827
:10A2D00043B050B9B8F1010F12D0B8F1000F04D15A
:10A2E000A18FA1F57F40FF380AD0A08F40B18DF833
:10A2F0003CB04FF4806000E037E0ADF850000DE076
:10A300000FA91B98FBF757FC82468DF83CB04FF421
:10A310008060ADF85000BAF1020F06D0FC4800682A
:10A32000C07928B18DF8180027E0A4F8188044E01F
:10A33000BAF1000F03D081208DF818003DE007A886
:10A3400000904346012221461B98FFF7E8FB8DF859
:10A35000180021461B98FFF7CAFB9DF8180020B98A
:10A36000192189F80010012038809DF83C0020B1A7
:10A370000FA91B98FBF71FFC8246BAF1000F33D0E0
:10A380001BE018E08DF818E031E02078000712D5C6
:10A39000012E10D10A208DF83C00E088ADF8400075
:10A3A00003201B9907F09EFB0820ADF85000C1E682
:10A3B00048067FF5F6AC4FF0040A2088BDF850102F
:10A3C00008432080BDF8500080050BD5A18FA1F572
:10A3D0007F40FE3806D11E98E06228982063A6864A
:10A3E0004FF0030A5046A1E49DF8180078B101200F
:10A3F00089F80000297889F80110BDF81C10A9F827
:10A4000002109DF8181089F8041005203880208863
:10A41000BDF8501088432080E4E72DE9FF4F8846BF
:10A42000087895B0012181404FF20900249C014039
:10A43000ADF820102088DDF88890A0F57F424FF01D
:10A44000000AFF3A06D039B1000705D5012019B03E
:10A45000BDE8F08F0820FAE7239E4FF0000B0EA80E
:10A4600086F800B018995D460988ADF83410A849FF
:10A470008DF81CB0179A0A718DF838B0086098F8FA
:10A48000000001283BD0022809D003286FD1307882
:10A4900020F03F001D303070B8F80400E08098F8DC
:10A4A00000100320022904D1317821F03F011B3133
:10A4B000317094F84610090759D505ABB9F1000F72
:10A4C00013D0002102AA82E80B000720CDE9000981
:10A4D000BDF83400B8F80410C01E83B200221598ED
:10A4E00000F0A8FD0028D1D101E0F11CEAE7B8F89E
:10A4F0000400A6F80100BDF81400C01C04E198F89F
:10A5000005108DF81C1098F80400012806D04FF4AF
:10A51000007A02282CD00328B8D16CE12188B8F841
:10A52000080011F40061ADF8201020D017281CD3CA
:10A53000B4F84010814218D3B4F84410172901D35D
:10A54000814212D1317821F03F01C91C3170A6F847
:10A5500001000321ADF83410A4F8440094F846003B
:10A5600020F0020084F8460065E105257EE177E1F0
:10A57000208808F1080700F4FE60ADF8200010F014
:10A58000F00F1BD010F0C00F03D03888228B904200
:10A59000EBD199B9B878C00710D0B9680720CDE9D8
:10A5A00002B1CDF804B00090CDF810B0FB88BA88A5
:10A5B0003988159800F014FB0028D6D12398BDF8EF
:10A5C0002010401C80294ED006DC10290DD02029F7
:10A5D0000BD0402987D124E0B1F5807F6ED0514562
:10A5E0007ED0B1F5806F97D1DEE0C80601D5082096
:10A5F00000E0102082460DA907AA0520CDE902211E
:10A600008DF83800ADF83CB0CDE9049608A938883B
:10A61000CDE900015346072221461598FFF7B4F80B
:10A62000A8E09DF81C2001214FF00A0A002A9BD1C6
:10A6300005ABB9F1000F00D00020CDE902100720D2
:10A64000CDE90009BDF834000493401E83B2218B8C
:10A650000022159800F0EEFC8DF81C000B203070E5
:10A66000BDF8140020E09DF81C2001214FF00C0AD9
:10A67000002A22D113ABB9F1000F00D00020CDE9A0
:10A6800002100720CDE900090493BDF83400228CA4
:10A69000401E83B2218B159800F0CCFC8DF81C0075
:10A6A0000D203070BDF84C00401CADF83400052082
:10A6B0008DF83800208BADF83C00BCE03888218B49
:10A6C00088427FF452AF9DF81C004FF0120A002818
:10A6D0001CD1606AA8B1B878C0073FF446AF00E06B
:10A6E00018E0BA680720CDE902B2CDF804B00090B6
:10A6F000CDF810B0FB88BA88159800F071FA8DF883
:10A700001C00132030700120ADF8340093E00000ED
:10A71000500000203988208B8142D2D19DF81C0046
:10A720004FF0160A0028A06B08D0E0B34FF6FF7078
:10A7300000215F46ADF808B0019027E068B1B97814
:10A74000C907BED1E18F0DAB0844821D03968DE889
:10A750000C0243888288018809E0B878C007BCD021
:10A76000BA680DAB03968DE80C02BB88FA88159881
:10A77000FFF7F3F905005ED0072D72D076E0019067
:10A7800005AA02A92046FFF729F90146E28FBDF884
:10A790000800824201D00029F1D0E08FA16B08446B
:10A7A00007800198E08746E09DF81C004FF0180AEA
:10A7B00040B1208BC8B13888208321461598FFF717
:10A7C00096F938E004F118000090237E012221461A
:10A7D0001598FFF7A4F98DF81C000028EDD1192079
:10A7E00030700120ADF83400E7E7052521461598C3
:10A7F000FFF77DF93AE0208800F40070ADF8200002
:10A8000050452DD1A08FA0F57F41FE3901D00625FE
:10A810002CE0D8F808004FF0160A48B1A063B8F849
:10A820000C10A1874FF6FF71E187A0F800B002E09D
:10A830004FF6FF70A087BDF8200030F47F611AD07A
:10A84000782300220320159907F0A2F898F8000059
:10A8500020712088BDF82010084320800EE000E021
:10A8600007252088BDF8201088432080208810F418
:10A870007F6F1CD03AE02188814321809DF8380009
:10A8800020B10EA91598FBF796F905469DF81C0016
:10A890000028EBD086F801A001203070208B70805A
:10A8A0009DF81C0030710520ADF83400DEE7A18E64
:10A8B000E1B118980DAB0088ADF834002398CDE9CC
:10A8C0000304CDE90139206B0090E36A179A1598CB
:10A8D000FFF7FCF9054601208DF838000EA9159800
:10A8E000FBF769F900B10546A4F834B094F84600C6
:10A8F00040070AD52046FFF7A0F910F03E0F04D11B
:10A9000014F8460F20F0040020701898BDF8341099
:10A91000018028469BE500B585B0032806D10220BA
:10A920008DF8000088B26946FBF745F905B000BD17
:10A9300010B5384C0B782268012B02D0022B2AD19B
:10A9400011E013780BB1052B01D104231370236898
:10A950008A889A802268CB88D38022680B891381E9
:10A96000498951810DE08B8893802268CB88D38000
:10A9700022680B8913814B8953818B8993810969E3
:10A9800011612168FBF717F9226800210228117074
:10A9900003D0002800D0812010BD832010BD806B23
:10A9A000002800D0012070478178012909D1008852
:10A9B000B0F5205F03D042F60101884201D10020AA
:10A9C000704707207047F0B587B0002415460E4643
:10A9D0000746ADF8184011E00598008828800598D2
:10A9E0000194811DCDE902410721049400918388DF
:10A9F00042880188384600F0F3F830B905AA06A964
:10AA00003046FEF7EBFF0028E6D00A2800D10020F0
:10AA100007B0F0BD5000002010B58B7883B10278EC
:10AA20009A4205D10B885BB102E08B79091D4BB1CD
:10AA30008B789A42F9D1B0F801300C88A342F4D156
:10AA4000002010BD812010BD072826D012B1012A98
:10AA500027D103E0497801F0070102E04978C1F30A
:10AA6000C20105291DD2DFE801F00318080C12000D
:10AA70000AB1032070470220704704280DD250B15C
:10AA80000DE0052809D2801E022808D303E006281D
:10AA900003D0032803D005207047002070470F2003
:10AAA000704781207047C0B282060BD4000607D5DC
:10AAB000FE48807A4143C01D01EBD00080B2704750
:10AAC000084670470020704770B513880B800B78DC
:10AAD0001C0625D5F54CA47A844204D843F0100016
:10AAE0000870002070BD956800F0070605EBD005E2
:10AAF0002D78F54065F304130B701378D17803F0CB
:10AB0000030341EA032140F20123B1FBF3F503FB08
:10AB100015119268E41D00FB012000EBD40070BD0C
:10AB2000906870BD37B51446BDF8041011809DF8CB
:10AB300004100A061ED5C1F30013DC49A568897A02
:10AB4000814208D8FE2811D1C91DC9085A42284699
:10AB50000DF0E9FC0AE005EBD00100F00702012549
:10AB600008789540A843934018430870207820F057
:10AB7000100020703EBD2DE9F0410746C81C0E466E
:10AB800020F00300B04202D08620BDE8F081C74D1E
:10AB9000002034462E60AF802881AA72E8801AE037
:10ABA000E988491CE980810614D4E17800F00300AB
:10ABB00041EA002040F20121B0FBF1F201FB120159
:10ABC0002068FFF770FF2989084480B22881381A6D
:10ABD0003044A0600C3420784107E1D40020D4E751
:10ABE0002DE9FF4F89B01646DDE9168A0F469946D2
:10ABF00023F44045084600F00DFB04000FD00998EF
:10AC000003F018FA0290207800060AD5A748817A46
:10AC10000298814205D887200DB0BDE8F08F012051
:10AC2000FAE7224601A90298FFF74EFF834600206B
:10AC30008DF80C004046B8F1070F1AD001222146CA
:10AC4000FFF702FF0028E7D12078400611D5022047
:10AC50008DF80C00ADF81070BDF80400ADF81200CE
:10AC6000ADF814601898ADF81650CDF81CA0ADF8EA
:10AC700018005FEA094004D500252E46A8460127A2
:10AC80000CE02178E07801F0030140EA012040F275
:10AC90000121B0FBF1F2804601FB12875FEA4940D7
:10ACA00009D5B84507D1A178207901F0030140EA20
:10ACB0000120B04201D3BE4201D90720ACE7A81958
:10ACC0001FFA80F9B94501D90D20A5E79DF80C00C0
:10ACD00028B103A90998FAF76CFF00289CD1B84560
:10ACE00007D1A0784FEA192161F30100A07084F820
:10ACF00004901A9800B10580199850EA0A0027D0EC
:10AD0000199830B10BEB06002A4619990DF094FB07
:10AD10000EE00BEB06085746189E099803F0F2FA6E
:10AD20002B46F61DB5B239464246009502F0FBFEB1
:10AD3000224601A90298FFF7C7FE9DF804002246AB
:10AD400020F010008DF80400DDE90110FFF7EAFEA5
:10AD5000002061E72DE9FF4FDFF85091824617464A
:10AD6000B9F80610D9F8000001EB410100EB8104AD
:10AD700040F20120B2FBF0F185B000FB11764D46A8
:10AD8000DDF84C8031460698FFF78DFE29682A8948
:10AD90008B46611A0C3101441144AB8889B28B4255
:10ADA00002D8842009B038E70699CDB2290603D528
:10ADB000A90601D50620F5E7B9F806C00CF1010C8B
:10ADC0001FFA8CFCA9F806C0149909B1A1F800C0BB
:10ADD000A90602D5C4F8088007E0104480B2A9F89B
:10ADE0000800191A01EB0B00A0602246FE2006990C
:10ADF000FFF798FEE77026712078390A61F30100A9
:10AE0000320AA17840F0040062F30101A1702070C1
:10AE10009AF802006071BAF80000E08000262673FC
:10AE2000280602D599F80A7000E00127A80601D586
:10AE30004FF000084D4600244FF007090FE0CDE920
:10AE400002680196CDF800900496E9882046129B8E
:10AE5000089AFFF7C5FE0028A4D1641CE4B2BC42E6
:10AE6000EDD300209EE72DE9F047804600F0D2F9AF
:10AE7000070005D0002644460C4D40F2012919E098
:10AE80000120BDE8F087204600F0C4F90278C178BF
:10AE900002F0030241EA0222B2FBF9F309FB13219B
:10AEA0000068FFF700FE304486B201E0B8040020DD
:10AEB000641CA4B2E988601E8142E4DCA8F10100B0
:10AEC000E8802889801B288100203870D9E710B5D8
:10AED000144631B1491E218003F0ACF8A070002067
:10AEE00010BD012010BD10B5D24904460088CA88A3
:10AEF000904201D30A2010BD096800EB400001EB2D
:10AF000080025079A072D08820819178107901F068
:10AF1000030140EA0120A081A078E11CFFF7D4FDE5
:10AF200020612088401C2080E080002010BD01218D
:10AF3000018270472DE9FF4F85B04FF6FF788246BA
:10AF4000A3F8008048681F460D4680788DF80600FB
:10AF500048680088ADF8040000208DF80A00088ACF
:10AF60000C88A04200D304462C8241E0288A401C71
:10AF70002882701D6968FFF74FFDB8BB39884145CD
:10AF800001D1601E38806888A04236D3B17830790C
:10AF900001F0030140EA012901A9701DFFF73CFD02
:10AFA00020BB298941452CD0002231460798FFF764
:10AFB0004BFDD8B92989494518D1E9680391B5F8FD
:10AFC0000AC0D6F808B05046CDF800C003F09AF990
:10AFD000DDF800C05A460CF1070C1FFA8CFC4B46FA
:10AFE0000399CDF800C002F068FD50B1641CA4B212
:10AFF000204600F00FF90600B8D1641E2C820A200A
:10B00000D0E67C807079B871F088B8803178F078BB
:10B0100001F0030140EA01207881A7F80C90504626
:10B0200003F008F8324607F10801FFF74DFD3861DB
:10B030000020B7E62DE9FF4F87B081461C469246B7
:10B04000DDF860B0DDF85480089800F0E3F8050002
:10B050000CD0484602F0EEFF2978090608D575495C
:10B06000897A814204D887200BB0D6E50120FBE71E
:10B07000CAF309062A4601A9FFF726FD07461498D8
:10B0800007281CD000222946FFF7DEFC0028EBD160
:10B090002878400613D501208DF808000898ADF8EF
:10B0A0000C00BDF80400ADF80E00ADF81060ADF86E
:10B0B000124002A94846FAF77CFD0028D4D129782D
:10B0C000E87801F0030140EA0121AA78287902F02A
:10B0D000030240EA0220564507D0B1F5007F04D9AB
:10B0E000611E814201DD0B20BEE7864201D90720A7
:10B0F000BAE7801B85B2A54200D92546BBF1000FF7
:10B1000001D0ABF80050179818B1B9192A460DF0C4
:10B1100093F9B8F1000F0DD03E4448464446169FBF
:10B1200003F002F92146FF1DBCB232462B460094C3
:10B1300002F02DFD002097E72DE9F04107461D465E
:10B140001646084600F066F804000BD0384602F0B8
:10B1500071FF2178090607D53649897A814203D8DB
:10B16000872012E5012010E522463146FFF7ACFCAE
:10B1700065B12178E07801F0030140EA0120B0F5E3
:10B18000007F01D8012000E0002028700020FCE4AE
:10B190002DE9F04107461D461646084600F03AF8EC
:10B1A00004000BD0384602F045FF2178090607D588
:10B1B0002049897A814203D88720E6E40120E4E42B
:10B1C00022463146FFF7AEFCFF2D14D02178E078FF
:10B1D00001F0030240EA022040F20122B0FBF2F348
:10B1E00002FB130015B900F2012080B2E070000AE2
:10B1F00060F3010121700020C7E410B50C4600F097
:10B2000009F828B1C18821804079A070002010BDC4
:10B21000012010BD0749CA88824209D340B109689C
:10B2200000EB40006FF00B0202EB80000844704717
:10B2300000207047B804002010B506F0EDFDF7F7C8
:10B2400073FD06F09BFCBDE8104006F02DBD2028E4
:10B2500001D2012070470020704701224FF0A04327
:10B26000824011B1C3F80C257047C3F80825704718
:10B270004FF0A04101228240C1F81825704770B5F7
:10B280000346002002466FF02F050EE09C5CA4F1FF
:10B2900030060A2E02D34FF0FF3070BD00EB800065
:10B2A00005EB4000521C2044D2B28A42EED370BD5E
:10B2B00030B50A230BE0B0FBF3F403FB1404B0FB3E
:10B2C000F3F08D183034521E05F8014CD2B2002A2A
:10B2D000F1D130BD30B500234FF6FF7510E0040A00
:10B2E00044EA002084B2C85C6040C0F303146040AC
:10B2F00005EA00344440E0B25B1C84EA40109BB293
:10B300009342ECD330BD000070B514460B88012287
:10B31000A240134207D113430B8001230922011DD0
:10B3200002F063FD047070BD2DE9FF4F81B0087815
:10B33000DDE90E7B9A4691460E4640072CD40198D3
:10B3400002F0F2FF040000D1FFDF07F104082046FD
:10B350001FFA88F102F04FF9050000D1FFDF204607
:10B3600029466A4602F099FB0098A0F80370A0F8FD
:10B3700005A0284602F03FFC017869F306016BF353
:10B38000C711017020461FFA88F102F077F900B961
:10B39000FFDF019801F0B0FA06EB0900017E491CBD
:10B3A000017605B0BDE8F08F2DE9F84F0E469A46BC
:10B3B00091460746032102F073FE0446808CDFF8B5
:10B3C0009085002518B198F80000B0421ED138468B
:10B3D00002F0AAFF070000D1FFDF09F1040138469F
:10B3E00089B202F008F9050010D0384629466A46AD
:10B3F00002F053FB009800210A460180817001F0A1
:10B40000E7FA0098C01DCAF8000021E098F8000093
:10B41000B04216D104F1220734F8301F012000FA9F
:10B4200006F911EA090F00D0FFDF2088012340EA66
:10B43000090020800922391D384602F0F1FC06700F
:10B4400006E0324604F1300104F12200FFF75CFF10
:10B45000092188F800102846BDE8F88FFEB515468A
:10B460000C46064602AB0C220621FFF79DFF002882
:10B4700027D00299607812220A70801C4870082236
:10B480004A80A07002982988052381806988C1803C
:10B49000A9880181E988418100250C20CDE90005BA
:10B4A000062221463046FFF73FFF2946002266F379
:10B4B0001F41F023104606F06BFA6078801C607024
:10B4C0000120FEBD10B50446032102F0E9FD01464E
:10B4D00000F110022046BDE81040BFE72DE9FE4311
:10B4E000814650781646884640B1FFDF3168C8F87B
:10B4F00004107168C8F80810BDE8FE83B77802240C
:10B5000017B1022F13D0FFDF251D2A4602AB0721FA
:10B510004846FFF749FF0028E8D002980121022F92
:10B520000170317841704480878002D005E00624A4
:10B53000EAE7B188C180F18801810024CDE9005497
:10B540000523072241464846FFF7EEFE88F80440EF
:10B55000D2E710B50446032102F0A2FD0146021D08
:10B560002046BDE81040B9E7F94A002009211170D2
:10B57000704770B50C461546342120460CF0FDFF8F
:10B5800001206070092104F118000CF0F6FF05B9E4
:10B59000FFDF2978207861F30100207070BD7047CB
:10B5A000002110B560F31F41002006F09BFA002037
:10B5B00010BDFEB506460F0CFCF784FC050007D055
:10B5C0006F800321384602F06BFD040008D106E0CD
:10B5D00003B03846BDE8F0401321F7F77FB8FFDF2E
:10B5E0000EB1FFDFFEBD20782A4620F00800207053
:10B5F00002208DF800004FF6FF70ADF80200ADF8A4
:10B60000040069463846F6F7A4FCFEBD00B5FFDF2E
:10B61000002000BD2DE9FC410C461E461746804621
:10B62000032102F03DFD0546092C0AD2DFE804F0B3
:10B6300005050505050509090700042303E00623A0
:10B6400001E0FFDF0023CDE900762246294640468F
:10B65000FFF76AFEBDE8FC8138B50546A0F57F40DE
:10B66000FF381CD0284602F04DFE040000D1FFDF59
:10B67000204602F0F0F9002810D001466A46204624
:10B6800002F00BFA00980321B0F80540284602F0BA
:10B6900007FD052C03D1007908B1002038BD012039
:10B6A00038BD2DE9F041054686B0408802F02AFEFB
:10B6B000040000D1FFDF03AA2046696800F037F9D3
:10B6C000039C001F80B234F8031F218061886180D1
:10B6D000228882420AD104290BD0052918D00629D4
:10B6E00004D16888211D6B68F7F7E2FF06B0BDE85A
:10B6F000F0811646241D2A4621463046F9F761FDA1
:10B700000828F3D12A4621463046FAF7BCFDEDE77A
:10B7100016466888032102F0C3FC00218DF8001052
:10B72000042EE3D36279002AE0D0237902274FF672
:10B73000FF78012B28D0122B01D0132B0BD00491B2
:10B74000059161798DF810106B88014604AA18469E
:10B75000FFF7C4FECAE783789342C7D10278130784
:10B76000C4D5062EC2D122F008020270688860F3A8
:10B770001F41002006F0B6F98DF80070ADF8028088
:10B780002089ADF8040017E0062EAFD383789342EA
:10B79000ACD102781307A9D522F00802027068889C
:10B7A00060F31F41002006F09DF98DF8007020899C
:10B7B000ADF80200ADF8048068882A466946F6F7BD
:10B7C000C8FB93E770B50D460646032102F068FCFE
:10B7D000040004D02078000704D5112070BD43F286
:10B7E000020070BD2A4621463046FFF737FE18B9E1
:10B7F0002868206168686061207840F00800207047
:10B80000002070BD2DE9F04F0E4691B08046032117
:10B8100002F046FC0446404602F086FD0746002042
:10B82000079008900990ADF830000A9002900390BC
:10B83000049004B9FFDF0DF10809FFB9FFDF1DE037
:10B8400038460BA9002201F0C9FF9DF82C0000F03A
:10B850007F05092D00D3FFDF6019017E491E0176A7
:10B860009DF82C00000609D52A460CA907A8FFF769
:10B870004BFD19F80510491C09F80510761EF6B2A3
:10B88000DED204F13000324D04F1220BDFF8C4A007
:10B8900004F12607069010E05846069900F049F892
:10B8A00006462870092800D3FFDF5AF826104046C4
:10B8B0008847608CC05DB04202D0A08C0028EBD1DC
:10B8C00009202870234D4E4624350EE00CA907A808
:10B8D00000F02FF80446375D55F8240000B9FFDF6B
:10B8E00055F82420394640469047BDF81E000028F0
:10B8F000ECD111B056E510B5032102F0D1FB0400E4
:10B9000000D1FFDF092104F118000CF036FE207889
:10B9100040F00400207010BD10B50C46032102F069
:10B92000BFFB2044007E002800D0012010BD02F0A3
:10B93000B4B810B50C4601230922011D02F08BFAA0
:10B9400000782188012282409143218010BD0000AF
:10B95000580000203C890100FE4A137882F88730A5
:10B96000A2F8880082F88610012082F8840092F8FC
:10B97000600008B192F85C0082F88A00704710B548
:10B980000B46114658B11846FFF7E6FFF2488068AB
:10B99000008802F0B7FCBDE8104002F06BB9BDE8CA
:10B9A00010404FF6FF70D7E770B5EB4E0446316894
:10B9B00091F89200002501280DD091F88C00012803
:10B9C00018D091F8620001281ED091F88400012857
:10B9D00038D0002070BD65701720207051F8930F8B
:10B9E000C4F802004868C4F80600087AA07201F89A
:10B9F000015C32E0657005202070D1F88E00C4F83B
:10BA0000020081F88C5028E06570112020702022FF
:10BA1000A01C64310CF010FD0121A171306880F888
:10BA20006250CC48B0F86620A0F88E20B268537BF4
:10BA300080F8903080F88C10108802F063FC02F0DF
:10BA400028F90AE065701320207051F8860FC4F8B9
:10BA500002008888E08001F8025C012070BDBE48C9
:10BA6000006890F8621011B1B0F8660070474FF6A8
:10BA7000FF70704770B5B84C206800B9FFDF2068D0
:10BA8000417811B10C25284670BD00259C210CF091
:10BA900074FD2168FF2008707F2081F83600132094
:10BAA0004884282081F86100012081F85800002096
:10BAB00081F85B0006F072FD06F088F8E3E770B5E8
:10BAC000A54C0546206800B9FFDF216800204870BA
:10BAD0006560FFF7CFFF002800D0FFDF70BD9E49F3
:10BAE00009680978814201D1012070470020704720
:10BAF000994800B5016891F82400498CC0F3800290
:10BB0000C0F340031A4400F001001044132915D07B
:10BB100004DC102909D0122904D10FE0152908D01E
:10BB20001D2904D0FFDF002000BD8C4903E08C48B4
:10BB300000BD8A49083131F8100000BD8749083935
:10BB4000F9E7854840F271210068806A48437047F0
:10BB50008148006890F83500002800D00120704727
:10BB600010B57C4C207B00F033FD40B1207D04F10A
:10BB700015010AF033FD082801D0012010BD207BFB
:10BB800030B1022804D00120BDE8104007F08BB886
:10BB90000020F9E76F49087370476F49096881F819
:10BBA0003000704770B506466A4890F82D000AF0DC
:10BBB000A3FC050018D010210AF059FF002813D16A
:10BBC000654C012032462168C87628461C3107F0B2
:10BBD00077F8D4E900101C310BF0CAF96068BDE8B1
:10BBE000704001210BF0D3B970BD2DE9F041594CE3
:10BBF000074694F82D000AF0FCFC064694F82F0046
:10BC000004F10E0528B126B194F82D000AF017FCB6
:10BC1000A0B194F83000002824D094F82E00002819
:10BC200020D0607B294600F0E4FCA8B10AF089FD31
:10BC30003A462946BDE8F04107F042B8012060735A
:10BC40003A462946304607F03BF894F82D1028462E
:10BC5000BDE8F0410AF064BD39462846BDE8F04130
:10BC600007F062B8BDE8F08170B53B4C2168087BF5
:10BC7000B0B1022814D0012048730E3106F0FDFF48
:10BC80002068007B00F0A4FC216881F82F000820C8
:10BC900081F82D00487B0E3100F0A2FC40B901E094
:10BCA0000020E9E72168487B0E3100F0A2FC00B1DA
:10BCB0000120216881F82E0091F82F0018B991F821
:10BCC0002200400706D5087D15310AF087FC21685F
:10BCD00081F82D0020680025456004F023FB2168D1
:10BCE00088600020FFF781FF2068C57690F8220069
:10BCF000400703D5BDE87040002053E770BD164AE9
:10BD00001268137B0370D2F80E000860508A888096
:10BD1000704778B50F4904460F4D407B08732A6879
:10BD2000207810706088ADF8000080B200F001014A
:10BD3000C0F3400341EA4301C0F3800341EA8301B9
:10BD4000C0F3C00341EAC301C0F3001341EA031189
:10BD500008E00000C40400205C0000209489010079
:10BD60008E891300C0F3401341EA4311C0F38010E1
:10BD700041EA80105084E07D012825D0022825D09A
:10BD8000FFDF286880F85A60217B80F82410418CFE
:10BD90001D291DD061688162617D80F83510A17B0D
:10BDA000C1B1022916D00121017554F80F1FC0F846
:10BDB0001510A188A0F81910217B012900D00021BD
:10BDC00080F83410002078BD0126DAE70226D8E793
:10BDD0000021E0E70021E7E7F948006890F8220039
:10BDE000C0F38000704700B5FFF7F6FF08B10020F0
:10BDF00000BD1F2000BD00B5FFF7F5FF002800D0F3
:10BE0000012000BDEE4900220968CA654B8C1D2B3C
:10BE100002D081F86000704781F860207047E84ADE
:10BE20000023126882F8593042F8481F90800120A0
:10BE300050747047E24A0023126882F85830A2F822
:10BE4000540042F8501F012010727047DC49096805
:10BE500081F85B007047DA48006890F95B00704732
:10BE6000D748006890F8220000F001007047D448DD
:10BE7000006890F82200C0F340007047002070472F
:10BE8000CF48006890F82200C0F3C000704701203E
:10BE90007047012070470120704770B500F0BDFB6E
:10BEA000C74C2068C16D491CC16590F8330000255E
:10BEB00030B106F073FB05F089FE206880F833503E
:10BEC0002068457090F8371009B102201AE090F808
:10BED0006010B1B1C06D814213D8022007F048FB59
:10BEE000206890F82200C00704D0A068432201888F
:10BEF000012003E043224FF6FF710020BDE87040AF
:10BF00003DE50020BDE8704007F032BB10B50128C8
:10BF10000DD002280DD004280FD0FFDFA8480068FC
:10BF200090F85A10BDE81040252005F0DBBF252011
:10BF300000E0262006F0AEF8F0E72720FAE70246F8
:10BF40000020D30701D0CB0705D0930705D58B0779
:10BF500003D402207047012070475207FCD54907DF
:10BF6000FAD4042070472DE9F041954C206800B9BF
:10BF7000FFDF20684178D1BB0178FF2938D0002548
:10BF800080F83150A0F85650857080F83750284618
:10BF900006F066FA05F0B2FF206890F95B0006F043
:10BFA00069F8884806F06CF88648C01E06F043FA27
:10BFB000606806F058FA2068002190F82400FFF726
:10BFC000BEFFFFF7A3FF206880F82C5006F042FA6E
:10BFD000206890F85A10002006F0E5F80F2105209F
:10BFE00006F01FF8206890F82E1051B902E0FFE724
:10BFF0000C2037E690F82F1019B990F8220040076E
:10C000002BD504F08FF9804620684146806804F003
:10C01000A2FE6D4F064690FBF7F007FB1060414211
:10C02000404603F080FE2168886096FBF7F04A687E
:10C03000104448600AF0CEFA21684A6890420CD851
:10C04000C1E901580120FFF7D0FD206890F82200D7
:10C05000400702D50120FFF7A5FD2068417B0E3087
:10C0600005F0D3FF206890F8581039B1B0F854109B
:10C07000A0F84410016D016480F8585090F85910F0
:10C0800031B1B0F84C108187816C816380F85950D0
:10C090000AF00DFB032160680AF040FB216881F87B
:10C0A00033000020DEE54649886070472DE9F04105
:10C0B000434C0746002620683146C57E60680680EE
:10C0C00000F0A2FA2068408C132837D004DC102836
:10C0D00058D0122804D153E0152838D01D2836D066
:10C0E000FFDF00BF00F0A4FA2068418C1D2907D0B3
:10C0F000152905D0B0F84420016C60680AF04EFFA5
:10C10000206890F82C1090F82400FFF718FF0546DF
:10C110003FB1FFF7FBFE01224FF49671002006F0BD
:10C1200002F9206890F82C10294380F82C1090F820
:10C1300024208A434FF0010129D02DE000216068BE
:10C140000AF0EAFE0121606800F05EFACAE7012108
:10C1500060680AF0E1FE0121606800F055FAD4E958
:10C16000001025B11C310AF003FF012104E0153154
:10C170000AF0FEFE2068017D60680AF008FFB1E762
:10C18000062100E0022160680AF0C6FEAAE7428CA0
:10C190001D2A0BD080F831104170418C132915D025
:10C1A00007DC10290AD0122907D10FE080F82C6093
:10C1B000F2E715290AD01D2908D0FFDF52E500005B
:10C1C0005C0000208789010040420F0090F85A204F
:10C1D000BDE8F0410121084606F01DBAFA4810B545
:10C1E0000068417841B90078FF2805D00021084651
:10C1F00000F02CFA002010BD00F00FFA0C2010BD4A
:10C2000010B5F14C206890F82200C00704D0A06857
:10C210003C220188012003E03C224FF6FF71002000
:10C22000FFF7ADFB2168012081F8370010BDE6491A
:10C23000096881F83200704770B5002507F0F9F8F9
:10C2400050B1E14C20684178012908D0022901D081
:10C25000032936D0FFDF70BDBDE870401DE6817850
:10C260000029F8D1418C102913D090F8330020B167
:10C2700005F09EFC402006F07EF9206890F8221020
:10C28000490710D490F83510012904D0032902D0B1
:10C2900002E0002119E0102590F85A2045F00E0127
:10C2A000002006F0B8F9206890F8340008B106F0D4
:10C2B0008FF90021962006F002F9216802204870CB
:10C2C00070BD81780029FBD18178BDE870400120E4
:10C2D00000F0BCB9E1E510B5BB4C206890F8340023
:10C2E00008B100F0C6F9206890F8330018B106F0E4
:10C2F00055F905F06BFC07F09CF888B12068407890
:10C30000022800D0FFDF0021012000F09FF9206803
:10C310004178002903D04078012800D0FFDF10BD0C
:10C32000BDE81040B9E510B50AF058F904460AF026
:10C330000AFA38B120460AF0DFF818B110210AF0E5
:10C3400096FB08B1002010BD012010BD2DE9F04181
:10C350009D4C05460F46206890F8620000B1FFDF53
:10C360002168002681F864602888A1F86600688842
:10C37000A1F87C00A888A1F87E00E888A1F88000D8
:10C3800095F84C0181F8820091F82F0020B1487B8C
:10C390000E3100F02EF940B9216891F8300060B1FB
:10C3A000487B0E3100F01CF938B12068D0F80E102F
:10C3B0000167418AA0F8741003E020680667A0F8BE
:10C3C00074606168FF2F0878C0F380106876D1F838
:10C3D0000300C5F81A00B1F80710E98314D02168EA
:10C3E00001F16A02C1F87600E88BA1F87A003846BC
:10C3F00069310AF008F900B9FFDF206810F8691FF9
:10C4000041F0020101702DE42068C0F87660A0F8C8
:10C410007A60697E80F86910D5F81A1040F86A1FB2
:10C42000E98B81801EE42DE9F047DFF89C910E46F0
:10C430000746032809D0FFF713FD0446D9F800008A
:10C4400090F8320020B1012003E0FFF710FD044610
:10C450000020804605F010FE0546032F2BD0012753
:10C4600034EA080453D0D9F800004C4690F8330061
:10C4700068B10AF002F930700146FF2807D0606801
:10C48000C01C0AF0D7F830780AF001F9054360685B
:10C490000178C1F3801221680B7D9A4205D10622F2
:10C4A000C01C15310BF09CFF38B100203178FF29FA
:10C4B0000BD0D8B903E00227D2E70120F6E72068C5
:10C4C00090F82D00884211D008E038B1616811F869
:10C4D000030BC0F38010FFF726FF38B1002021685E
:10C4E00091F82210490703D5A0B910E00120F6E722
:10C4F00085B9364890F8350008B1B84207D161686F
:10C5000011F8030BC0F38010FFF70DFF10B10020EE
:10C51000BDE8F0870120FBE72DE9F0412A4C0746F2
:10C52000002520684078022800D0FFDF206890F8BE
:10C53000340008B100F09DF860680AF00FFD06466F
:10C540009FB160680AF04AFD78B105F066FD60B100
:10C55000062E0AD2DFE806F009090903090600F0F1
:10C56000CAF801E000F094F800B90125206890F8BD
:10C57000330018B106F012F805F028FB1DB10021B8
:10C58000012000F063F820684178002906D0417846
:10C59000012903D04078032800D0FFDF29E570B5DA
:10C5A000094E05460C463068807800280BD105F00E
:10C5B00061FC03463068214690F85A202846BDE8C1
:10C5C000704007F0DCB970BD5C000020C40400209E
:10C5D000022803D0032801D00020704701207047B3
:10C5E000012802D14879800901D00020704701203C
:10C5F0007047012806D148790121B1EB901F01D184
:10C6000001207047002070470278202322F020028A
:10C6100003EA41110A430270704710B505F09EFF0E
:10C6200005F07DFF05F0D2FEBDE8104005F009BF22
:10C6300010B57A4C784960680AF094FC76480E3858
:10C64000417B6068BDE810400AF098BC734A10B5A1
:10C65000126892F8313033B1508C1D2800D1FFDFC1
:10C66000BDE8104019E4002902D1BDE810401DE5E5
:10C6700010BD10B5694C2068363005F0B4FF18B90C
:10C6800021687F2081F83600BDE8104005F096BF94
:10C6900038B5FF208DF80000012569460520FFF719
:10C6A000C2FE28B35D4C2068807800BB6268A06839
:10C6B0001278417BC2F3401211404173012100F016
:10C6C00048F89DF80010A068FFF740FE206801219F
:10C6D00000F8621F827881880120FFF750F92168F5
:10C6E00000204870FFF799FF012006F041FF00E0AD
:10C6F0000025284638BD38B5FF208DF800000125FB
:10C7000069460320FFF78FFE444C002820681BD0A9
:10C7100090F8341031B190F8920018B99DF80000EB
:10C7200000F046F860680021018004210AF0F4FB63
:10C73000FFF77EFF2068828F816B60680AF03EFC05
:10C7400021680320487002E0807800B9002528465F
:10C7500038BD324B10B55A6852F80F4FC0F80E4032
:10C760009488448294790475D47944751489C48278
:10C770005489448094898480D489C48014698460F5
:10C78000147D0473547D04F01F040476527D520915
:10C7900080F84C2180F8341080F83510196891F831
:10C7A000612080F8362091F85B1080F8371010BDBA
:10C7B00070B51A4C0122216881F892200A7881F81C
:10C7C0009320FF280DD001F19502943109F01BFF51
:10C7D00000B9FFDF206810F8941F41F002010170DA
:10C7E0000CE060680278C2F3801281F89420D0F8DF
:10C7F000032041F8952FB0F807008880256895F848
:10C8000036009B357F2800D1FFDF206810F8361FE7
:10C8100029707F210170D6E6D20400205C00002040
:10C820002DE9FC470C460646694600F0D2FD00287B
:10C8300060D1FFF714F9B0425CD02146304608F0D1
:10C840009CFA28BB019D95F8EC00383518B9E87EB4
:10C8500008B1012000E00020814695F837004FF034
:10C8600000084FF0010AA0B195F83800800710D5F4
:10C8700084F8018084F800A084F80280A68095F8EE
:10C880003910A171698F2181A98F618185F8378065
:10C890002DE0304601F048FD070000D1FFDF3846AB
:10C8A00000F076FF40B184F801800D212170A68050
:10C8B000E08084F802A01AE0304601F023FD070072
:10C8C00000D1FFDFB9F1000F14D0384600F0B7FFF8
:10C8D00080B1304606F04DF984F801800A212170BC
:10C8E00084F80280A680297FA17185F81B80012031
:10C8F000BDE8FC870020FBE71CB5694600F069FD38
:10C9000000B1FFDF684600F075FDFC490020896832
:10C91000A1F8B2001CBD2DE9FC4104460E460620DC
:10C9200001F06AFB00250746A846064417E0208868
:10C93000401C80B22080B04202D34046A4F8008060
:10C9400080B2B84204D3B04202D20020BDE8FC81DC
:10C95000694600F03EFD0028F8D06D1CEDB2AE42F5
:10C96000E5D84FF6FF7020801220EFE710B506F0F3
:10C9700071F909F06EFDE2484FF6FF710422418122
:10C9800081810021017003218170C2701B2282808D
:10C99000C280018110BD70B5D84C0D466060217019
:10C9A00006F0E5F800F032FDFFF7E0FF207809F02F
:10C9B00013F8284606F054FED1482838FFF77FF8D0
:10C9C0002178606808F09BFABDE8704009F041BD2D
:10C9D00010B501240AB1002010BD21B1012903D0F6
:10C9E0000024204610BD02210AF028FBF9E72DE9BA
:10C9F000F041040000D1FFDFC14802210C30804625
:10CA0000FFF789FF00B1FFDFBD4D0620AF8901F0C0
:10CA1000F3FA0646A889B04217D12046FEF7C4FFB4
:10CA2000D0B12078132814D1A07890B1A088062125
:10CA300001F036FB68B1008806F09BF8A08806215B
:10CA400001F040FB28B1FFDF03E02146FFF7E8FEDD
:10CA500010B10120BDE8F08102214046FFF75BFFE5
:10CA600010B9A889B842D5D10020F3E710B500F07D
:10CA700091FC08B10C2010BD09F025FD002010BD6F
:10CA800010B50446007818B1012801D0122010BD5D
:10CA900000F08BFC20B109F08DFD08B10C2010BD19
:10CAA000207800F061FCE21D04F11703611CBDE871
:10CAB000104009F02BBD10B5044600F06BFC08B126
:10CAC0000C2010BD207818B1012801D0122010BD13
:10CAD00000F04AFC611C09F0D0FC08B1002010BD38
:10CAE000072010BD10B509F069FD08B1002010BD88
:10CAF000302010BD10B5044600F057FC08B10C20E2
:10CB000010BD204609F052FD002010BD10B500F008
:10CB10004CFC20B109F04EFD08B10C2010BD09F00D
:10CB200037FD002010BDFF2181704FF6FF7181801D
:10CB3000724949680A7882718A88028149884181EC
:10CB400001214170002070471CB5002412F1080F2C
:10CB500015D00CDC12F1280F11D012F1140F0ED0E9
:10CB600012F1100F0BD012F10C0F0CD107E012F1E3
:10CB7000040F04D01AB1032A01D0042A03D10128DA
:10CB800004D0032806D0122420461CBD1046FFF70F
:10CB90005DF9F9E708461446694600F01AFC08B149
:10CBA0000224F1E7019880F837400024ECE710B543
:10CBB0001346012209F077FF002010BD10B504468E
:10CBC00000F0F3FB08B10C2010BD2146002006F058
:10CBD00042F8002010BD10B5044606F0FBFE20B15F
:10CBE000207806F065FD002010BD0C2010BD10B5AA
:10CBF000044600F0DAFB08B10C2010BD21460120EC
:10CC000006F029F8002010BD38B504464FF6FF7035
:10CC1000ADF80000A079E179884216D02079FEF7BE
:10CC200016FB90B16079FEF712FB70B10022A0797B
:10CC300011460AF061FE40B90022E07911460AF07F
:10CC40005BFE10B9207A072801D9122038BD06F002
:10CC5000CDFE48B900216846FFF75DFE20B12046B1
:10CC600005F019F9002038BD0C2038BD2DE9FC4134
:10CC7000817804461A2925D00EDC16292DD2DFE84A
:10CC800001F02C2C2C2C2C212C2C2C2C2C2C2C2C56
:10CC90002C2C2C2C2C2121212A291ED00BDCA1F19B
:10CCA0001E010C2919D2DFE801F0181818181818FD
:10CCB00018181818180D3A3904290ED2DFE801F0B7
:10CCC0000D020D022088B0F5706F06D2012769466B
:10CCD00000F07FFB18B1022038E6122036E6019DF5
:10CCE00068462E4605F5A87506F2511600F064FB5D
:10CCF00008B1287830B10C2028E600006800002038
:10CD0000880500202F70A0783070684600F072FB14
:10CD100000201BE61CB50C46694600F05AFB0021BA
:10CD200018B12160217102201CBD019802463830E3
:10CD300080F8401093682360137B237190F8403093
:10CD4000002BF5D100201CBD10B5044600F02DFBD2
:10CD500020B109F02FFC08B10C2010BD207800F0A4
:10CD600003FBE279611C09F0FAFC08B1002010BD58
:10CD7000022010BD887800B90320C97801B90321C9
:10CD800010701970002070471FB50446008801A973
:10CD900000F01FFB002806D1A08830B1012804D084
:10CDA000022802D0122004B010BD6B4603AA21460F
:10CDB00001A8FFF7DFFF0028F5D1029A012182F8D0
:10CDC0007B11029A92F8AE213AB9029A92F87A212E
:10CDD0001AB9029A92F85D200AB13A200CE0029A40
:10CDE00082F87A11029A9DF80C1082F87C11029A4E
:10CDF0009DF8001082F87D11029A002182F87B11C3
:10CE0000D1E710B504460020A17801B90120E278ED
:10CE10000AB940F0020000F00DFB002803D12046C3
:10CE2000BDE81040B0E710BDF0B544888188C288E5
:10CE3000038945898089A71F40F67B46B74215D2F2
:10CE40008F1FB74212D28C4210D8B2F5FA7F0DD2A2
:10CE5000A3F10A04361FB44208D2521C4A43B2EB73
:10CE6000830F03DA854201D80020F0BD3020F0BDE9
:10CE7000F8B515460E46044606F0B8FD08B10C207C
:10CE8000F8BD204600F0E6FA0028F9D1A078C106E6
:10CE90004FF01100F4D5E17D0329F1D0FEF7DBFF5F
:10CEA0003070A07555B9FF208DF80000694600204C
:10CEB000FEF7C0FF69460020FEF7B1FF2046BDE83F
:10CEC000F840FEF726BF0022D2E770B50C460546B3
:10CED00012B11F2907D80CE0FF2C04D8FEF7D9FFA8
:10CEE00018B11F2C01D9122070BD2846FEF7F7FD9E
:10CEF00008B1002070BD422070BD10B504464088C6
:10CF000010B1FEF778FF78B12078618800F0010257
:10CF10006078FFF7DAFF002805D1FEF764FF62882A
:10CF2000824203D9072010BD122010BD104661684F
:10CF3000FEF780FF002010BD10B50446408810B1F8
:10CF4000FEF795FF70B12078618800F001026078EB
:10CF5000FFF7BBFF002804D160886168FEF75FFF20
:10CF6000002010BD122010BD7CB50446407842253B
:10CF7000012808D8A078FEF7B2FD20B1207812254C
:10CF8000012802D090B128467CBDFEF779FF20B180
:10CF9000A0880028F7D08028F5D8FEF778FF60B188
:10CFA00060780028EFD02078012808D005F0CEFE68
:10CFB000044606F02BFB002864D00C207CBDFEF755
:10CFC000CFFD10B9FEF75AFF60B306F00FFD002841
:10CFD000F3D1FEF744FDA0F57F41FF39EDD1FEF717
:10CFE00043FEA68842F210704643A079FEF70AFF7E
:10CFF000FEF736FFC0B10022062101A801F022F899
:10D00000040018D0F84803218460204609F08AFC07
:10D010002046FFF748F8FEF73CFFF44D68B1288939
:10D0200001210EE012207CBD3146002006F043FBBA
:10D0300038B3FFDF30E009207CBDFEF72CFF01464E
:10D04000288906F0DAFB0146A0620022204605F09E
:10D0500080FEFEF71EFF08B9FEF71DFFE87800907E
:10D06000AB78EA88A988208801F0D5F800B1FFDF05
:10D07000208805F07DFD3146204606F01CFB00B1FE
:10D08000FFDF09E044B1208805F073FD2088062108
:10D0900001F018F800B1FFDF00207CBD002163E73C
:10D0A00070B50D46062100F0FBFF040003D094F894
:10D0B000530110B10AE0022070BD94F84500142815
:10D0C00001D0152802D194F8940108B10C2070BD4C
:10D0D0001022294604F5AA700BF0AEF9012084F85D
:10D0E0005301002070BD10B5062100F0D9FF18B122
:10D0F00090F8531111B107E0022010BD90F84510CF
:10D10000142903D0152901D00C2010BD022180F86C
:10D110005311002010BD2DE9FC410D464BF6803225
:10D120001221954213D895B1694600F052F90028B2
:10D130000CD1019EB41C383627882A463946304621
:10D1400009F0B1FB2088B842F6D100200DE4084672
:10D150000BE41CB504460088694600F03AF9002843
:10D1600008D10199A378084691F82C2038319A42C9
:10D1700001D10C201CBD7F220A728A720022CA7261
:10D18000E17880F82D10217980F82E10A17880F8B0
:10D190002C1010461CBD1CB50C46694600F019F950
:10D1A000002806D1019890F8530000B101202070AA
:10D1B00000201CBD7CB50D461446694600F009F9F7
:10D1C000002805D1019890F82C00012801D00C20EE
:10D1D0007CBD019890F84010297090F841002070B3
:10D1E00000207CBD70B50D461646062100F058FFA4
:10D1F00018B381880124C388428804EB4104AC42FF
:10D2000017D842F210746343A4106243B3FBF2F2E6
:10D21000521E94B24FF4FA72944200D91446A542B9
:10D2200000D22C46491C641CB4FBF1F24A43521E46
:10D2300091B290F880211AB901E0022070BD0184FA
:10D240003180002070BD10B50C46062100F028FF8B
:10D2500048B180F8BF4024B190F8BD1009B106F084
:10D26000E3FA002010BD022010BD017899B1417889
:10D2700089B141881B290ED381881B290BD3C18812
:10D28000022908D359490268283941F82A2F4068F1
:10D290004860002070471220704710B506F07FFAF2
:10D2A000002010BD10B506F07DFA002010BD70B54D
:10D2B00015460A46064600240121104606F09DFA4E
:10D2C000002800D9044601213046653C00F053F89F
:10D2D00006460121002000F04EF831180120963159
:10D2E0008C4206D901F19600611AB1FBF0F0401CA6
:10D2F00080B22880002070BD10B5044600F055F8BB
:10D3000008B10C2010BD601C09F016FA207800F05E
:10D310000100FEF742FC002010BD10B506F03CFAFB
:10D32000002010BD10B50446062000F057FE08B1DD
:10D330000C2010BD2078C00710D000226078114664
:10D340000AF0DAFA08B1122010BDA06808F02BF933
:10D350006078616808F030F9002010BD002008F006
:10D3600022F900210846F5E718B1022801D0012072
:10D3700070470020704710B5012904D0022905D05C
:10D38000FFDF204610BDC000503001E080002C308F
:10D3900084B2F6E710B506F029FB20B1FEF7D8FB02
:10D3A00008B1012010BD002010BD10B506F01EFB15
:10D3B000002800D0012010BD416891F8EC0091F8E0
:10D3C000531021B918B1042801D001207047002062
:10D3D000704710B50C46062100F062FE606038B15F
:10D3E00001202070002010BD68000020880500206A
:10D3F0000220F8E7416891F8BD20002A05D00022FC
:10D4000081F8BD20406806F00FBA704708B54FF6A6
:10D41000FF70ADF8000006E00621BDF8000000F046
:10D4200051FE00B1FFDF00216846FFF774FA0028C3
:10D43000F2D008BD70B514460546012200F055F83B
:10D44000002806D121462846BDE87040002200F0A1
:10D450004CB870BD38B504460078EF2841D86088D4
:10D46000ADF80000009800F04DF888B36188080717
:10D4700008D4D4E90120824233D8202A31D3B0F530
:10D48000804F2ED8207B18B307282AD8607B28B17C
:10D49000012803D0022801D0032822D14A0703D44F
:10D4A000022801D0032805D1A07B08B1012818D19A
:10D4B000480707D4607D28B1012803D0022801D095
:10D4C00003280ED1C806E07D03D5012809D104E068
:10D4D00007E0012801D0032803D1E07E18B101281C
:10D4E00001D0122038BD002038BD0AB1012200E071
:10D4F0000222024202D1880802D109B100207047FD
:10D500001120704780B2C1060BD401071CD48106DC
:10D510004FEAC07101D5B9B900E099B1800713D4C1
:10D5200010E0410610D481060ED4C1074FEA807185
:10D5300004D0002902DB400704D405E0010703D42E
:10D54000400701D4012070470020704730B505889E
:10D5500025F4004421448CB24FF4004194420AD295
:10D56000121B92B21B339A4201D2A94307E005F481
:10D570000041214303E0A21A92B2A9431143018062
:10D5800030BD0844083050434A31084480B27047E7
:10D5900070B51D4616460B46044629463046049A89
:10D5A000FFF7EFFF0646B34200D2FFDF28212046F7
:10D5B0000AF0E3FF4FF6FF70A082283EB0B2657715
:10D5C0006080B0F5004F00D9FFDF618805F13C00B5
:10D5D000814200D2FFDF60880835401B343880B2BA
:10D5E00020801B2800D21B2020800020A07770BD47
:10D5F0008161886170472DE9F05F0D46C18804465E
:10D6000000F12809008921F4004620F4004800F0C8
:10D6100062FB10B10020BDE8F09F4FF0000A4FF010
:10D62000010BB0450CD9617FA8EB0600401A083801
:10D63000854219DC09EB06000021058041801AE0D3
:10D640006088617F801B471A083F0DD41B2F00DACA
:10D65000FFDFBD4201DC294600E0B9B2681A0204CE
:10D66000120C04D0424502DD84F817A0D2E709EB82
:10D6700006000180428084F817B0CCE770B50446FC
:10D6800000F12802C088E37D20F400402BB1104453
:10D690000288438813448B4201D2002070BD0025CC
:10D6A0008A4202D30180458008E0891A0904090CE6
:10D6B000418003D0A01D00F01EFB08E0637F0088BE
:10D6C0000833184481B26288A01DFFF73FFFE5755B
:10D6D000012070BD70B5034600F12804C58880881C
:10D6E00020F400462644A84202D10020188270BDD2
:10D6F00098893588A84206D3401B75882D1A204486
:10D70000ADB2C01E05E02C1AA5B25C7F20443044A7
:10D71000401D0C88AC4200D90D809C8924B10024A6
:10D7200014700988198270BD0124F9E770B50446A8
:10D7300000F12801808820F400404518208A002844
:10D7400025D0A189084480B2A08129886A88114423
:10D75000814200D2FFDF2888698800260844A18919
:10D76000884212D1A069807F2871698819B1201D73
:10D7700000F0C1FA08E0637F28880833184481B2BA
:10D780006288201DFFF7E2FEA6812682012070BD7F
:10D790002DE9F041418987880026044600F12805DB
:10D7A000B94218D004F10A0821F400402844418805
:10D7B00019B1404600F09FFA08E0637F0088083303
:10D7C000184481B262884046FFF7C0FE761C61892A
:10D7D000B6B2B942E8D13046BDE8F0812DE9F0415A
:10D7E00004460B4627892830A68827F40041B4F860
:10D7F0000A8001440D46B74201D10020ECE70AB18E
:10D80000481D106023B1627F691D18460AF014FE9E
:10D810002E88698804F1080021B18A1996B200F0B7
:10D820006AFA06E0637F62880833991989B2FFF7C4
:10D830008DFE474501D1208960813046CCE7818843
:10D84000C088814201D101207047002070470189C2
:10D850008088814201D1012070470020704770B557
:10D860008588C38800F1280425F4004223F4004190
:10D8700014449D421AD08389058A5E1925886388DD
:10D88000EC18A64214D313B18B4211D30EE0437FA0
:10D8900008325C192244408892B2801A80B2233345
:10D8A000984201D211B103E08A4201D1002070BD3B
:10D8B000012070BD2DE9F0478846C18804460089E3
:10D8C00021F4004604F1280720F4004507EB06097F
:10D8D00000F001FA002178BBB54204D9627FA81B91
:10D8E000801A002503E06088627F801B801A083858
:10D8F00023D4E28962B1B9F80020B9F802303BB113
:10D90000E81A2177404518DBE0893844801A09E09D
:10D91000801A217740450ADB607FE1890830304476
:10D9200039440844C01EA4F81280BDE8F08745457C
:10D9300003DB01202077E7E7FFE761820020F4E7BF
:10D940002DE9F74F044600F12805C088884620F4E9
:10D95000004A608A05EB0A0608B1404502D2002061
:10D96000BDE8FE8FE08978B13788B6F8029007EB02
:10D970000901884200D0FFDF207F4FF0000B50EA02
:10D98000090106D088B33BE00027A07FB94630717B
:10D99000F2E7E18959B1607F2944083050440844D6
:10D9A000B4F81F1020F8031D94F821108170E2894B
:10D9B00007EB080002EB0801E1813080A6F802B015
:10D9C00002985F4650B1637F30880833184481B2B3
:10D9D0006288A01DFFF7BAFDE78121E0607FE18941
:10D9E00008305044294408442DE0FFE7E089B4F8AA
:10D9F0001F102844C01B20F8031D94F821108170CB
:10DA000009EB0800E28981B202EB0800E08137806F
:10DA100071800298A0B1A01D00F06DF9A4F80EB0BD
:10DA2000A07F401CA077A07D08B1E088A08284F888
:10DA300016B000BFA4F812B084F817B001208FE729
:10DA4000E0892844C01B30F8031DA4F81F1080781B
:10DA500084F82100EEE710B5818800F1280321F455
:10DA600000442344848AC288A14212D0914210D03B
:10DA7000818971B9826972B11046FFF7E8FE50B929
:10DA80001089283220F40040104419790079884226
:10DA900001D1002010BD184610BD00F12803407FC1
:10DAA00008300844C01E1060088808B9DB1E1360E7
:10DAB00008884988084480B270472DE9F04100F198
:10DAC0002806407F1C4608309046431808884D8839
:10DAD000069ADB1EA0B1C01C80B2904214D9801AF5
:10DAE000A04200DB204687B298183A4641460AF029
:10DAF00077FC002816D1E01B84B2B844002005E072
:10DB0000ED1CADB2F61EE8E7101A80B20119A94269
:10DB100006D8304422464146BDE8F0410AF060BCD8
:10DB20004FF0FF3058E62DE9F04100F12804407F26
:10DB30001E46083090464318002508884F88069AEC
:10DB4000DB1E90B1C01C80B2904212D9801AB04244
:10DB500000DB304685B299182A4640460AF06CFC34
:10DB6000701B86B2A844002005E0FF1CBFB2E41E73
:10DB7000EAE7101A80B28119B94206D82118324654
:10DB800040460AF059FCA81985B2284624E62DE93A
:10DB9000F04100F12804407F1E46083090464318AB
:10DBA000002508884F88069ADB1E90B1C01C80B201
:10DBB000904212D9801AB04200DB304685B29818E4
:10DBC0002A4641460AF038FC701B86B2A844002061
:10DBD00005E0FF1CBFB2E41EEAE7101A80B281190B
:10DBE000B94206D82044324641460AF025FCA8191D
:10DBF00085B22846F0E5401D704710B5044600F197
:10DC00002801C288808820F400431944904206D03D
:10DC1000A28922B9228A12B9A28A904201D1002097
:10DC200010BD0888498831B1201D00F064F800203B
:10DC30002082012010BD637F62880833184481B2BE
:10DC4000201DFFF783FCF2E70021C18101774182AB
:10DC5000C1758175704703881380C28942B1C2883B
:10DC600022F4004300F128021A440A60C089704778
:10DC70000020704710B50446808AA0F57F41FF3927
:10DC800000D0FFDFE088A082E08900B10120A0750C
:10DC900010BD4FF6FF71818200218175704710B56C
:10DCA0000446808AA0F57F41FF3900D1FFDFA07DC7
:10DCB00028B9A088A18A884201D1002010BD012086
:10DCC00010BD8188828A914201D1807D08B10020F7
:10DCD00070470120704720F4004221F400439A422B
:10DCE00007D100F4004001F40041884201D0012036
:10DCF00070470020704730B5044600880D4620F478
:10DD00000040A84200D2FFDF21884FF40040884342
:10DD10002843208030BD70B50C00054609D0082C82
:10DD200000D2FFDF1DB1A1B2286800F044F8201D29
:10DD300070BD0DB100202860002070BD0021026878
:10DD400003E093881268194489B2002AF9D100F0DF
:10DD500032B870B500260D460446082900D2FFDF10
:10DD6000206808B91EE0044620688188A94202D0D4
:10DD700001680029F7D181880646A94201D10068CF
:10DD80000DE005F1080293B20022994209D328441C
:10DD9000491B026081802168096821600160206060
:10DDA00000E00026304670BD00230B608A800268C8
:10DDB0000A600160704700234360021D0181026018
:10DDC0007047F0B50F460188408815460C181E466E
:10DDD000AC4200D3641B3044A84200D9FFDFA01935
:10DDE000A84200D9FFDF3819F0BD2DE9F04188467F
:10DDF00006460188408815460C181F46AC4200D3E1
:10DE0000641B3844A84200D9FFDFE019A84200D9BA
:10DE1000FFDF70883844708008EB0400BDE8F081B3
:10DE20002DE9F041054600881E461746841B8846AA
:10DE3000BC4200D33C442C8068883044B84200D9AE
:10DE4000FFDFA019B84200D9FFDF6888304468803E
:10DE500008EB0400E2E72DE9F04106881D46044680
:10DE6000701980B2174688462080B84201D3C01B83
:10DE700020806088A84200D2FFDF7019B84200D924
:10DE8000FFDF6088401B608008EB0600C6E70000EB
:10DE90002DE9F041BF4D04469046A8780E46A042B9
:10DEA00000D8FFDF05EB8607786A50F8240000B140
:10DEB000FFDFB868002816D0304600F032F901467E
:10DEC000B868FFF746FF05000CD0786A072E40F8C7
:10DED000245000D3FFDFB0484246294650F8263090
:10DEE000204698472846BDE8F0812DE9F843050013
:10DEF0000C46009524D00026E81C20F00300A84220
:10DF000000D0FFDFDFF88C820027314688F80070F0
:10DF100088F8014088F8024088F8034088F80440F7
:10DF200088F8054088F80640684600F003F90020AC
:10DF300042460099C91C21F00301009116B10FE07F
:10DF40000126D9E702EB80035962002106E000BFF9
:10DF5000D3F824C04CF82170491CC9B2A142F7D3B0
:10DF60000099401C01EB8401C0B200910728E0D366
:10DF7000481BBDE8F88310B50446F3F7B0F908B1C3
:10DF8000102010BD2078834A618802EB80009278CF
:10DF90000EE0436A53F8213043B14A1C6280A180ED
:10DFA000406A50F82100A060002010BD491C89B2D1
:10DFB0008A42EED86180052010BD70B505460C463A
:10DFC0000846F3F78CF908B1102070BD072D01D376
:10DFD000072070BD25700020608070BD0EB56946B9
:10DFE000FFF7EBFF00B1FFDF6846FFF7C4FF08B1A2
:10DFF00000200EBD01200EBD10B50446072800D339
:10E00000FFDF6448005D10BD3EB50546002469464B
:10E01000FFF7D3FF18B1FFDF01E0641CE4B26846EC
:10E02000FFF7A9FF0028F8D02846FFF7E5FF001BFF
:10E03000C0B23EBD57498978814201D9C0B270470C
:10E04000FF2070472DE9F04106291BD1514C0027D4
:10E050003B464FF6FF7604EB810514F801C00AE059
:10E06000DC19D5F824E0A4B25EF824E0BEF1000F7C
:10E0700004D05B1C9BB29C45F2D8344604802046F9
:10E08000B44201D100202EE7BDE8F04100E7A0F541
:10E090007F43FF3B01D0072901D300207047F7E6FB
:10E0A000A0F57F42FF3A0BD0072909D2394A93786D
:10E0B000834205D902EB8101496A51F8200070477B
:10E0C000002070472DE9F04104460D46A4F57F413C
:10E0D00043F20200FF3902D0072D01D3072002E7E7
:10E0E0002C494FF000088A78A242F8D901EB850646
:10E0F000726A52F82470002FF1D0274839461C303C
:10E1000050F8252020469047716A284641F824801F
:10E1100000F007F802463946B068FFF745FE0020D8
:10E12000E1E61D49383131F810004FF6FC71C01C92
:10E13000084070472DE9F843164E884605460024EE
:10E140002868C01C20F0030028602046FFF7E9FF84
:10E15000315D4843B8F1000F01D0002200E02A6889
:10E160000146009232B100274FEA0D00FFF7D3FDC0
:10E170001FB106E001270020F8E706EB8401009AB2
:10E180008A602968641C0844E4B22860072CD7D34D
:10E19000EFE6000098050020A489010070B50E4646
:10E1A0001D46114600F0D4F804462946304600F0DA
:10E1B000D8F82044001D70BD2DE9F04190460D4671
:10E1C00004004FF0000610D00027E01C20F00300F0
:10E1D000A04200D0FFDFDDB141460020FFF79BFDEC
:10E1E0000C3000EB850617B112E00127EDE7614F17
:10E1F00004F10C00A9003C602572606000EB850012
:10E20000206060680AF0B9F941463868FFF783FD7D
:10E210003046BDE8F0812DE9FF4F564C804681B075
:10E2200020689A46934600B9FFDF2068027A42458B
:10E2300003D9416851F8280020B143F2020005B02B
:10E24000BDE8F08F5146029800F082F886B2584639
:10E250000E9900F086F885B27019001D87B220680B
:10E26000A14639460068FFF774FD04001FD067809F
:10E2700025802946201D0E9D07465A4601230095FC
:10E28000FFF786F92088314638440123029ACDF8F9
:10E2900000A0FFF77DF92088C1193846FFF7A8F9DB
:10E2A000D9F800004168002041F82840C7E7042061
:10E2B000C5E770B52F4C0546206800B9FFDF206820
:10E2C000017AA9420ED9426852F8251051B10023B3
:10E2D00042F825304A880068FFF766FD2168002073
:10E2E0000A7A08E043F2020070BD4B6853F8203010
:10E2F00033B9401CC0B28242F7D80868FFF71EFD50
:10E30000002070BD70B51B4E05460024306800B972
:10E31000FFDF3068017AA94204D9406850F825002F
:10E3200000B1041D204670BD70B5124E0546002494
:10E33000306800B9FFDF3068017AA94206D9406829
:10E3400050F8251011B131F8040B4418204670BD67
:10E3500010B50A460121FFF714F9C01C20F0030094
:10E3600010BD10B50A460121FFF70BF9C01C20F0C3
:10E37000030010BD7400002070B50446C2F1100502
:10E3800028190AF059F815F0FF0108D0491EC9B242
:10E39000802060542046BDE870400AF0CCB870BDC3
:10E3A00030B505E05B1EDBB2CC5CD55C6C40C45480
:10E3B000002BF7D130BD10B5002409E00B78521EB8
:10E3C00044EA430300F8013B11F8013BD2B2DC09F7
:10E3D000002AF3D110BD2DE9F04389B01E46DDE9D6
:10E3E000107990460D00044622D002460846F949AD
:10E3F000FEF7DDFB102221463846FFF7DCFFE07B0D
:10E40000000606D5F34A3946102310320846FFF7B6
:10E41000C7FF102239464846FFF7CDFFF87B0006BC
:10E4200006D5EC4A4946102310320846FFF7B8FFDC
:10E43000102120460AF07FF80DE0103EB6B208EB3E
:10E440000601102322466846FFF7AAFF2246284607
:10E450006946FEF7ACFB102EEFD818D0F2B2414659
:10E460006846FFF789FF10234A46694604A8FFF76C
:10E4700097FF1023224604A96846FFF791FF224622
:10E4800028466946FEF793FB09B0BDE8F0831023E8
:10E490003A464146EAE770B59CB01E46054613462B
:10E4A00020980C468DF80800202219460DF109002D
:10E4B00009F0C2FF202221460DF1290009F0BCFF1E
:10E4C00017A913A8CDE90001412302AA3146284625
:10E4D000FFF781FF1CB070BD2DE9FF4F9FB014AE58
:10E4E000DDE92D5410AFBB49CDE900762023203162
:10E4F0001AA8FFF770FF4FF000088DF808804FF062
:10E5000001098DF8099054F8010FCDF80A00A08890
:10E51000ADF80E0014F8010C1022C0F340008DF885
:10E52000100055F8010FCDF81100A888ADF81500BE
:10E5300015F8010C2C99C0F340008DF8170006A8BF
:10E54000824609F079FF0AA883461022229909F031
:10E5500073FFA0483523083802AA40688DF83C8034
:10E56000CDE900760E901AA91F98FFF734FF8DF8B9
:10E5700008808DF809902068CDF80A00A088ADF8D1
:10E580000E0014F8010C1022C0F340008DF81000AA
:10E590002868CDF81100A888ADF8150015F8010C11
:10E5A0002C99C0F340008DF81700504609F044FF45
:10E5B00058461022229909F03FFF86483523083833
:10E5C00002AA40688DF83C90CDE900760E901AA919
:10E5D0002098FFF700FF23B0BDE8F08FF0B59BB0A7
:10E5E0000C460546DDE922101E461746DDE92032BD
:10E5F000D0F801C0CDF808C0B0F805C0ADF80CC027
:10E600000078C0F340008DF80E00D1F80100CDF87D
:10E610000F00B1F80500ADF8130008781946C0F3F3
:10E6200040008DF815001088ADF8160090788DF830
:10E6300018000DF11900102209F0FEFE0DF129005D
:10E640001022314609F0F8FE0DF13900102239464A
:10E6500009F0F2FE17A913A8CDE90001412302AA8F
:10E6600021462846FFF7B7FE1BB0F0BDF0B5A3B0BA
:10E6700017460D4604461E46102202A8289909F0A6
:10E68000DBFE06A82022394609F0D6FE0EA820227D
:10E69000294609F0D1FE1EA91AA8CDE90001502390
:10E6A00002AA314616A8FFF796FE1698206023B0FE
:10E6B000F0BDF0B589B00446DDE90E070D463978A6
:10E6C000109EC1F340018DF8001031789446C1F3DB
:10E6D00040018DF801101968CDF802109988ADF845
:10E6E000061099798DF808100168CDF80910818815
:10E6F000ADF80D1080798DF80F0010236A46614641
:10E7000004A8FFF74DFE2246284604A9FEF74FFA5B
:10E71000D6F801000090B6F80500ADF80400D7F86F
:10E720000100CDF80600B7F80500ADF80A0000209A
:10E73000039010236A46214604A8FFF731FE2246C3
:10E74000284604A9FEF733FA09B0F0BD1FB51C68CE
:10E7500000945B6801931368029352680392024627
:10E7600008466946FEF723FA1FBD10B588B0044677
:10E7700010680490506805900020069007900846A5
:10E780006A4604A9FEF713FABDF80000208008B01D
:10E7900010BD1FB51288ADF800201A88ADF8022010
:10E7A0000022019202920392024608466946FEF751
:10E7B000FEF91FBD7FB5074B14460546083B9A1C62
:10E7C0006846FFF7E6FF224669462846FFF7CDFF79
:10E7D0007FBD0000F289010070B5044600780E4646
:10E7E000012813D0052802D0092813D10EE0A06813
:10E7F00061690578042003F075F9052D0AD07823A6
:10E8000000220420616903F0C3F803E00420616979
:10E8100003F068F931462046BDE8704001F084B845
:10E8200010B500F12D03C2799C78411D144064F3AA
:10E830000102C271D2070DD04A795C7922404A7137
:10E840000A791B791A400A718278C9788A4200D9FC
:10E85000817010BD00224A71F5E74178012900D08E
:10E860000C21017070472DE9F04F93B04FF0000B71
:10E870000C690D468DF820B0097801260C2017464A
:10E880004FF00D084FF0110A4FF008091B2975D2FF
:10E89000DFE811F01B00C20205031D035C036F03D8
:10E8A000A103B603F7031804600492049F04EB0469
:10E8B0002905330551055C05ED0530063306620672
:10E8C0007E06F8061C07E506EA0614B120781D2826
:10E8D0002AD0D5F808805FEA08004FD001208DF8D3
:10E8E0002000686A02220D908DF824200A208DF8FD
:10E8F0002500A8690A90A8880028EED098F8001092
:10E9000091B10F2910D27DD2DFE801F07C1349DEEE
:10E91000FCFBFAF9F8F738089CF6F50002282DD12F
:10E9200024B120780C2801D00026EEE38DF82020B9
:10E93000CAE10420696A03F0D5F8A8880728EED157
:10E94000204600F0ECFF022809D0204600F0E7FF47
:10E95000032807D9204600F0E2FF072802D2012051
:10E96000207004E0002CB8D020780128D7D198F886
:10E970000400C11F0A2902D30A2061E0C3E1A0708C
:10E98000D8F80010E162B8F80410218698F8060063
:10E9900084F83200012028700320207044E007280A
:10E9A000BDD1002C99D020780D28B8D198F803104B
:10E9B00094F82F20C1F3C000C2F3C002104201D06E
:10E9C000062000E00720890707D198F805100142CA
:10E9D000D2D198F806100142CED194F8312098F89F
:10E9E000051020EA02021142C6D194F8322098F8AC
:10E9F000061090430142BFD198F80400C11F0A29B4
:10EA0000BAD200E006E2617D81427CD8D8F80010DD
:10EA10006160B8F80410218198F80600A072012006
:10EA200028700E20207003208DF82000686A0D9059
:10EA300004F12D000990601D0A900F300B9021E128
:10EA40002875FDE3412891D1204600F068FF042895
:10EA500002D1E078C00704D1204600F060FF0F2803
:10EA600084D1A88CD5F80C8080B24FF0400BE669B9
:10EA7000FFF748FC324641465B464E46CDF80090D3
:10EA8000FFF751F80B208DF82000686A0D90E069BF
:10EA90000990002108A8FFF79FFE2078042806D0DF
:10EAA000A07D58B1012809D003280AD048E30520E9
:10EAB0002070032028708DF82060CCE184F800A03D
:10EAC00032E712202070E8E11128BCD1204600F086
:10EAD00026FF042802D1E078C00719D0204600F0B4
:10EAE0001EFF062805D1E078C00711D1A07D0228BD
:10EAF0000ED0204608E0CBE084E070E14FE122E157
:10EB000002E1E8E019E0AEE100F009FF11289AD136
:10EB1000102208F1010104F13C0009F08DFC60783D
:10EB200001286ED012202070E078C00760D0A07D50
:10EB30000028C8D00128C6D05AE0112890D120461C
:10EB400000F0EDFE082804D0204600F0E8FE13286F
:10EB500086D104F16C00102208F10101064609F08B
:10EB60006BFC207808280DD014202070E178C807AD
:10EB70000DD0A07D02280AD06278022A04D0032892
:10EB8000A1D035E00920F0E708B1012837D1C80746
:10EB900013D0A07D02281DD000200090D4E90621CA
:10EBA00033460EA8FFF777FC10220EA904F13C00B3
:10EBB00009F016FCC8B1042042E7D4E90912201D6F
:10EBC0008DE8070004F12C0332460EA8616BFFF7B5
:10EBD00070FDE9E7606BC1F34401491E0068C8405D
:10EBE00000F0010040F08000D7E72078092806D126
:10EBF00085F800908DF8209032E32870EBE309202F
:10EC0000FBE79CE1112899D1204600F088FE0A28F4
:10EC100002D1E078C00704D1204600F080FE15281C
:10EC20008CD104F13C00102208F10101064609F0E4
:10EC300003FC20780A2816D016202070D4E9093267
:10EC4000606B611D8DE80F0004F15C0304F16C0240
:10EC500047310EA8FFF7C2FC10220EA9304609F07A
:10EC6000BFFB18B1F6E20B20207071E22046FFF7DF
:10EC7000D7FDA078216A0A18C0F11001104609F0EA
:10EC80005AFC23E3394608A8FFF7A6FD06463BE2F7
:10EC90000228B8D1204600F042FE042804D32046C2
:10ECA00000F03DFE082809D3204600F038FE0E286B
:10ECB00029D3204600F033FE122824D2A07D02285A
:10ECC000A1D10E208DF82000686A0D9098F80100FF
:10ECD0008DF82400F0E3022895D1204600F01FFEB5
:10ECE000002810D0204600F01AFE0128F9D0204656
:10ECF00000F015FE0C28F4D004208DF8240098F8BC
:10ED000001008DF825005EE21128FCD1002CFAD01C
:10ED100020781728F7D16178606A022911D0002184
:10ED200001EB4101182606EBC1011022405808F101
:10ED3000010109F081FB0420696A00F0E3FD2670FF
:10ED4000F2E50121ECE70B28DDD1002CDBD02078A7
:10ED50001828D8D16078616A02281CD05FF00000C2
:10ED600000EB4002102000EBC2000958B8F8010087
:10ED700008806078616A02280FD0002000EB400212
:10ED8000142000EBC2000958404650F8032F0A60D7
:10ED90004068486039E00120E2E70120EEE71128F1
:10EDA000B1D1002CAFD020781928ACD16178606A3D
:10EDB000022912D05FF0000101EB41011C2202EB9D
:10EDC000C1011022405808F1010109F035FB04206F
:10EDD000696A00F097FD1A20B6E00121ECE70828E7
:10EDE00091D1002C8FD020781A288CD1606A98F8A5
:10EDF0000120017862F347010170616AD8F80220AE
:10EE000041F8012FB8F8060088800420696A00F0F4
:10EE100079FD8EE2072013E63878012894D1182274
:10EE200004F11400796809F04CFBE079C10894F80A
:10EE30002F0001EAD001E07861F30000E070217D4D
:10EE4000002974D12178032909D0C00725D00320D7
:10EE500028708DF82090686A0D90412004E3607D51
:10EE6000A178884201D90620EAE502262671E179D7
:10EE7000204621F0E001E171617A21F0F001617238
:10EE8000A17A21F0F001A172FFF7CAFC2E708DF873
:10EE90002090686A0D900720E6E20420ADE63878FD
:10EEA00005289DD18DF82000686A0D90B8680A90F9
:10EEB0000720ADF824000A988DF830B06168016031
:10EEC00021898180A17A817104202070F4E239784F
:10EED000052985D18DF82010696A0D91391D09AE7B
:10EEE0000EC986E80E004121ADF824108DF830B02F
:10EEF0001070A88CD7F80C8080B24026A769FFF765
:10EF000013FA41463A463346C846CDF80090FEF71C
:10EF10003EFE002108A8FFF75FFCE07820F03E00ED
:10EF2000801CE0702078052802D00F200CE049E119
:10EF3000A07D20B1012802D0032802D002E10720E1
:10EF4000C0E584F80080EFE42070EDE4102104F1C6
:10EF50005C0002F0E8FA606BB0BBA07D18B101283C
:10EF600001D00520FDE006202870F7486063A0630B
:10EF7000BEE23878022894D1387908B12875B3E315
:10EF8000A07D022802D0032805D022E0B86800281E
:10EF9000F5D060631CE06078012806D0A07994F871
:10EFA0002E10012805D0E84806E0A17994F82E003B
:10EFB000F7E7B8680028E2D06063E078C00701D0C6
:10EFC000012902D0E04803E003E0F8680028D6D029
:10EFD000A063062011E68DF82090696A0D91E17812
:10EFE0004846C90709D06178022903D1A17D29B11A
:10EFF000012903D0A17D032900D00720287031E129
:10F0000038780528BBD1207807281ED084F800A0C6
:10F0100005208DF82000686A0D90B8680A90ADF858
:10F0200024A08DF830B003210170E178CA070FD019
:10F03000A27D022A1AD000210091D4E9061204F11F
:10F040005C03401CFFF727FA67E384F80090DFE7D2
:10F05000D4E90923211D8DE80E0004F12C0304F1ED
:10F060005C02401C616BFFF724FB56E3626BC1F34B
:10F070004401491E1268CA4002F0010141F08001BA
:10F08000DAE738780528BDD18DF82000686A0D9040
:10F09000B8680A90ADF824A08DF830B0042100F8CB
:10F0A000011B102204F15C0109F0C6F9002108A837
:10F0B000FFF792FB2078092801D0132044E70A20AB
:10F0C00020709CE5E078C10742D0A17D012902D0E3
:10F0D000022927D038E0617808A8012916D004F168
:10F0E0006C010091D4E9061204F15C03001DFFF7E6
:10F0F000BDFA0A20287003268DF82080686A0D90DA
:10F10000002108A8FFF768FBDDE2C3E204F15C011F
:10F110000091D4E9062104F16C03001DFFF7A6FA63
:10F120000026E9E7C0F3440114290DD24FF0006135
:10F1300001EBB0104FEAB060E0706078012801D0B8
:10F140001020BFE40620FFE6607801283FF4B8AC49
:10F150000A2052E5E178C90708D0A17D012903D131
:10F160000B20287004202FE028702DE00E2028703E
:10F170006078616B012817D004F15C0304F16C0224
:10F180000EA8FFF7E3FA2046FFF74AFBA0780EAE81
:10F19000C0F11001304409F0CEF906208DF82000AE
:10F1A000686A09960D909AE004F16C0304F15C0220
:10F1B0000EA8FFF7CBFAE9E73978022903D13979AC
:10F1C0000029D1D029758FE28DF82000686A0D9052
:10F1D00058E538780728F6D1D4E909216078012864
:10F1E00009D000BF04F16C00CDE90002029105D105
:10F1F00004F16C0304E004F15C00F5E704F15C0346
:10F2000004F14C007A680646216AFFF765F96078D8
:10F21000012821D1A078216A0A18C0F110011046F6
:10F2200009F089F9D4E90923606B04F12D018DE817
:10F230000F0004F15C0304F16C0231460EA800E0FB
:10F2400054E2FFF7CBF910220EA904F13C0009F0BB
:10F25000C7F808B10B20AFE485F800808DF8209046
:10F26000686A0D908DF824A00CE538780528AAD19D
:10F270008DF82000686A0D90B8680A90ADF824A057
:10F280008DF830B080F80080617801291AD0D4E977
:10F29000093204F12D01A66B03920096CDE901130A
:10F2A00004F16C0304F15C0204F14C01401CFFF713
:10F2B00095F9002108A8FFF78FFA6078012805D09A
:10F2C000152041E6D4E90923611DE4E70E202870EA
:10F2D00006208DF82000686ACDF824B00D90A07843
:10F2E0008DF82800CEE438780328C0D1E079C00733
:10F2F00070D00F202870072066E7387804286BD17B
:10F300001422391D04F1140009F0DBF8616A208C25
:10F31000A1F80900616AA078C871E179626A01F018
:10F3200003011172616A627A0A73616AA07A81F8D4
:10F330002400162061E485F800A08DF82090696A09
:10F3400050460D9190E00000F289010038780528C0
:10F3500042D1B868A8616178606A022901D00121B0
:10F3600000E0002101EB4101142606EBC1014058E9
:10F37000082102F0D8F86178606A022901D00121E1
:10F3800000E0002101EB410106EBC101425802A857
:10F39000E169FFF70FFA6078626A022801D0012064
:10F3A00000E0002000EB4001102000EBC100022330
:10F3B000105802A90932FEF7F3FF626AFD4B0EA84E
:10F3C0000932A169FFF7E5F96178606A022904D082
:10F3D000012103E042E18BE0BDE0002101EB4101AE
:10F3E000182606EBC101A27840580EA909F024F8AE
:10F3F0006178606A022901D0012100E0002101EB5F
:10F40000410106EBC1014058A1780844C1F1100147
:10F4100009F091F805208DF82000686A0D90A86920
:10F420000A90ADF824A08DF830B006210170627802
:10F43000616A022A01D0012200E0002202EB4202AE
:10F4400006EBC202401C8958102208F0F5FF00218B
:10F4500008A8FFF7C1F91220C5F818B028708DF878
:10F460002090686A0D900B208DF824000AE438780B
:10F47000052870D18DF82000686A0D90B8680A9050
:10F480000B20ADF824000A98072101706178626AA8
:10F49000022901D0012100E0002101EB41031021EC
:10F4A00001EBC30151580988A0F801106178626A24
:10F4B000022902D0012101E02FE1002101EB4103EB
:10F4C000142101EBC30151580A6840F8032F496821
:10F4D000416059E01920287001208DF8300077E64E
:10F4E000162028708DF830B0002108A8FFF774F9B5
:10F4F000032617E114202870B0E6387805282AD1B1
:10F500008DF82000686A0D90B8680A90ADF824A0C4
:10F510008DF830B080F800906278616A4E46022A19
:10F5200001D0012200E0002202EB42021C2303EB87
:10F53000C202401C8958102208F07EFF002108A852
:10F54000FFF74AF9152028708DF82060686A0D9041
:10F550008DF824603CE680E0387805287DD18DF870
:10F560002000686A0D90B8680A90ADF824900921CF
:10F5700001706169097849084170616951F8012F8A
:10F58000C0F802208988C18020781C28A8D1A1E772
:10F59000E078C00702D04FF0060C01E04FF0070CF6
:10F5A000607802280AD000BF4FF0000000EB040191
:10F5B00001F1090105D04FF0010004E04FF0010016
:10F5C000F4E74FF000000B78204413EA0C030B70B3
:10F5D00010F8092F02EA0C02027004D14FF01B0C44
:10F5E00084F800C0D2B394F801C0BCF1010F00D080
:10F5F0009BB990F800C0E0465FEACC7C04D028F0CC
:10F6000001060670102606E05FEA887C05D528F022
:10F610000206067013262E70032694F801C0BCF172
:10F62000020F00D092B991F800C05FEACC7804D004
:10F630002CF001060E70172106E05FEA8C7805D5E4
:10F640002CF002060E701921217000260078D0BB24
:10F65000CAB3C3BB1C20207035E012E002E038784A
:10F66000062841D11A2019E4207801283CD00C2822
:10F670003AD02046FFF7F1F809208DF82000686A9B
:10F680000D9031E03878052805D006203870032623
:10F690001820287046E005218DF82010686A0D902A
:10F6A000B8680A900220ADF8240001208DF83000DF
:10F6B0000A980170297D4170394608A8FFF78CF837
:10F6C000064618202870012E0ED02BE001208DF860
:10F6D0002000686A0D9003208DF82400287D8DF8A5
:10F6E000250085F814B012E0287D80B11D2020701F
:10F6F000172028708DF82090686A0D9002208DF8F0
:10F700002400394608A8FFF767F806460AE00CB15E
:10F71000FE2020709DF8200020B1002108A8FFF7EE
:10F720005BF810E413B03046BDE8F08F2DE9F043EC
:10F7300087B00C464E6900218DF804100120257811
:10F74000034602274FF007094FF0050C85B1012D44
:10F7500053D0022D39D1FE2030708DF80030606A10
:10F76000059003208DF80400207E8DF8050063E0ED
:10F770002179012925D002292DD0032928D0042957
:10F7800023D1B17D022920D131780D1F042D04D35E
:10F790000A3D032D01D31D2917D12189022914D334
:10F7A0008DF80470237020899DF8041088421BD2C4
:10F7B000082001E0EA8901008DF80000606A0590E8
:10F7C00057E070780128EBD0052007B0BDE8F08342
:10F7D0001D203070E4E771780229F5D131780C29C9
:10F7E000F3D18DF80490DDE7083402F804CB94E8F7
:10F7F0000B0082E80B000320E7E71578052DE4D124
:10F800008DF800C0656A0595956802958DF8101011
:10F8100094F80480B8F1010F13D0B8F1020F2DD085
:10F82000B8F1030F1CD0B8F1040FCED1ADF80470BD
:10F830000E202870207E687000216846FEF7CCFFFD
:10F840000CE0ADF804700B202870207E002100F041
:10F850001F0068706846FEF7BFFF37700020B4E7EE
:10F86000ADF804708DF8103085F800C0207E687007
:10F87000277011466846FEF7AFFFA6E7ADF8049083
:10F880002B70207F6870607F00F00100A870A07F5F
:10F8900000F01F00E870E27F2A71C0071CD094F8C6
:10F8A000200000F00700687194F8210000F00700C4
:10F8B000A87100216846FEF78FFF2868F062A888CB
:10F8C0003086A87986F83200A0694078707528796A
:10F8D000B0700D203070C1E7A9716971E9E700B51A
:10F8E00087B004280CD101208DF800008DF80400A9
:10F8F000002005918DF8050001466846FEF76CFF73
:10F9000007B000BD70B50C46054602F0EBF8214685
:10F910002846BDE870407823002202F039B808B1CB
:10F92000007870470C20704770B50C0005784FF0D8
:10F9300000010CD021702146F3F76EFC6948217854
:10F94000405D884201D1032070BD022070BDF3F7F5
:10F9500063FC002070BD0279012A05D000220A70E4
:10F960004B78012B02D003E0042070470A758A61AE
:10F9700002799300521C0271C15003207047F0B508
:10F9800087B00F4605460124287905EB800050F822
:10F99000046C7078411E02290AD252493A4608394D
:10F9A00001EB8000314650F8043C28469847044655
:10F9B0000CB1012C11D12879401E10F0FF002871E4
:10F9C00001D00324E0E70A208DF80000706A05905A
:10F9D000002101966846FFF7A7FF032CD4D007B09B
:10F9E0002046F0BD70B515460A4604462946104625
:10F9F000FFF7C5FF064674B12078FE280BD1207CA6
:10FA000030B100202870294604F10C00FFF7B7FF41
:10FA10002046FEF722FF304670BD704770B50E4697
:10FA200004467C2108F0A9FD0225012E03D0022EF8
:10FA300004D0052070BD0120607000E06570204694
:10FA4000FEF70BFFA575002070BD28B1027C1AB12E
:10FA50000A4600F10C01C5E70120704710B50446C5
:10FA600086B0042002F03EF82078FE2806D0002060
:10FA70008DF8000069462046FFF7E7FF06B010BD8D
:10FA80007CB50E4600218DF804104178012903D081
:10FA9000022903D0002405E0046900E044690CB1A8
:10FAA000217C89B16D4601462846FFF754FF0328A3
:10FAB00009D1324629462046FFF794FF9DF80410ED
:10FAC000002900D004207CBD04F10C05EBE730B424
:10FAD0000C460146034A204630BC034B0C3AFEF765
:10FAE00058BE0000308A0100EA89010070B50D4659
:10FAF000040011D085B12101284608F01CFD102218
:10FB00005449284608F098FC5248012108380180E1
:10FB100044804560002070BD012070BD70B54D4E21
:10FB200000240546083E10E07068AA7B00EB041034
:10FB3000817B914208D1C17BEA7B914204D10C22A6
:10FB4000294608F04DFC30B1641C30888442EBDB60
:10FB50004FF0FF3070BD204670BD70B50D460600F9
:10FB600006D02DB1FFF7DAFF002803DB401C14E0BC
:10FB7000102070BD374C083C20886288411C91429F
:10FB800001D9042070BD6168102201EB00103146DC
:10FB900008F052FC2088401C20802870002070BD96
:10FBA0002C480838008870472A49083908880128F5
:10FBB00002D0401E08800020704770B514460D002A
:10FBC00018D0BCB10021A170022802D0102811D198
:10FBD00005E0288870B10121A170108008E0284656
:10FBE000FFF79CFF002805DB401CA070A88920803F
:10FBF000002070BD012070BD70B5054614460E0092
:10FC00000BD000203070A878012808D005D9114900
:10FC1000A1F108010A8890420AD9012070BD24B1DF
:10FC2000287820702888000A5070022008700FE0A1
:10FC300064B14968102201EB00112046103908F028
:10FC4000FBFB287820732888000A6073102030702E
:10FC5000002070BD800000202DE9F04190460C4648
:10FC600007460025FE48072F00EB881607D2DFE87D
:10FC700007F00707070704040400012500E0FFDF81
:10FC800006F81470002D13D0F548803000EB880181
:10FC900091F82700202803D006EB4000447001E0D3
:10FCA00081F8264006EB44022020507081F827405E
:10FCB000BDE8F081F0B51F4614460E460546202AE1
:10FCC00000D1FFDFE649E648803100EB871C0CEBF2
:10FCD000440001EB8702202E07D00CEB4601407850
:10FCE0004B784870184620210AE092F82530407879
:10FCF00082F82500F6E701460CEB410005704078DC
:10FD0000A142F8D192F82740202C03D00CEB4404F8
:10FD1000637001E082F826300CEB4104202363700D
:10FD200082F82710F0BD30B50D46CE4B44190022A5
:10FD3000181A72EB020100D2FFDFCB48854200DDCA
:10FD4000FFDFC9484042854200DAFFDFC548401C5A
:10FD5000844207DA002C01DB204630BDC148401C3C
:10FD6000201830BDBF48C043FAE710B5044601680B
:10FD7000407ABE4A52F82020114450B10220084473
:10FD800020F07F40F8F7CBFE94F90810BDE8104052
:10FD9000C9E70420F3E72DE9F047B14E803696F825
:10FDA0002D50DFF8BC9206EB850090F8264034E039
:10FDB00009EB85174FF0070817F81400012806D043
:10FDC00004282ED005282ED0062800D0FFDF01F011
:10FDD0000AF9014607EB4400427806EB850080F8FB
:10FDE000262090F82720A24202D1202280F8272046
:10FDF000084601F003F92A4621460120FFF72CFFAF
:10FE00009B48414600EB041002682046904796F854
:10FE10002D5006EB850090F82640202CC8D1BDE877
:10FE2000F087022000E003208046D0E710B58C4C1C
:10FE30002021803484F8251084F8261084F82710B7
:10FE4000002084F8280084F82D0084F82E10411E2C
:10FE5000A16044F8100B2074607420736073A07369
:10FE60008449E07720750870487000217C4A103C76
:10FE700002F81100491CC9B22029F9D30120F8F772
:10FE800042FD0020F8F73FFD012084F82200F3F73F
:10FE900025F87948F3F737F8764CA41E2070774898
:10FEA000F3F731F86070BDE81040F8F7B9BC10B551
:10FEB000F8F7DBFC6F4CA41E2078F3F73DF8607870
:10FEC000F3F73AF8BDE8104001F0C5B820207047BC
:10FED0002DE9F34F624C0025803404EB810A89B090
:10FEE0009AF82500202821D0691E029160490095CA
:10FEF00001EB0017391D03AB07C983E80700A18B8D
:10FF0000ADF81C10A07F8DF81E009DF81500A046CE
:10FF1000C8B10226554951F820400399A21911444D
:10FF200021F07F41019184B102210FE00120F8F717
:10FF3000EAFC0020F8F7E7FCF8F7B5FC01F08BF8D5
:10FF400084F82F50A7E00426E4E700218DF818106C
:10FF5000022801D0012820D1039801190998081A14
:10FF6000801C9DF81C1020F07F4001B1022135312A
:10FF700081420BD203208DF815000398C4F13201A1
:10FF8000401A20F07F40322403900CE098F82400BF
:10FF900018B901F0F8F900284DD0322C03D214B171
:10FFA00001F04DF801E001F056F8324A107820B324
:10FFB00093465278039B121B00219DF818409946E6
:10FFC00001281BD0032819D05FF000008DF81E0017
:10FFD000002A04DD981A039001208DF818009DF87E
:10FFE0001C0000B102210398254A20F07F400390B5
:10FFF00003AB099801F03BF810B110E00120E5E7F0
:020000040001F9
:100000009DF81D0018B99BF80000032812D08DF848
:100010001C50CDF80C908DF818408DF81E509DF8AE
:10002000180058B103980123811900221846F8F7E7
:10003000BDFC06E000200BB0BDE8F08F0120F8F712
:1000400062FC97F90C20012300200199F8F7AEFC1F
:10005000F87BC00701D0F8F78EFD012112E0000007
:10006000D8070020FF7F841E0020A107408A0100DE
:10007000D8050020920000203F18010097FD0000E5
:10008000FFFF3F0088F82F108AF828502022694689
:10009000F74808F016FA0120CDE72DE9F05FDFF808
:1000A000D083064608EB860090F82550202D1FD0FF
:1000B000A8F180002C4600EB8617A0F50079DFF848
:1000C000B4B305E0A24607EB4A004478202C0AD0DE
:1000D000F8F7B7FC09EB04135A4601211B1D00F089
:1000E000C6FF0028EED0AC4202D0334652461EE096
:1000F000E14808B1AFF30080F8F7A3FC98F82F208F
:100100006AB1D8F80C20411C891A0902CA1701EB00
:1001100012610912002902DD0020BDE8F09F31467E
:10012000FFF7D6FE08B10120F7E733462A46202123
:100130000420FFF7BFFDEFE72DE9F041CC4C256926
:10014000F8F77FFC401B0002C11700EB11600012A2
:1001500000D4FFDF94F8220000B1FFDF012784F80C
:10016000227094F82E00202800D1FFDF94F82E6032
:10017000202084F82E00002584F82F5084F8205089
:1001800084F82150BD4825600078022833D0032828
:1001900031D000202077A068401C05D04FF0FF3000
:1001A000A0600120F8F7AFFB0020F8F7ACFBF8F7F0
:1001B000A3FCF8F79BFCF8F776FB07F039FCB04896
:1001C000056005604FF0E0214FF40040B846C1F8EB
:1001D0008002F2F7E9FD94F82D703846FFF75DFFD5
:1001E0000028FAD0A248803800EB871010F81600DB
:1001F000022802D006E00120CCE73A46314606202C
:10020000FFF72AFD84F8238004EB870090F826008E
:10021000202804D09948801E4078F2F793FE207F72
:10022000002803D0F8F758FC2577657740E590491A
:1002300010B591F82D200024803901EB821100BF08
:1002400011F814302BB1641CE4B2202CF8D3202018
:1002500010BD8C4901EB041108600020C8732146D1
:100260000120FFF7F9FC204610BD10B5012801D090
:10027000032800D171B37E4A92F82D307C4C0022C5
:10028000803C04EB831300BF13F812400CB108202C
:1002900010BD521CD2B2202AF6D3784A48B10228A7
:1002A00007D0072916D2DFE801F01506080A0C0E60
:1002B000100000210AE01B2108E03A2106E0582145
:1002C00004E0772102E0962100E0B5215170107022
:1002D000002010BD072010BD684810B54078F8F721
:1002E0001EFC80B210BD10B5202811D2604991F8D3
:1002F0002D30A1F1800202EB831414F810303BB1D1
:1003000091F82D3002EB831212F81020012A01D04F
:10031000002010BD91F82D2001460020FFF79CFC25
:10032000012010BD10B5F8F78CFBBDE81040F8F7C0
:10033000F6BB2DE9F0410E464D4F01782025803F58
:100340000C4607EB831303E0254603EB4504647872
:10035000944202D0202CF7D108E0202C06D0A142F4
:1003600006D103EB41014978017007E000209FE4CA
:1003700003EB440003EB450140784870424F7EB1E7
:1003800027B1002140F2DD30AFF300803078A04289
:1003900006D127B100214FF47870AFF3008035709B
:1003A00027B1002140F2E530AFF3008001207FE467
:1003B00010B542680B689A1A1202D41702EB146245
:1003C000121216D4497A91B1427A82B92F4A006842
:1003D00052F82110126819441044001D891C081A93
:1003E0000002C11700EB11600012322801DB01206E
:1003F00010BD002010BD2DE9F04781461C48214E5C
:1004000000EB8100984690F825402020107006F5FA
:100410000070154600EB81170BE000BF06EB0410DF
:100420004946001DFFF7C4FF28B107EB44002C70BC
:100430004478202CF2D1297888F8001013E000BF0E
:1004400006EB0415291D4846FFF7B2FF68B988F886
:100450000040A97B99F80A00814201D80020DEE41F
:1004600007EB44004478202CEAD10120D7E40000B7
:1004700058080020FFFF3F0000000000920000200D
:1004800000F50040D805002000000000408A01006F
:100490002DE9FC410E4607460024FE4D09E000BF51
:1004A0009DF8000005EB00108168384600F0F3FD70
:1004B00001246B4601AA31463846FFF79CFF00280D
:1004C000EED02046BDE8FC8170B50446F248012517
:1004D000A54300EB841100EB8510402207F0ACFF30
:1004E000EE4E26B1002140F25F40AFF30080EA48B3
:1004F000803000EB850100EB8400D0F82500C1F8C6
:10050000250026B1002140F26340AFF30080284669
:1005100070BD2DE9FC418446DF481546089C00EB80
:1005200085170E4617F81400012803D0022801D0C1
:100530000020C7E70B46DA4A0121604600F097FD2C
:10054000A8B101AB6A4629463046FFF754FF70B1A7
:10055000D1489DF804209DF80010803000EB8506FE
:100560008A4208D02B460520FFF7A4FB0BE02A4661
:100570002146042014E0202903D007EB41004078F5
:1005800001E096F8250007EB440148709DF8000053
:10059000202809D007EB400044702A46214603205A
:1005A000FFF75AFB01208DE706F8254F0120F07078
:1005B000F3E7B84901EB0010001DFFF7D6BB7CB58F
:1005C0001D46134604460E4600F108022146184611
:1005D000F8F7B2FA94F908000F2804DD1F382072EA
:1005E0002068401C206096B10220AE4951F82610C8
:1005F000461820686946801B20F07F40206094F9EF
:1006000008002844C01C1F2803DA012009E0042048
:10061000EBE701AAF8F790FA9DF8040010B10098F2
:10062000401C00900099206831440844C01C20F010
:100630007F4060607CBD2DE9FE430C46064609788C
:1006400060799072207998461546507241B192486F
:10065000803090F82E1020290AD00069401D0BE050
:10066000D4E90223217903B02846BDE8F043A6E788
:100670008D484178701D084420F07F472179002281
:100680002846A368FFF79BFF3946284600F003FD84
:10069000D4E9023221796846FFF791FF41462846A6
:1006A000019CFFF7F5FE2B4622460021304600F064
:1006B000DEFC002803D13146284600F0ECFCBDE802
:1006C000FE832DE9FE4F814600F0A1FC30B10027EA
:1006D00099F8000020B10020BDE8FE8F0127F7E760
:1006E0006D4D6E4C4FF0000A803524B1002140F270
:1006F000D640AFF3008095F82D8085F823A0002622
:1007000024B1002140F2DB40AFF300801FB9404626
:10071000FFF7DAFE804624B1002140F2E340AFF358
:100720000080F8F78EF943466A464946FFF783FF93
:1007300024B1002140F2E940AFF3008095F82E008B
:1007400020280CD029690098401A0002C21700EB3B
:100750001260001203D5684600F09DFC012624B10A
:10076000002140F2F340AFF3008095F82300002809
:10077000BBD124B1002140F2F940AFF30080F8F77B
:1007800060F96B46464A002100F071FC0028A3D0B6
:1007900027B941466846FFF77BFE064326B1684607
:1007A000FFF7E3FAC9F8080024B1002140F20C5029
:1007B000AFF3008001208FE72DE9F04F89B08B4621
:1007C000824600F024FC344C803428B39BF80000AF
:1007D000002710B1012800D0FFDF304D25B10021E6
:1007E00040F28250AFF300802A49012001EB0A1841
:1007F000A94607905FEA090604D0002140F28A501A
:10080000AFF30080079800F0F9FB94F82D5000201A
:1008100084F8230067B119E094F82E0001272028FE
:1008200000D1FFDF9BF800000028D6D0FFDFD4E71F
:100830002846FFF749FE054626B1002140F29450B4
:10084000AFF3008094F823000028D3D126B1002113
:1008500040F29E50AFF30080F8F7F3F82B4602AA5F
:1008600059460790FFF7E7FE98F80F005FEA060980
:1008700000F001008DF8130004D000214FF4B560A2
:10088000AFF300803B462A4602A9CDF800A00798A6
:100890000CE00000D8050020D80700200000000070
:1008A000FFFF3F00408A010092000020FFF731FE69
:1008B000064604EB850090F828000090B9F1000F7F
:1008C00004D0002140F2AF50AFF3008000F08BFB6A
:1008D0000790B9F1000F04D0002140F2B550AFF3FA
:1008E000008094F82300002884D1B9F1000F04D0CF
:1008F000002140F2BD50AFF300800DF1080C9CE8E0
:100900000E00C8E90112C8F80C304EB35FEA0906C0
:1009100004D0002140F2CA50AFF300800098B843E1
:1009200012D094F82E0020280ED126B1002140F2DA
:10093000CF50AFF300802846FFF7AFFB20B99BF8FC
:100940000000D8B3012849D0B9F1000F04D000212C
:1009500040F2EC50AFF30080284600F03DFB01264A
:100960005FEA090504D0002140F2F550AFF30080A2
:10097000079800F043FB25B1002140F2F950AFF396
:1009800000808EB194F82D0004EB800090F82600D2
:10099000202809D025B100214FF4C060AFF30080BA
:1009A000F9484078F2F7CEFA25B1002140F205600F
:1009B000AFF3008009B03046BDE8F08FFFE7B9F132
:1009C000000F04D0002140F2D750AFF3008094F81C
:1009D0002D2051460420FFF73FF9C0E7002E3FF4D9
:1009E00009AF002140F2E250AFF3008002E72DE9A9
:1009F000F84FE64D814695F82D004FF00008E44C85
:100A00004FF0010B474624B1002140F21360AFF3D1
:100A10000080584600F0F2FA85F8237024B10021D6
:100A20004FF4C360AFF3008095F82D00FFF74CFD45
:100A3000064695F8230028B1002CE4D0002140F2AE
:100A40001E604BE024B1002140F22260AFF3008031
:100A5000CE48803800EB861111F81900032856D1D2
:100A6000334605EB830A4A469AF82500904201D1A5
:100A7000012000E0002000900AF125000021FFF78E
:100A800058FC01460098014203D001228AF8282030
:100A9000AF77E1B324B1002140F22760AFF30080CB
:100AA000324649460120FFF7D7F89AF828A024B12A
:100AB000002140F23260AFF3008000F094FA8346E8
:100AC00024B1002140F23760AFF3008095F8230095
:100AD00038B1002C97D0002140F23B60AFF300808A
:100AE00091E7BAF1000F07D095F82E00202803D126
:100AF0003046FFF7D2FAE0B124B1002140F24F6056
:100B0000AFF30080304600F067FA4FF0010824B1DF
:100B100000214FF4CB60AFF30080584600F06EFA2E
:100B200024B1002140F25C60AFF300804046BDE894
:100B3000F88F002CF1D0002140F24A60AFF3008022
:100B4000E6E70020F7F7B8BE0120F7F7B5BE8E48FC
:100B5000007870472DE9F0418C4C94F82E00202845
:100B60001FD194F82D6004EB860797F82550202DAF
:100B700000D1FFDF8549803901EB861000EB45008D
:100B8000407807F8250F0120F87084F823002946E3
:100B900084F82E50324602202234FFF75DF8002000
:100BA000207004E42DE9F0417A4E784C012538B1EB
:100BB000012821D0022879D003287DD0FFDFF0E77B
:100BC00000F03DFAFFF7C6FF207E00B1FFDF84F89A
:100BD00021500020F7F797FEA168481C04D001239C
:100BE00000221846F7F7E2FE14F82E0F217806EBE4
:100BF00001110A68012154E0FFF7ACFF0120F7F76B
:100C000082FE94F8210050B1A068401C07D014F86F
:100C10002E0F217806EB01110A68062141E0207EA3
:100C2000DFF86481002708F10208012803D00228B8
:100C30001ED0FFDFB5E7A777F7F74EFF98F8000063
:100C4000032801D165772577607D534951F820004D
:100C500094F8201051B948B161680123091A0022A3
:100C60001846F7F7A3FE022020769AE7277698E742
:100C700084F8205000F0E3F9A07F50B198F801000B
:100C800061680123091A00221846F7F78FFE2576BE
:100C900000E0277614F82E0F217806EB01110A6880
:100CA0000021BDE8F041104700E005E0364800783B
:100CB000BDE8F041F2F746B9FFF74CFF14F82E0FEC
:100CC000217806EB01110A680521EAE710B52F4CDF
:100CD00094F82E00202800D1FFDF14F82E0F217881
:100CE0002C4A02EB01110A68BDE8104004211047AC
:100CF0007CB5264C054694F82E00202800D1FFDF55
:100D0000A068401C00D0FFDF94F82E00214901AA02
:100D100001EB0010694690F90C002844F7F70CFF2E
:100D20009DF904000F2801DD012000E0002000995A
:100D300008446168084420F07F41A16094F82100D4
:100D4000002807D002B00123BDE8704000221846F9
:100D5000F7F72CBE7CBD30B5104A0B1A541CB3EB10
:100D6000940F1FD3451AB5EB940F1BD3934203D9AD
:100D7000101A43185B1C15E0954211D9511A08440A
:100D8000401C43420EE00000900000205808002064
:100D900000000000D8050020408A0100FF7F841E6B
:100DA000FFDF0023184630BD012300220146022048
:100DB000F7F7FCBD0220F7F7A6BDF7F742BE2DE915
:100DC000FC47BA4C054694F82E00202800D1FFDFDE
:100DD000642D58D3B64A0021521B71EB010052D347
:100DE00094F82E20A0462046DFF8C89290F82D7087
:100DF00009EB0214D8F8000001AA28446946F7F765
:100E00009BFE9DF90400002802DD0098401C009024
:100E1000A068009962684618B21A22F07F42B2F5C3
:100E2000800F30D208EB8702444692F82520202A12
:100E30000AD009EB02125268101A0002C21700EB26
:100E40001260001288421EDBA068401C10D0F7F729
:100E5000F8FDA168081A0002C11700EB116000122A
:100E6000022810DD0120F7F74EFD4FF0FF30A060A3
:100E700020682844206026F07F402061012084F80B
:100E80002300BDE8FC870020FBE72DE9F047874CF5
:100E9000074694F82D00A4F1800606EB801010F8A8
:100EA000170000B9FFDF94F82D50A046824C24B102
:100EB00000214FF40760AFF3008040F67C0940F654
:100EC000850A06EB851600BF16F81700012818D012
:100ED000042810D005280ED006280CD01CB1002103
:100EE0004846AFF3008020BF002CEDD000215046D3
:100EF000AFF30080E8E72A4639460120FEF7ACFE52
:100F0000F2E74FF0010A4FF00009454624B10021F5
:100F100040F68C00AFF30080504600F06FF885F883
:100F2000239024B1002140F69100AFF3008095F8A2
:100F30002D00FFF7C9FA064695F8230028B1002CCA
:100F4000E4D0002140F697001FE024B1002140F6D4
:100F50009B00AFF3008005EB860000F127013346CC
:100F60003A462630FFF7E5F924B1002140F69F000C
:100F7000AFF3008000F037F8824695F8230038B1CF
:100F8000002CC3D0002140F6A500AFF30080BDE7E0
:100F900085F82D60012085F82300504600F02EF8DA
:100FA000002C04D0002140F6B200AFF30080BDE871
:100FB000F08730B504463D480D4690F82D003B497A
:100FC000803901EB801010F8140000B9FFDF3948B8
:100FD00000EB0410C57330BD344981F82D000120A9
:100FE00081F82300704710B5344808B1AFF3008092
:100FF000EFF3108000F0010072B610BD10B50028AC
:1010000004D12F4808B1AFF3008062B610BD2D485F
:101010000068C005C00D10D0103840B2002804DBB5
:1010200000F1E02090F8000405E000F00F0000F16E
:10103000E02090F8140D400970470820704710B563
:101040001A4C94F82400002804D1F7F7E9FD012098
:1010500084F8240010BD10B5144C94F82400002826
:1010600004D0F7F706FE002084F8240010BD10B568
:101070001C685B68241A181A24F07F4420F07F4013
:10108000A14206D8B4F5800F03D2904201D80120C6
:1010900010BD002010BDD0E90032D21A21F07F43EC
:1010A000114421F07F41C0E9003170475808002009
:1010B000FF1FA107D805002000000000000000006D
:1010C0000000000004ED00E02DE9F0410446800737
:1010D0004FF000054FF001060CD56B480560066027
:1010E00006F02FFB20B16948016841F4806101607E
:1010F00024F00204E0044FF0FF3705D56448466051
:10110000C0F8087324F48054600003D5614805607A
:1011100024F08044E0050FD55F48C0F80052C0F8C5
:1011200008735E490D60091D0D605C4A04210C3294
:101130001160066124F48074A00409D55848466003
:10114000C0F80052C0F808735648056024F40054F3
:10115000C4F38030C4F3C031884200D0FFDF14F400
:10116000404F14D050484660C0F808734F4886601E
:10117000C0F80052C0F808734D490D600A1D166092
:101180008660C0F808730D60166024F440442005A2
:101190000AD5484846608660C0F80873C0F84873AE
:1011A0004548056024F4006406F01CFC43480442F2
:1011B00000D0FFDFBDE8F081F0B50022202501233B
:1011C0004FEA020420FA02F1C9072DD051B20029DA
:1011D00010DB00BF4FEA51174FEA870701F01F06E7
:1011E00007F1E02703FA06F6C7F88061BFF34F8FD7
:1011F000BFF36F8F0CDB00BF4FEA51174FEA870731
:1012000001F01F0607F1E02703FA06F6C7F880622F
:1012100004DB01F1E02181F8004405E001F00F0159
:1012200001F1E02181F8144D02F10102AA42C9D373
:10123000F0BD10B5224C20600846F7F708FE206884
:10124000FFF742FF2068FFF7B7FF06F007F800F04E
:101250001AF906F0C7FB06F012FBF1F73FFEBDE8F6
:10126000104006F0ABB810B5154C2068FFF72CFF06
:101270002068FFF7A1FF06F0B5FBF7F7A0FE0020FE
:10128000206010BD0A207047FC1F00403C17004042
:1012900000C0004004E5014000800040048500409B
:1012A00000D0004004D5004000E0004000F00040C5
:1012B00000F5004000B0004008B50040FEFF0FFD03
:1012C0009400002070B526490A680AB3002215462A
:1012D00001244B685B1C4B60092B00D34D600E79D9
:1012E00004FA06F30E681E420FD0EFF3108212F0DC
:1012F000010272B600D001220C689C430C6002B956
:1013000062B649680160002070BD521C092AE0D312
:10131000052070BD4FF0E0214FF48000C1F80002BD
:101320007047EFF3108111F0010F72B64FF0010218
:1013300002FA00F20A48036842EA0302026000D19E
:1013400062B6E7E70648002101604160704701216D
:10135000814003480068084000D001207047000029
:10136000980000200120810708607047012188074C
:1013700041600021C0F800111848017070471749FA
:101380000120087070474FF08040D0F8000101281C
:1013900003D012480078002800D001207047104880
:1013A0000068C00700D0012070470D480C3000686D
:1013B000C00700D00120704709481430006870470A
:1013C000074910310A68D20306D5096801F0030104
:1013D000814201D10120704700207047A000002009
:1013E00008040040002101700846704701460020B3
:1013F00008707047EFF3108101F0010172B60278B6
:10140000012A01D0012200E000220123037001B96A
:1014100062B60AB1002070474FF400507047E9E708
:10142000EFF3108111F0010F72B64FF0000202705D
:1014300000D162B600207047F2E700002DE9F041CC
:1014400015460E460446002700F0E7F8A84215D3DB
:10145000002341200FE000BF94F84220A25CF25428
:1014600094F84210491CB1FBF0F200FB12115B1C16
:1014700084F84210DBB2AB42EED3012700F0D9F87A
:101480003846BDE8F081704910B5802081F800042D
:101490006E49002081F8420081F84100433181F813
:1014A000420081F84100433181F8420081F8410057
:1014B0006748FFF797FF6648401CFFF793FFF1F777
:1014C0007FFCBDE8104000F0B4B8402070475F4892
:1014D00000F0A3B80A4601465C48AFE740207047D9
:1014E0005A48433000F099B80A46014657484330FD
:1014F000A4E7402101700020704710B5044653480E
:10150000863000F08AF82070002010BD0A4601469F
:101510004E4810B58630FFF791FF08B1002010BD8E
:1015200042F2070010BD70B50C460546412900D9AE
:10153000FFDF48480068103840B200F050F8C6B2EB
:101540000D2000F04CF8C0B2864203D2FFDF01E06C
:10155000F1F77EFC224629463C48FFF76FFF002842
:10156000F6D070BD2DE9F041394F002506463F1DEC
:1015700057F82540204600F041F810B36D1CEDB23D
:10158000032DF5D33148433000F038F8002825D03A
:101590002E4800F033F8002820D02C48863000F088
:1015A0002DF800281AD0F1F731FC2948FFF722FF67
:1015B000B0F5005F00D0FFDFBDE8F0412448FFF741
:1015C0002FBF94F841004121265414F8410F401CCC
:1015D000B0FBF1F201FB12002070D3E751E70028C5
:1015E00004DB00F1E02090F8000405E000F00F00BB
:1015F00000F1E02090F8140D4009704710F8411FE9
:101600004122491CB1FBF2F302FB131140788142E5
:1016100001D1012070470020704710F8411F407829
:10162000814201D3081A02E0C0F141000844C0B26F
:10163000704710B50648FFF7DDFE002803D1BDE86E
:101640001040F1F7CEBB10BD0DE000E0880800208F
:10165000A400002004ED00E070B5154D2878401C72
:10166000C4B26878844202D0F1F735FC2C7070BDAA
:101670002DE9F0410E4C4FF0E02600BFF1F729FCB8
:1016800020BF40BF20BF677820786070D6F8005236
:10169000EFF79CFE854305D1D6F8040210B92078F7
:1016A000B842EBD0F1F714FC0020BDE8F081000057
:1016B000B40000202DE9F041012528034FF0E0217E
:1016C0000026C1F88001BFF34F8FBFF36F8F1F4C0F
:1016D000C4F800610C2000F02CF81D480168026875
:1016E000C94341F3001142F010020260C4F80453F0
:1016F0002560491C00E020BFD4F80021002AFAD060
:1017000019B9016821F0100101601248076865608D
:10171000C4F80853C4F800610C2000F00AF83846F9
:10172000BDE8F08110B50446FFF7C4FF206000203B
:1017300010BD002809DB00F01F0201219140400983
:10174000800000F1E020C0F88012704700C0004027
:1017500010ED00E008C500402DE9F047FF4C0646BB
:10176000FF21A06800EB061211702178FF2910D02C
:101770004FF0080909EB011109EB06174158C05950
:1017800000F0F4F9002807DDA168207801EB0611CC
:1017900008702670BDE8F08794F8008045460DE09B
:1017A000A06809EB05114158C05900F0DFF9002885
:1017B00006DCA068A84600EB08100578FF2DEFD1E5
:1017C000A06800EB061100EB08100D700670E1E751
:1017D000F0B5E24B0446002001259A680C269B7860
:1017E0000CE000BF05EB0017D75DA74204D106EB64
:1017F0000017D7598F4204D0401CC0B28342F1D8A1
:10180000FF20F0BD70B5FFF7D8FAD44C0825227838
:10181000A16805EB0212895800F0A8F9012808DD3B
:101820002178A06805EB01114058BDE87040FFF732
:10183000BBBAFFF78CF9BDE87040F1F783BB2DE927
:10184000F041C64C2578FFF7B8FAFF2D6ED04FF067
:101850000808A26808EB0516915900F087F90228DC
:10186000A06801DD80595DE000EB05110978217069
:10187000022101EB0511425C5AB1521E42548159BA
:1018800001F5800121F07F4181512846FFF764FF77
:1018900034E00423012203EB051302EB051250F898
:1018A00003C0875CBCF1000F10D0BCF5007F10D9DD
:1018B000CCF3080250F806C00CEB423C2CF07F4CF5
:1018C00040F806C0C3589A1A520A09E0FF21815411
:1018D0000AE0825902EB4C3222F07F428251002210
:1018E00042542846FFF738FF0C21A06801EB051190
:1018F0004158E06850F82720384690472078FF2864
:1019000014D0FFF75AFA2278A16808EB0212454674
:10191000895800F02BF9012893DD2178A06805EBA8
:1019200001114058BDE8F041FFF73EBABDE8F08133
:10193000F0B51D4614460E460746FF2B00D3FFDFC9
:10194000A00700D0FFDF8548FF210022C0E9024741
:10195000C57006710170427082701046012204E069
:1019600002EB0013401CE154C0B2A842F8D3F0BD12
:1019700070B57A4C064665782079854200D3FFDF42
:10198000E06840F825606078401C6070284670BDB3
:101990002DE9FF5F1D468B460746FF24FFF70DFA32
:1019A000DFF8B891064699F80100B84200D8FFDF89
:1019B00000214FF001084FF00C0A99F80220D9F8E5
:1019C00008000EE008EB0113C35CFF2B0ED0BB42F6
:1019D00005D10AEB011350F803C0DC450CD0491CBB
:1019E000C9B28A42EED8FF2C02D00DE00C46F6E7D1
:1019F00099F803108A4203D1FF2004B0BDE8F09F9C
:101A00001446521C89F8022008EB04110AEB041258
:101A1000475440F802B00421029B0022012B01EB45
:101A200004110CD040F801204FF4007808234FF047
:101A3000020C454513D9E905C90D02D002E0455015
:101A4000F2E7414606EB413203EB041322F07F42FA
:101A5000C250691A0CEB0412490A81540BE005B913
:101A6000012506EB453103EB041321F07F41C15002
:101A70000CEB0411425499F800502046FFF76CFE1D
:101A800099F80000A84201D0FFF7BCFE3846B4E741
:101A900070B50C460546FFF790F9064621462846E4
:101AA000FFF796FE0446FF281AD02C4D082101EBC3
:101AB0000411A8684158304600F058F800F58050ED
:101AC000C11700EBD14040130221AA6801EB0411B9
:101AD000515C09B100EB4120002800DC012070BD01
:101AE000002070BD2DE9F04788468146FFF770FE63
:101AF0000746FF281BD0194D2E78A868314634467A
:101B000005E0BC4206D0264600EB06121478FF2CF6
:101B1000F7D10CE0FF2C0AD0A6420CD100EB01104B
:101B200000782870FF2804D0FFF76CFE03E0002047
:101B300030E6FFF73FF941464846FFF7A9FF01238A
:101B4000A968024603EB0413FF20C854A878401E7E
:101B5000B84200D1A87001EB041001E05409002044
:101B600001EB061100780870104613E6081A00020F
:101B7000C11700EB116000127047000045480021BA
:101B80000170417010218170704770B5054616468E
:101B90000C460220F1F7D4F83E490120F61E0870E9
:101BA0003D4806603C4808380560001F046070BD71
:101BB00010B50220F1F7C4F836490120087000F092
:101BC00051F836494FF40000086010BD10B5314C93
:101BD000207888B131494FF40000091D086000F0F9
:101BE0004AF8002120B1012060702D48006801E012
:101BF00061701020A0702170BDE810400020F1F746
:101C00009FB8244810B5017859B12648D0F8000192
:101C100028B100F030F8002800D0012010BD0220CB
:101C200010BD407810BD10B5C824641EE4B2FFF7A3
:101C3000E8FF022803D0012800D0002010BD002CAE
:101C4000F3D1FFDFF9E7134810B5017841B100F097
:101C500012F818B112480068C0B210BD102010BDB3
:101C6000807810BD0F480021C0F80011C0F80411A1
:101C7000C0F8081170470B48D0F8001129B1D0F80E
:101C8000041111B1D0F8080108B1002070470120FB
:101C900070470000B600002010F5004004F5014038
:101CA00000F4004000F000404948002101704170FC
:101CB000704770B5064614460D460120F1F740F80E
:101CC00044480660001D0460001D056070BD2DE9DC
:101CD000F04105460C463E483E4901260670091F64
:101CE00045EA0240086005F002FD10B9394810309D
:101CF0000460394C0027C4F8047138494FF0407033
:101D0000086065B1012D00D0FFDFC4F800722660C5
:101D100032494FF00070091F0860BDE8F081C4F837
:101D200000622660F9E72A48017871B12B4A4FF02A
:101D3000407111602849D1F8042100211AB1284AC4
:101D40001268427000E0417001700020F0F7F8BFA7
:101D50001F48017841B12048D0F80401002802D082
:101D60001F480068C0B270474078704770B50028BF
:101D700028D01748007800B9FFDF1748D0F80411C1
:101D800000291FD10223C0F8043316490A680C68E1
:101D9000D24342F3001244F010040C609C034FF055
:101DA000E025521C03E000BFC5F8804220BFD0F8F8
:101DB0000461002EF8D01AB90A6822F010020A60F5
:101DC000C0F8083370BD04490120886070470000E6
:101DD000B900002008F5004000F0004008F501407F
:101DE00000F4004010ED00E038B5FC4D0024C5F8CB
:101DF0000041C5F80C41C5F81041C5F80441C5F8CB
:101E00001441C5F8184105F08AFC08B1C5F828410D
:101E1000F3480068009038BD70B5F24D00246C7036
:101E20002C7000F0D2FD85F82540EC62092105F107
:101E30001800AC6306F0A1FBEB49601E0860091DA9
:101E40000860091D0C60091D0860091D0C60091D52
:101E50000860091D0860091D0860091D0860091D4A
:101E60000860091D0860091D0860091D0860091D3A
:101E7000086070BDDD4800B5016801F00F0103295D
:101E800005D0006800F00F00042802D0FFDF012019
:101E900000BD022000BD10B5D24C0168A1614168AF
:101EA000E161007A84F82000207E50B1207FF9F7AC
:101EB000DFF9A07E08B1012100E00021207FF9F7C1
:101EC000CCF9607E00280CD0607FF9F7D1F9E07E74
:101ED00008B1012100E00021607FBDE81040F9F762
:101EE000BCB910BD00F078BD10B500F075FDBB4861
:101EF000D0F80001002800D0FFDF10BD70B5012030
:101F000000F045FDBA48002505600126066005F091
:101F100018FCB84C18B1206840F48060206005F0CF
:101F2000E6FB28B12068B44920F077000843206020
:101F300005F0F5FB38B1AF48001D016821F47F4181
:101F400041F4B0510160AB49AC483C31086005F048
:101F5000E6FBA44C60B1A5490220503184F8210071
:101F60000860A849A64808609D481030091F08600D
:101F70004FF01020806C411C05D09C497C310A68D0
:101F800060F317420A60994940F25B6028310860AB
:101F9000091F40F203100860081F066093490320E0
:101FA00008609448EC38066094F8211011B14FF4A1
:101FB000C02100E09449934A41F46021943A1160B1
:101FC0008F49904A091F0832116085490839121F4C
:101FD0001160016821F440710160016841F4807171
:101FE0000160012000F0E4FC7C491020C1F80403EA
:101FF00084F83150E56270BD7E483830016821F0C8
:10200000010141F0807101607047764A0368C2F8AF
:1020100002308088D08011727047724890F8250095
:102020007047704A517010707047F0B505468400D3
:102030006A488B882044C0F820360B78D1F801100C
:1020400043EA0121C0F8001605F108000127694C98
:1020500007FA00F6FC3C52B1012A00D0FFDF2068ED
:10206000304320602068AF4038432060F0BD2068D6
:10207000B043F6E705F0FCBD5A4890F832007047CF
:102080005A4AC178143211600068584900020C3174
:1020900008607047252807D0262807D0272807D0B2
:1020A0000A2807D8042206E0022107E01A2105E0E9
:1020B000502103E0062202EB4001C9B24B4A083A24
:1020C00011604A494431086070474648817A0129C5
:1020D00017D0022914D1417E002911D0827F01211D
:1020E000C37F01FA02F299400A43464994390A60D3
